:020000040000fa
:080000000014040000000000e0
:020000040000fa
:102800008f622100007f240000018800000000008a
:102810000c00070040c52600010020001100070041
:10282000000020000000e000020032000000020072
:1028300000000000d26f0200000000000040da003b
:102840000000fe004440a900c01f21000000e0007d
:102850000300320000002000a00188004440a800ce
:102860000000060091018800800078000000eb0065
:1028700015003700e280400032a0b4009101ba0098
:10288000e280400032a0b4009102ba00e280400031
:1028900032a0b4000002eb00472bde00f507b200c7
:1028a000602ce10004003a000059eb008301e900cc
:1028b000fdff3e00040037006128e1000100320006
:1028c0000082eb00040007001101ba000200e000e2
:1028d000e8ff3a00000006003159ba008301e90020
:1028e0000c0032002159ba008301e90008003200cf
:1028f0000400e00003003a00e280400032a0b4008f
:10290000f5ff370011d9ba008301e900faff3a0058
:102910008100e800e180400032a0b4000000060021
:102920000e600400000000001e60040000000000b3
:102930002e600400000000003e6004000000000063
:102940005860040000000000fe6004000000000069
:102950000a610400000000003e6104000000000065
:10296000b062040000000000da6204000000000011
:10297000f86204000000000004630400000000008e
:102980002a630400000000005063040000000000ff
:1029900076630400000000009c6304000000000057
:1029a000c263040000000000e863040000000000af
:1029b00070640400000000000e64040000000000c9
:1029c00080640400000000008c640400000000002b
:1029d0009e64040000000000086504000000000080
:1029e0006065040000000000ae6504000000000007
:1029f000b865040000000000c2650400000000008b
:102a0000f4650400000000002666040000000000d9
:102a10004e66040000000000746604000000000020
:102a2000e2670400000000001668040000000000d7
:102a30002e6804000000000046680400000000004a
:102a40005e680400000000007668040000000000da
:102a50008e680400000000007a17040000000000e7
:102a6000a817040000000000fc2104000000000082
:102a7000f821040000000000000004000000000035
:102a8000000178001001e200030035001061a80089
:102a9000000028001021b7003008800041088000a5
:102aa0000200e000010032000089be0000000600c4
:102ab000800078001106b100030035009101b100db
:102ac00001003c000050a100000006000003b1001e
:102ad0000b0035009000b100080034008000b10008
:102ae000070035009001b100040034007000b1000f
:102af000030035009001b10001003c00100005000a
:102b0000000005000400fa00889fbe00d06f80001e
:102b10000000e0000100320000000100405380008e
:102b20000000e0000100320000000100b06f8000f2
:102b30000000e0000100320000000100915480001c
:102b4000c06f8000810f50002f0032001104e000a0
:102b500002003a00d20107009054880066815700b5
:102b60002100200090548000290207000004780012
:102b7000a2002000e8805700450207000001be00c7
:102b8000906f8800a16f88004fb8970088005000b0
:102b90005fb89700808f500009003a00c0ae2f0048
:102ba000f1ff2f00800f5100818f59000400340085
:102bb00030512000800f5100e08f59000300340095
:102bc0006000b800906f8800a16f8800986f800047
:102bd000a96f800042062000030020000800be000c
:102be000a9170700820220000300200065160700d5
:102bf0000800500089805800906f8800a16f8800fd
:102c000090548000c06f880042fc2f00f3ff2f001b
:102c1000906f8000a16f80005a1607004f04be001d
:102c20000080fa0000000600889fbe001004be006d
:102c3000b4ff070008014000898148008080eb0054
:102c40000000eb00770207004f04be000000060002
:102c50001000fa00889fbe008a9fbe008c1f78007b
:102c600000067800c0019000c20020001100090099
:102c70008201d800000178006c10b90080815100f9
:102c800002003b00ec8141000201e9000200e0008b
:102c900006003d000000280002005000dc0090000b
:102ca000808f500008003d007a0037000200e000ed
:102cb00005003200f0ff270002005000dc00900009
:102cc000810f5000730035005c049000080441003f
:102cd0008300780008007800360207000000e90051
:102ce000cf80de0001017800820178000418250001
:102cf000150020006033b80072170700f0b79f007e
:102d000081bf9f0092bf9f00a3bf9f00cfc4de0082
:102d1000090578008a05780004382300151e200074
:102d20006033b8000800be000a01be006517070046
:102d30007fb297008fba97001fbb9700afbb970079
:102d40000404400085844800060549008785490041
:102d50003c009000cf80de00010178008201780005
:102d600004182500150020006033b800551707002f
:102d700008044000898448000a0549008b85490001
:102d8000b8b79f00c9b79f00dab79f00ebb79f00a5
:102d90002c009000cf80de000101780082017800d5
:102da00004e12000050020006033b800451707004b
:102db0000205be000004be001c009000cf80de00b3
:102dc0000101780082017800c40320000500200082
:102dd0006033b8003b1707000804400089844800ae
:102de0000a0549008b8549001c007800cf80de0071
:102df00001017800820178000804400089844800bd
:102e00000a0549008b8549003fb09700cfb0970075
:102e10005fb19700efb197000004440081844c003b
:102e200002054d0083854d000800be000a01be006a
:102e3000521707006011b8008c1707000000e0006f
:102e4000140035000805be0000e82700a13a28005c
:102e50000004540081845c008c0890000801be00ce
:102e60000c007800ef0107000c0890000000e00063
:102e70000400340000c92800a13a280000045500cd
:102e800081845d001fff07000000540081805c000a
:102e9000020037000080eb008080eb004f067800d6
:102ea0004f05be004f04be000080fa00000006007f
:102eb0000418280055c527000201420083814a00fa
:102ec0000000420081804a00800f5100818f59002c
:102ed00003003c000200500083805800bf153700fb
:102ee0000000510081805900bc15070001f0a200cc
:102ef00000000600881f780002047800cc0007005c
:102f0000080040004f047800000006000000fa00ae
:102f1000881f7800000478003fb99700ea815700c5
:102f200080007800a0772100390207008000780037
:102f30000000e000020035000040eb0000f47800e3
:102f4000010078004f0478000080fa0000000600bd
:102f5000900178000200e00002003a000308e90056
:102f6000050037008080eb001304e000020032000f
:102f70000308e8009300fb00010078000000060051
:102f80000200fa00f0bf9f003fb99700ea815700a6
:102f90008f80e900807a2100d60207000080fa00c5
:102fa00000000600ec874700889fbe008a9fbe0095
:102fb0008c9fbe008e1f7800f0b79f0081bf9f00de
:102fc0008204780000047800010037000804e8005b
:102fd000184778000e00fb008e0307000000e00099
:102fe000faff3a00d0c2b300804f5700050032000c
:102ff00000c0e900804f570002003200004778000f
:10300000010037000804e8000900e0004500350031
:10301000e18f54004300320040022000808f5400b2
:1030200040003c000900e0000e003400f08f540026
:103030001a003a0000c3b300984f100016003a007f
:103040009840900080c7b30080cf5000030032004a
:1030500080c5b30080cf50000f003a000884e8001c
:103060000e003700a900200000c3b300984f1000e5
:103070000a003a009840900080c7b30080cf50000b
:10308000040032008900200080c5b30080cf5000ca
:1030900002003a000884e8000901200008057800d1
:1030a00000c3b300010037000a05e8009a4f100082
:1030b000fdff32008a0578006066b8000e00370018
:1030c00090bf200000425200c4ef9f006149b90048
:1030d0000c00be002b1507004fea97000401fb000f
:1030e000cf91de008b05e800ccb79f00ddb79f00d5
:1030f00000064100818649001b00fb004d030700cc
:10310000800078000901780090bf2000500307007c
:10311000000278000000e000e9ff3a008b0f540045
:1031200006003a000fb897000000e00029003200c6
:10313000ffb0970001087800260037008a8055000c
:1031400040bd200060c07c000000fb0000805000fb
:10315000160033004240a9000f003c004fe99700e1
:103160000200fb00cf80de000000560081805e0080
:10317000800f5600818f5e00070039006149b90059
:10318000061507004fb19700dfb19700820f50007e
:10319000838f58000500320020022000e070880074
:1031a0000086eb008086eb0005003700d0c2b3003c
:1031b000804f570002003a0060061600e0861e00ad
:1031c0008fb997000300e000030032008b097800fc
:1031d000010037006066b8000c00be004f077800a1
:1031e0004f06be004f05be004f04be00cf00b10029
:1031f000000006008001780000017800010037001f
:103200000201e8001204e000fdff3a00020037006e
:103210000201e8008100e8001140780000497800d0
:103220000004e000faff3a00030078000000060006
:103230008001eb000200370061f079008301e800b3
:10324000828f5100fcff3a000000060040538000ce
:103250000000e0000100320000000100a0a62000f4
:1032600000000600881f780000047800206c8000b1
:103270000000e0000100320000000100a4ba2000bc
:103280008801780022e12000a101200060d8200000
:10329000d703070060d820004f0478000000060024
:1032a000889fbe008a1f780080e120001004e000a3
:1032b00053003a00a0dd20008c140700b070880095
:1032c0000000e00046003a0030de200087140700ce
:1032d000b07088000000e000410032000004780077
:1032e0007adb2000984478000900fb002f040700d7
:1032f0000000e00038003200094d78000801780035
:1033000032407800404598000a05e800a0db200024
:10331000800f55000200320002047800f1ff3700f0
:1033200092407800d0c2b30080cf50000500320038
:1033300000c0e90080cf50000200320080407800d9
:10334000010037000881e800f0db20000148780028
:10335000924078000100fb0003fd2f0003004000b5
:10336000e90f50001c003e0000dc200001487800fe
:10337000924090000100fb0003004000e90f500064
:1033800015003e0010dc2000014878000284e800af
:103390001800fb00050407000000e0000b003200ed
:1033a000badb2000984478000900fb00ff03070007
:1033b0000000e00008003200095d78000804e80021
:1033c000e0db2000800f5500f6ff3a0060db2000b4
:1033d0001804e000010032000000eb00b07088002b
:1033e000b07080000000e00002003a00a06d800094
:1033f000b070880021c0b30080e12000014878004f
:10340000b07080004f0578004f04be000000060039
:10341000889fbe008a9fbe000004be00820578001f
:10342000104578000a04e000010032000004e800c2
:103430008a00fb00080078009a0207000000e00004
:1034400003003a0008007800e2030700000044008f
:103450000900e00002003c00880d50000800370021
:103460001004e00003003a00800deb000004780037
:10347000030037008904e9000004e800ecff37008e
:10348000080078004f05be004f04be000000060093
:103490000200fa00889fbe008a9fbe008c1f780041
:1034a0008005780001057800020678000100e00040
:1034b00001003a006c8557000b04780001003700ca
:1034c0000804e800984478000900fb005102070056
:1034d0000000e000faff3a00d0c2b30080cf5400f1
:1034e0000500320000c0e90080cf54000200320025
:1034f00080447800010037000804e8000c017800df
:103500008a00780008007800a6fe07000001be00cf
:103510009a0f540001003a000b0d78009a8f550065
:1035200003003a00e00f5100e08f59000f003a000d
:10353000b0c2b30080cf540004003a00e00f510045
:10354000e08f590015003d0008003700d0c2b300dd
:1035500080cf540011003a00000020000100280034
:10356000800f5100818f59000a0036002002200090
:10357000e070880002002000030028006b4040003b
:1035800080cf540005003200f2ff2f00f3ff270028
:103590000200370060011100e08119000200be0046
:1035a0004f0678004f05be004f04be000080fa00b1
:1035b0000000060080017800010278000000e000b1
:1035c000060034000000e90042002000110009005c
:1035d0000200d80000017800080037000001eb006d
:1035e000e40f400005003c00640010004200200091
:1035f000110009000200d8000001e80063806100aa
:1036000003003a0021ce20000300e00001003a0050
:10361000a1cf200004004200010040001000410042
:10362000000006000800fa00889fbe008a9fbe00c6
:103630008c1f7800000678000104780000e827005d
:10364000a13a28000201400083814800f2b79f00a0
:1036500083bf9f000c00e00005003a00906d8000e1
:103660000cda20000000e000010032000000010040
:10367000080e98007fb097008fb8970090bf9f000a
:10368000a1bf9f0002182500130020001fb897005b
:10369000afb89700c11307000005be0061004000ed
:1036a000e080480072002000030020007115070030
:1036b00060069800d2162000030020000a00be0019
:1036c000f114070000047800010037000804e90045
:1036d0008000eb0008007800b6ff07006101b90028
:1036e000d016200000c0b9000200400083804800ce
:1036f000800f5500818f5d00f4ff350000015500fb
:1037000081815d00580698000203780072069800d7
:103710006300640003003a0020ce20000800e000af
:1037200001003a00a0cf200076024000c500200032
:103730008502e90024007800cf80de00800f510070
:10374000818f5900faff350045069800140090005b
:10375000000053000000e800300698000218250021
:10376000130020001fb89700afb89700501507004e
:103770000004be0002e120000300200087130700c0
:103780002006980002e12000030020000800be008f
:10379000471507000004be00c203200003002000fc
:1037a0007e13070010069800c203200003002000cb
:1037b0000800be003e150700000e78000c089000bf
:1037c0000000e0000c003d000c007800150307002d
:1037d000000e98000000e0000700340000e1200027
:1037e000010020007fb197008fb9970002004000d0
:1037f00083804800a1ff37000c0078004f06780056
:103800004f05be004f04be000080fa000000060015
:103810006200fa00889fbe008a9fbe000004be00be
:10382000020578008300780060f92f000f00400047
:103830009701070088979f0099979f000000eb0071
:10384000a09f9f009a4578000b80fb000000ea00d3
:10385000cf04de0050c2b30080cf5500020032001a
:1038600009047800010037000904e9000800e000bd
:103870000b0034001f909700080178008a00780040
:103880008f9197000300010090979f000000e000d7
:10389000930032002f98970000004400a09f9f00e3
:1038a0000905450050c2b30080cf55000400320026
:1038b0000b04e000e3ff3a002f98970089003700df
:1038c0000000eb00809f9f00f0979f00e0979f0013
:1038d000d0979f00c0979f00b0979f00c09f9f0008
:1038e0000900370020dd200000805000000040006b
:1038f00061dc2000e10078004f9897000100700023
:10390000c09f9f000a05e8001a4478008800fb0069
:1039100020dd200063010700800078000000e00047
:10392000f0ff3a00a0c2b300804f54000e003a00ee
:10393000bf8897000180e900b08f9f0010007800d9
:10394000b09f9f000000e00005003d000000ea007d
:10395000b09f9f004f9897000020a000c09f9f003d
:103960000a05e80010003700b19f9f0003fd2f00fb
:10397000f4ff2700080037003f989700840f50009d
:10398000040032006a00b90000004100030040005a
:10399000b09f9f000a05e8001a01fb0003004100e8
:1039a000e90f5000f4ff3600e0c2b3009a4f100058
:1039b000040032000080eb00909f9f008a04780092
:1039c0001c0037008a04e800a0c2b300994f100021
:1039d00007003a00bf8897000180e900b08f9f0080
:1039e00010007800909f9f008a84e8001100370043
:1039f0000000eb00909f9f0003fd2f00f4ff2700c5
:103a0000080037001f989700840f50000400320010
:103a10006a00b9000000410003004000909f9f0031
:103a20008904e8001901fb0003004100e90f500080
:103a3000f4ff3600194478008800fb00c0df200046
:103a4000180107000000e00002003a00004478007e
:103a5000010037008904e800a87f9f0080c6b300fa
:103a6000804f540004003a00994f14000a003a00b5
:103a70006640500006003700c0c6b300804f5400b7
:103a800005003a00994f140003003a0065404000d9
:103a9000a07f9f008904e8000905e800c8fb2f000b
:103aa0000f04440060f92f000f0040008085e800fb
:103ab0008801780019417800800078000b007800b8
:103ac000dc0207000000e00005003a0088007800f2
:103ad0000b007800fc0007000000e00059ff3d00eb
:103ae0000080eb004f05be004f04be000080fa00ce
:103af000000006001200fa00889fbe008a9fbe00e8
:103b00008c1f780002047800a0b79f00b1b79f0017
:103b10008300780078805700dd0007000000eb008c
:103b2000e0b79f00d8b79f0000067800dfb4970089
:103b3000194578000a80fb000000ea00cf05de008e
:103b40000a00fb00b30007000000e0001a0032008a
:103b50006fb097000000e800e0b79f003fb097000b
:103b6000120020008000eb00afb1970003000100bd
:103b700000047800a7000700000178000000e000c2
:103b8000f3ff3a006fb09700e10f440007003200e6
:103b90000000e900e0b79f003fb097008800780080
:103ba000afb1970003000100230037000000e900d7
:103bb000e0b79f002000370050c2b300804f55008f
:103bc000020032000b047800190037000b04e900f2
:103bd000170037006fb097000000e800e0b79f00c3
:103be0003fb09700120020008000eb00afb19700bb
:103bf00003000100800078001900fb00808f500056
:103c00000a003200e18f40007c0032006fb0970064
:103c10000000e900e0b79f003fb097000001eb0013
:103c2000afb1970003000100740037008904e80079
:103c30000804e900e7ff3b005fb097008080450083
:103c4000d1b79f0050c2b300804f5500030032002f
:103c50000a04e000b5ff3a0068003700a2c2b300d2
:103c60000040eb00914f110003003a000100e80012
:103c7000d0b79f0002407800a0f79f000000eb0043
:103c800080bf9f0003fd2f00f4ff27000a003700cc
:103c90000fb89700840f5000040032006a00b9008a
:103ca000000041000300400080bf9f005fb097000c
:103cb0000000e800d0b79f00dfb4970019447800f7
:103cc0000801fb0003004100e90f5000f0ff36003f
:103cd0008200780060de2000720007000000e00033
:103ce00002003a0000447800020037000900e800b2
:103cf000d0b79f00b8f79f0080c6b300804f540034
:103d000005003a00dfb09700914f14000c003a0014
:103d10006640500007003700c0c6b300804f540013
:103d200007003a00dfb09700914f140004003a00fa
:103d300065404000b0f79f000100e800d0b79f0049
:103d40005fb097009000fb00d0de20005500070018
:103d50000000e00019003a006fb097000000e80092
:103d6000e0b79f003fb09700120020008000eb00fa
:103d7000afb19700030001000004780025000700a0
:103d8000000178000000e000f3ff3a006fb09700f8
:103d9000e10f4400070032000000e900e0b79f0097
:103da0003fb0970088007800afb197000300010092
:103db000020037000000e900e0b79f007c80570058
:103dc000990307000000e00003003c000c00e00045
:103dd00009003200090037004ff097000004e000ae
:103de000010032000c06e8005fb097000000e80018
:103df000d0b79f004dff3700000678000c00780018
:103e00004f0678004f05be004f04be000080fa0048
:103e1000000006006900e100040035006d00e100cb
:103e2000030034000002b100010032000000050070
:103e300010000500800078001104b1000300350077
:103e40009101b10001003c000050a00000000600fc
:103e50008001eb00040037008301e80090cf1000e0
:103e6000040032000000e800828f5100faff3a009f
:103e70000000eb0000000600d07080000000e000b1
:103e80000100320000000100c0e120000000060037
:103e90000200fa00f1bf9f00010878000080fa00dc
:103ea00000000600040037000204e00001003a00b0
:103eb000000005000000e80010417800814f51002b
:103ec000f9ff3a00000006000400fa00889fbe00d7
:103ed0008a9fbe008c1f78000004780001067800dd
:103ee00070089000f80090000100500088089000d1
:103ef000010050009808900001005000a8089000b0
:103f000001005000b808900001005000c80890005f
:103f1000810550000002220090bf9f000003230093
:103f2000a0bf9f00081090000028a30018003a00ce
:103f30000b00e000160034008b04780009057800bf
:103f4000e28f5400020036002a00200002003700f1
:103f50000900e0000b00340058009000c8019000f8
:103f60000a017800ee805700030001005004980019
:103f70000000e00096003200680890000000450054
:103f8000600c98008a8454004240a900ebff3c007a
:103f9000780190000200e0000b003400580090000f
:103fa000c80190008c0078000300010050049800c4
:103fb0000000e0008600320068089000f8009000e1
:103fc00001004000600c9800880c90000900e0009f
:103fd0001500340009057800e28f54000200360015
:103fe0002a002000020037000900e0000b00340026
:103ff00058009000c80190000a017800ec8057003a
:1040000003000100500498000000e000700032003e
:104010006808900000004500600c98008a845400f5
:104020004240a900ebff3c00180990000200e000ac
:104030000b003400e800900058009000c801900088
:1040400003000100500498000000e000600032000e
:10405000680890009808900001004000600c9800eb
:10406000a80c90000900e000150034000905780054
:10407000e28f5400020036002a00200002003700c0
:104080000900e0000b00340058009000c8019000c7
:104090000a017800ec8057000300010050049800ea
:1040a0000000e0004a00320068089000000045006f
:1040b000600c98008a8454004240a900ebff3c0049
:1040c000380990000200e0000d003400e800900084
:1040d000180890008080400058009000c8019000af
:1040e00003000100500498000000e0003800320096
:1040f00068089000b808900001004000600c98002b
:10410000c80c90000900e000150034000905780093
:10411000e28f5400020036002a002000020037001f
:104120000900e0000b00340058009000c801900026
:104130000a017800ec805700030001005004980049
:104140000000e000220032006808900000004500f6
:10415000600c98008a8454004240a900ebff3c00a8
:10416000081090000028a3001b0032000b00e000a4
:10417000190034008b04780009057800e28f5400a0
:10418000020036002a002000020037000900e0008b
:104190000b00340058009000c80190000a0178001c
:1041a000ee80570003000100500498000000e0007a
:1041b000070032006808900000004500600c98007d
:1041c0008a8454004240a90003003400eaff37000b
:1041d0000080eb00010037000000eb004f06780084
:1041e0004f05be004f04be000080fa00000006002c
:1041f0008f02b000889fbe008a9fbe008c9fbe00c9
:104200008e1f78008005780001067800820478000f
:10421000f3b79f0084bf9f00020078006d00070085
:10422000000578000b0778008006eb004f00370090
:104230008d06e9000d804600c2fc2f000f014100f1
:104240008280e800e1047800e80041006105780020
:10425000994078000180fb000000ea004f04de0076
:10426000888444000805550050c2b30080cf500038
:1042700002003a000a00e00009003a00880f5600e8
:104280004300390088805400080178000b00780052
:10429000e7fb070088854500080656003300370015
:1042a0001944780050c4b300804f54000500320018
:1042b0006a404000804f5400020032000044eb008e
:1042c000010037008904e800a4fd2f008f0242009e
:1042d0006e0252000f0242009941780008417800b6
:1042e0008fb897007fb097006e05070080017800b7
:1042f0000804e000010032000a05e9008904e80032
:104300000a05e9006fa197000200e00009003400ef
:10431000820f56001e003900830078000b007800e1
:10432000c3fb07006fa0970080854500000656007c
:104330000e0037000a00e0000a003200e28f56004b
:1043400008003e000d804600c4fc2f000f02420012
:104350008480e80089307800e80042008a307800e4
:104360008d06e8000205ea00830478000a00e000f8
:10437000b7ff3a000d00e000adff3a000c00e0008e
:10438000030032008d4d78000e805500010037008b
:104390000000eb004f0778004f06be004f05be003f
:1043a0004f04be008f02b100000006001004b100ef
:1043b000070035009001b100040034007000b10026
:1043c000030035009001b10001003c001000050021
:1043d0000000050080007800010037000000e800c0
:1043e0001004e000fdff3a0001005000000006004c
:1043f000207080001a073700881f7800a8e020008e
:104400001804e00004003a00801f2200480707005b
:1044100020c0b300004c7800100020004f0478004a
:1044200000000600e6874700889fbe008a9fbe0006
:104430008c9fbe008e1f7800800578004070800041
:104440000000e0000100320000000100f070800078
:104450000000e00001003200000001004053800035
:104460000000e000010032000000010081548000e3
:1044700030708000810f50001b0032001104e000fa
:104480000e003a00905480001004e00002003a0050
:1044900083fb070090548800728157003100200090
:1044a00090548000dafb0700805488001004e0007c
:1044b000020032000000e90080548800805480002f
:1044c0003a070700000478000085eb000000e000d8
:1044d0005100320020708000e1060700287088003b
:1044e00080548000307088005b0090008000eb00fa
:1044f00030fc0700800678007b0090007800b9004f
:104500002b0190000000410080bf9f005b009000e5
:10451000d21620000280b9006169b9000000410094
:104520008180490061004000e08048007200200066
:1045300003002000cf1107006e07400028708000a4
:10454000e90444000005eb00300037006406440035
:104550005b0190001c80fb00820f500029003c0092
:10456000b84090008180fb000200780011fc070039
:104570000d005000a84090008180fb0081014000a8
:10458000184278000404e0000f0032000e80410061
:104590008480fb000100500072002000110009001f
:1045a0000200d8000100e00002003a00010078009b
:1045b000010037006780100080814100e74f520002
:1045c00001003e00e78151007819b90018409000c1
:1045d0000080fb00020040008fb89700808f5000e1
:1045e0000d0035001c467800994f560004003a0033
:1045f0000a00e00002003a001a0020000100370023
:104600000005eb0065044400e584440000c0eb00b5
:10461000984f1000cdff3a000a0078004f0778004d
:104620004f06be004f05be004f04be006f00b10034
:1046300000000600889fbe008a1f780000047800f2
:1046400001027800824478000305780070c6b30048
:10465000804f510021003c0000c0e900804f510014
:10466000de003d0072405000804f51004b0132008f
:104670000d003c006c405000804f51005e013c003a
:1046800000c0e900804f5100d4003d0050c2b3008b
:10469000804f5100550132007c404000804f510056
:1046a00055013a00cd00370010c6b300804f5100cd
:1046b000ca00320004003c0069405000804f5100a5
:1046c0004d013a007200370030c6b300804f5100f0
:1046d000180032000040e8000900370000c7b300ae
:1046e000804f51001e01320008003c0000c0e9006c
:1046f000804f5100e400320065003c0065405000ee
:1047000080cf54003c013a000f00370050c7b3007f
:10471000804f51005e00320063404000804f5100e6
:104720005b00320065405000804f510032013a007a
:104730001a0137009180e900010a780078009000a2
:104740009171780032013700a8609000c0c6b300b4
:1047500080cf50000a003a00940078006480500036
:10476000000a78001000be004f89de00cf91de0005
:104770000002be00020378008203780013003700b5
:1047800010c7b30080cf500003003200a0c6b300b2
:1047900080cf500006003a009400780068805000f6
:1047a000000a78003002be002003be000700370078
:1047b0001480e900000a78001000780000027800f8
:1047c000cfa2de000503780086037800049cbe00bb
:1047d0000694be00a860900080c6b30080cf500051
:1047e0000e00320020c6b30080cf500005003a0012
:1047f0000400fb00cf80de00010178008201780018
:104800000a00370040c7b30080cf500003003200d9
:104810006640400080cf500006003a000400780057
:10482000cf80de000101780082017800009cbe008c
:104830000294be003800be002801be00e00f500008
:10484000e08f5800e00f5900e08f590003003d0051
:1048500078009000d1c2b3000a0037000810900021
:104860000018a3000300320078009000b1c2b3002a
:10487000040037000008a3005300320078009000c5
:1048800001c2b300017578000000e8004d00370058
:10489000a8609000c0c6b30080cf500006003a0068
:1048a0009400780064805000000a78001002be0076
:1048b0006033b8001300370010c7b30080cf50003a
:1048c00003003200a0c6b30080cf500006003a00bb
:1048d0009400780068805000000a78003002be0022
:1048e0002003be00070037001480e900000a7800aa
:1048f000100078000002780005002000060020006b
:1049000007002000049cbe000694be00a860900032
:1049100080c6b30080cf50000e00320020c6b30026
:1049200080cf500005003a000480fb000100200009
:1049300002002000030020000a00370040c7b30037
:1049400080cf5000030032006640400080cf50000e
:1049500006003a0004007800010020000200200058
:1049600003002000009cbe000294be0008109000ce
:104970000038a300140032003800be002801be0039
:10498000e00f5000e08f5800e00f5900e08f590011
:104990000d00320080c7b30080cf54000300320006
:1049a00080c5b30080cf540007003a007800900023
:1049b00001c3b300017578008000e80009f57800b4
:1049c0000080e80070049800780090000000450026
:1049d00060049800894078006d003700a86090005e
:1049e000c0c4b30080cf500006003a0094007800a5
:1049f00068805000000a78005001be004000be00f0
:104a0000050037009400780064805000000a7800a8
:104a10001000be00a9100700009cbe000294be005a
:104a2000380090000000e00003003d007800900096
:104a3000d1c2b3000a003700081090000018a3008c
:104a40000300320078009000b1c2b30004003700c8
:104a50000008a300050032007800900001c2b300f6
:104a6000017578000000e80070049800780090005c
:104a70000000450060049800894078000800780034
:104a80004706070064003700a8609000c0c6b30066
:104a900080cf5000250032000a003c0064405000e6
:104aa00080cf50002800320000c0e80080cf5000c6
:104ab000140032006840500080cf500022003a00bd
:104ac0000a00370040c7b30080cf50001e003200fc
:104ad0006640400080cf50001b003200694050000b
:104ae00080cf500018003a00060037001480e9001b
:104af000000a780010007800485c900008487800b0
:104b0000450037001480e900000a780010027800a0
:104b100068089000cf80de000101780082017800f3
:104b2000009abe000292be003b0037001480e900ec
:104b3000000a78001001780068089000cf80de003d
:104b40000089be00340037001480e900000a7800b4
:104b500010007800680c9000080878002e003700dc
:104b60001180e9008008780010007800cf80de0016
:104b70000101780082017800009cbe000294be0012
:104b800078009000000045006004980081c7b300e1
:104b900008007800bb0007001f0037001480e90000
:104ba000000a78001000780060049800580990000e
:104bb0000200e00002003d0006fe07000900370089
:104bc0008000eb00a2fc0700800078000000e000fd
:104bd00003003200680090000080500001003700a0
:104be00058089000100c98000b00370078009000d7
:104bf00002757800060037007800900080004500bc
:104c00000904e00001003a0059c2b3008948780065
:104c10000000e800700498000000eb004f057800e9
:104c20004f04be0000000600881f780000047800d2
:104c30000040eb000054980038009000904078004d
:104c400090c6b30080cf50002a00320013003c0011
:104c50007140500080cf50002600320005003c001b
:104c600050c2b30080cf50006400320030c5b300a2
:104c70001b00370030c6b30080cf50001b0032004d
:104c80000040e80080cf50001a0032006940500018
:104c900080cf50006e003a007300370000c7b300a9
:104ca00080cf500007003c000040e90080cf50005a
:104cb00010003d000040e90080cf500064003a0041
:104cc0000f00370050c7b30080cf500009003200fa
:104cd0006340400080cf5000060032006540500025
:104ce00080cf500043003200590037008000eb00b5
:104cf0005e00370008007800d20707005f00370029
:104d0000684890000004e0005b003a00f84890001a
:104d1000c0c6b30080cf5000270032000a003c001c
:104d20006440500080cf50002b00320000c0e800eb
:104d300080cf5000150032006840500080cf5000f6
:104d400025003a000a00370040c7b30080cf50006a
:104d5000210032006640400080cf50001e0032002b
:104d60006940500080cf50001b003a000700370018
:104d7000280090000080e9002004980010007800ce
:104d8000084c9000084878003b003700280090004d
:104d90000080e9002004980010027800480090008c
:104da000cf80de000101780082017800009abe0009
:104db0000292be0030003700280090000080e90019
:104dc000200498001001780048009000cf80de0099
:104dd0000089be0028003700280090000080e9000c
:104de000200498001000780048049000080878001b
:104df00021003700110020001c00370048009000ff
:104e00000000e80040049800180090009801780025
:104e1000120020008000eb000300010080007800f9
:104e200050022000808f5000130032004800900094
:104e3000e18f4000080032000000e90040049800c3
:104e400018009000980178000001eb0003000100b9
:104e50000000eb00090037000000e9004004980062
:104e600001007800050037008080eb000800780022
:104e7000cd08070001003700100020004f04780023
:104e8000000006002f03b000889fbe008a9fbe006e
:104e90008c9fbe008e1f78000007780030d720005e
:104ea000c0b79f0080c5b30080cf5000080032001b
:104eb00022d62000c2b79f007740400080cf50002c
:104ec00003003a0083002000b3b79f000a003700b8
:104ed00080c7b30080cf500005003200a40020003e
:104ee000b4b79f0080c5b30080cf500002003a00e5
:104ef00005012000b5b79f003e04be002e05be0090
:104f000040c6b30080cf500003003200654040002f
:104f100080cf50000b003a00e00f5400e08f5c009f
:104f2000e00f5d00e08f5d0006003d006000b8000e
:104f30006011b80008045000898458000a0559001f
:104f40008b855900bfb39700e88f530003003200f0
:104f5000f08f530045003a00020037003600200071
:104f60000100370046002000e00f5400e08f5c0095
:104f7000e00f5d00e08f5d0005003a005e089000e4
:104f800081012000a1b79f000000e000080032006e
:104f90003fb197000200e90008006000cfb1970020
:104fa0006340780090df9f0074012000a4b79f0049
:104fb000860278008502e900050033008b05d100e8
:104fc0000a85d3008984d3000884d300f9ff370011
:104fd000089fbe000a97be00afb397000700e90024
:104fe00021fc2f008f804000008240003fb19700dd
:104ff0008202e90012003700afb397008703e9008f
:10500000a7b79f0000806200cfb097006152780080
:105010003e00be002e01be00860378008703e90033
:10502000050033008381d1000281d3008180d30049
:105030000080d300f9ff3700009fbe000297be003a
:105040003e00be002e01be00e00f5000e08f580071
:10505000e00f5900e08f5900d6003400afb397003d
:105060000700e000e4ff3c00d2003700ae60900093
:1050700080c6b30080cf50000b00320006003c0019
:105080000104e000080032006640500080cf50006c
:1050900073003a0004003700c0c6b30080cf500050
:1050a0006f003a0031003700080178000800e00086
:1050b00005003a005e08900081012000a1b79f0022
:1050c0000000e00009003200bfb1970011000900a4
:1050d0000381d8008000fd004fb297006440780043
:1050e00090df9f0075012000a5b79f00bfb3970018
:1050f000110009000781d80080017800afb0970047
:105100000100e90022fc2f000f01410000024100d4
:105110000c003700bfb29700110009008501d800cc
:1051200000017800afb397008703e900a7b79f009d
:105130000590b90000805100cfb09700615278000f
:10514000820178000300e000030034002fb19700d3
:105150000200e000efff3c0003007800cf80de009b
:1051600001017800820178003a0037000806be008d
:10517000e00f5400e08f5c0005003a005e089000ec
:1051800083012000a3b79f000000e0000900320067
:105190003fb297006121b9000c00be00c40e0700a9
:1051a000cfb297006540780090df9f007701200024
:1051b000a7b79f003fb297006121b9000c00be0065
:1051c000f60c07000006be00afb297000500e9002c
:1051d00027fc2f008f8343008083430097b79f00f5
:1051e000110037003fb197006114b9000801be00fb
:1051f0000c00be00240e07000005be00afb19700f2
:105200008301e900a3b79f000801be00dd0c070081
:10521000000056001fb29700cfb297006552780089
:1052200094b79f000a06be00e00f5600e08f5e00b4
:1052300003003400afb397000700e000e9ff3c0033
:105240004feade00cfa2de000c00be0004017800b1
:1052500084017800009fbe000297be005500370011
:10526000e00f5400e08f5c00e00f5d00e08f5d0018
:1052700005003a005e08900081012000a1b79f0060
:105280000000e0000d0032003fb1970002027800fc
:10529000cfa2de0005037800860378000800be0078
:1052a0000a01be00250f07004fb297006440780046
:1052b00090df9f0075012000a5b79f003fb19700c8
:1052c00002027800cfa2de00050378008603780092
:1052d0000800be000a01be00110f0700009fbe00bb
:1052e0000297be00afb197000300e90024fc2f0035
:1052f0000f0242000006420020003700bfb29700b4
:1053000005047800cfc4de00090578008a0578001e
:105310000802be000a03be005fa89700efa897002e
:105320007fa997008fb19700080f0700d0b79f00a3
:10533000e1b79f00f2b79f0083bf9f00afb3970014
:105340008703e900a7b79f000802be000a03be005a
:10535000dc0d07005faa970000005200cfb2970053
:10536000655678005fb09700efb097007fb1970067
:105370008fb99700009fbe000297be003e00be009e
:105380002e01be00d0af9f00e1af9f00f2af9f00a3
:1053900083b79f00e00f5000e08f5800e00f5900e6
:1053a000e08f590003003400afb097000100e00027
:1053b000d2ff3c003fb19700e80f510013003a00c4
:1053c0000e1090000038a30010003200afb197001b
:1053d000f78f510006003e0024fc2f000f02420010
:1053e0008300420000c3b300914f10000700320059
:1053f000afb297008502e900a5b79f0000c3b300d4
:1054000027fc2f008f83430080f37a00afb1970011
:1054100078811100120f98006e00900024fc2f007c
:105420000f0242008300420081f707001e0990002e
:105430005e089000800f510006003d000200500001
:10544000000f98000e1090000040a1000017980077
:105450000f0037000000e0000d003d000e1090002e
:1054600074006000f00f500009003a007e089000c0
:10547000fe009000010050008e08900001005000d6
:10548000020050004240a90001003400000f9800c3
:105490004f0778004f06be004f05be004f04be0008
:1054a0002f03b10000000600889fbe008a9fbe0047
:1054b00080057800010478000205780083047800f4
:1054c00084407800050178000800e00001003d00fc
:1054d0000004eb00f0c4b30080cf500006003a0097
:1054e000221090000901780088007800c8f70700b2
:1054f0001900e0000e003c008a0c78000a8145008b
:105500000049eb00a300200006003700110009004d
:105510000304d8008000fd0004c3b3000461400010
:10552000010478000a05e900f8ff3b00020078005a
:105530004f05be004f04be000000060080805000f2
:10554000e780400073002000110009008300d800ac
:105550008000fd000001510003014100110009001d
:105560000301d80000000600889fbe008104780077
:105570000204780010002000f0ff0700000278000d
:1055800080017800088054003017b00072002000bd
:10559000110009000200d800d016200001004000d0
:1055a000811f7800110009000200d8000101780075
:1055b000cf007800b0162000800f540003003400a4
:1055c000e20f510004003a0010003700a01620003e
:1055d000800f540003003400e30f510004003a0030
:1055e0000a00370090162000800f5400020034009b
:1055f000e40f5100050032000180e900e20f500085
:1056000003003e008401e800010037008081eb00c8
:10561000030078004f04be0000000600881f7800d9
:1056200000047800d0ff07000000e00002003a000c
:105630000804e900030037000000e00001003c001e
:105640000804e800080078004f0478000000060015
:105650000200fa00889fbe008a1f7800800478004c
:1056600001047800a2002000e880570008007800bc
:1056700087f707000002be004fb99700820f540061
:1056800035003200fac2b300924f150032003a00e2
:1056900059009000c176200001004000cf80de005c
:1056a000800f5200818f5a0004003200840f500096
:1056b000858f58002a003d002b0037000204e800c7
:1056c000a2002000e88057000800780070f707006b
:1056d0000003be004fba9700840f54001e00320032
:1056e000944f15001c003a00490090000000e800ab
:1056f0006101b900820f5300838f5b000400320008
:10570000860f5100878f590015003d0016003700a5
:105710000400e800a2002000e88057005cf70700c2
:105720000002be004fb89700800f54000a003200fc
:10573000390090006101b9000000eb00820f5200b7
:10574000838f5a0009003200840f5100858f590061
:1057500003003d0004003700200020000300370054
:1057600010002000010037000080eb004f0578009a
:105770004f04be000080fa00000006000200fa009c
:10578000889fbe008a9fbe008c1f7800800578002d
:10579000010678000005eb00340037008804e800bb
:1057a0006c815700110020000900780018f70700ed
:1057b000800078000b007800a5ff0700000178004a
:1057c00098407800d0c2b30080cf500004003a0067
:1057d0000200e800e10f500023003e000500370002
:1057e000b0c2b30080cf50001f003a00e10f51005b
:1057f0001d003e006c815700210020000900780048
:1058000003f707000001780010407800984f50001f
:1058100004003a0092409000a0c2b30080cf500034
:105820001a003200820078000b00780088ff070021
:105830000001780098407800d0c2b30080cf5000bb
:1058400003003a00e10f510007003e000f0037004f
:10585000b0c2b30080cf500003003a000200e8005d
:10586000e10f5000090036000a05e8001c10900006
:105870006c8157008a007800e5f607000004780084
:105880001004e000c5ff3a0028d12000080078008d
:105890004f0678004f05be004f04be000080fa009e
:1058a00000000600ea874700889fbe008a9fbe006e
:1058b0008c9fbe008e1f78008004780081057800e0
:1058c0000246780004057800050778000300fb0015
:1058d000cf80de005002b1000180b10052052000ef
:1058e000820f5000e08f5800d0013e0000600100a0
:1058f000ca013700cd013700cc013700cb0137009a
:10590000ca013700c9013700c8013700c701370095
:10591000c6013700c5013700c4013700c301370095
:10592000c2013700c1013700c0013700bf01370095
:10593000be013700bd013700bc013700bb01370095
:10594000ba013700b9013700b8013700b701370095
:10595000b6013700b5013700b4013700b301370095
:105960003d00370044003700510037006c0037001d
:10597000ae0137007c0037008a0037009400370002
:1059800095003700a9013700a8013700a7013700ab
:10599000a1003700a5013700a4013700a30137009b
:1059a000a2013700b3003700b6003700bf00370050
:1059b000c7003700ca003700e7003700f50037009e
:1059c00047013700890137009801370097013700f8
:1059d0009601370095013700940137009301370095
:1059e00019003700760037002800370044003700e0
:1059f0004f0037008d0137005f003700700037001f
:105a00008a0137007a0037008801370087013700a4
:105a10007e003700820037008401370084003700a1
:105a2000820137008a003700800137009b00370071
:105a3000a20037007d013700c1003700cc003700dd
:105a4000df00370046013700e90090008180400008
:105a50002b00900004003700e90090008180400096
:105a60008100e8003b0090000a01780068f607001a
:105a70000004780073013700c90090008180400065
:105a80008100e8006b009000f7ff370050c4b300be
:105a9000804f560002003a005b089000010037007a
:105aa0000b0890000a0178008000eb00c10037006d
:105ab00050c4b300804f56000a003a008b007800b3
:105ac000090078002dff07000000e8000a017800b7
:105ad000310020004ef60700000478001004e000ba
:105ae00058013a00d9009000420620001100090038
:105af0008200d8008000fd00f380400001003700e4
:105b0000b90090008b0278000c4278008a0178007e
:105b1000220020000e00780063fe0700d4ff37004b
:105b200080ff2f00000a780058d12000450137007f
:105b3000b90090008b0278000c4278008a0178004e
:105b4000220020000e00780057fe070000047800b5
:105b500000c3b3009e4f10003a013a00704050005d
:105b6000004f78003701370080ff2f00000a7800cf
:105b7000e8d120003301370079019000e90090005e
:105b800059009000a5fe0700420620001100090000
:105b90000200d8000100e000daff3d0082804000f2
:105ba000d8ff370079019000e9009000590090007b
:105bb0009afe0700c176200081004000db0037001c
:105bc000c9009000818040005b009000a6ff370074
:105bd000a9009000cbff3700290090006b00400027
:105be000c2002000110009000200d80008003700a0
:105bf000f90090008100e8008b0278000c427800e8
:105c00008a01780032002000c2ff3700c9009000ee
:105c10008100e800bbff370099009000b9ff370012
:105c200010002000000a780078d22000050137001b
:105c30008000eb0029009000eb0f500001003400c1
:105c4000110020000a0178001b00780087ff370050
:105c500050c4b300804f560002003a000b10900071
:105c6000010037003b0890000a0178003100200055
:105c700050003700b0ff2f00000a780098d22000b3
:105c8000f00037008b0278000c4278008a0178001f
:105c900022002000990078009eff370010002000ad
:105ca000000a7800f8d22000e600370080ff2f00bd
:105cb000000a780018d32000e2003700e9009000c5
:105cc0000100e0001f003a00710020001d003700b5
:105cd00079019000e90090000000eb0021003700fe
:105ce000f906900069049000d90490000d01780035
:105cf00088007800090078001bfe07000000e00023
:105d000006003a008d005400e78040000900e900d9
:105d1000d216200014fe0700030037000000e00048
:105d200001003c00100020008b0278000c4278003b
:105d30008a017800220020008000780075ff37007b
:105d4000e90090008b0278000c4278008a0178000c
:105d5000120020006fff370079019000e9009000e9
:105d600010002000f5fd07008000780065ff370077
:105d700050c4b300804f560002003a006b089000f8
:105d8000010037001b0890000a0178001100200074
:105d90000800370050c4b300804f560002003a009c
:105da0007b089000010037002b0890000a01780062
:105db0002100200096f507000004780066003700f7
:105dc0005900900042062000110009000200d8008e
:105dd000e1b79f000100e00002003d00828040002a
:105de000e1b79f0050c4b300804f560035003a0021
:105df0008b0078000900780060fe070080067800bc
:105e00000081e80082bf9f001204e0002d003200f4
:105e100059049000c076200000044400cfc4de0086
:105e20008d01e800f3b79f000a01780011002000ff
:105e30000300780076f50700a20020008000eb0048
:105e400093f507000004540081845c00d0c2b300c5
:105e50009d4f100002003a0060041400e0841c0012
:105e6000a2002000f68057000fb8970088f50700c1
:105e700008004000898048005fb197008fb9970003
:105e8000828f51000f00320012417800ffb197005d
:105e9000934f51000b003a00e0b79f00180020001c
:105ea000010037000804e800a200200003002000e1
:105eb000f50a0700e00f5000e08f5800f9ff3c00a2
:105ec00001003700280020008b0278000c42780087
:105ed0008a01780008017800efb097000dff3700c5
:105ee00050c4b300804f56000d003a008b0078007c
:105ef0000900780021fe07000000e8000a01780090
:105f00004100200042f5070000047800b0c3b30050
:105f1000984f1000020032001a00e00008003a001a
:105f2000d9009000c0762000808040008b0278006d
:105f30000c4278008a01780042002000f5fe37000c
:105f4000b103200008007800d6f707000000e00049
:105f500001003200080d50001a0dea003900370028
:105f60004b1090001004e00001003a00ccf4070050
:105f70000a0178002100200025f5070000047800c0
:105f80001a00e0002f003400090890000000e00033
:105f90002c003400a20020008000eb0008007800f4
:105fa0003bf50700410620008080400003003300dd
:105fb000b0c2b300004f780003003700d0c2b30076
:105fc000004f78008100ea000e00e8008b027800a4
:105fd0000c4278008a0178004200200032fd070060
:105fe0000004e9001a0de800160037000004eb0079
:105ff000090890000000e0000100340018002000b3
:106000004b1090001004e00001003a00a4f40700d7
:106010000a0178008800780094fe37001000200004
:10602000000a7800a8d3200006003700034f78004c
:106030000040eb00104798000e047800200020007c
:10604000000d7800080078004f0778004f06be006a
:106050004f05be004f04be00af00b10000000600b7
:106060000000e000310032008080e90091027800f9
:10607000e38f52002d0036000508a3002b003a00e4
:10608000827080000200e00002003200828f500027
:106090000400310002087800817088001600370083
:1060a00003017800920190000300e000020032003a
:1060b000818f5100faff390012027800040041007c
:1060c000808f500019003900810f500003003a0002
:1060d0000509420082007800070037000300e00055
:1060e0000300320005804000808f51000f0039000e
:1060f0009300980011019800110190000200e00047
:106100000a00320011804000820f500007003a0060
:10611000e0e020000008eb00110090001101780081
:1061200090084100100090009000980000000600c8
:1061300000017800000020000000e00008003200ac
:10614000000080000000e000050032000000e900cf
:1061500000008800000040000100800002b07800cc
:106160000000060080017800010178008000eb004b
:10617000040037006a08b9000000420085004000b2
:106180008301e8000201e900060033001302fb006e
:1061900005fd2f0005004200e90f5000f5ff360015
:1061a0008080eb000100780000000600e8874700cf
:1061b000889fbe008a9fbe008c9fbe008e1f780005
:1061c00030477800800478000e04e0006c00320054
:1061d0002a002000020037000800e8000a05e80055
:1061e0008e00fb002ff70700000478000000e0009d
:1061f000f9ff3a006550b900d804070080bf9f003e
:10620000800578000000e0005d0032000006e80034
:1062100000057800e8b79f0080c2b300994f1000d6
:106220000c003a000900e80041002000cdff070003
:1062300041892f0001004000e0b79f004800330073
:10624000d940900090c2b30080cf500044003a0083
:10625000e68444004fe89700e0ef9f004045980037
:106260002100200009007800beff0700e30645007a
:10627000804ee9000980e80021002000b9ff0700f6
:106280000a84e800004ce900648144001200fb002d
:106290000003b100e90f500006003e00210020007d
:1062a00002007800afff0700004e780066814400ce
:1062b00001003700004eeb00b0c0b3009d4f10004e
:1062c00027003e0030c6b300984f100024003e0067
:1062d0009c4f100022003e0092407800b0c2b300f4
:1062e00080cf50000500320000c0e80080cf500091
:1062f00002003200004deb00100037009241900088
:1063000000cdb30000c24100e64f520014003e0031
:1063100071c0b30000c3b30080cf51000100320050
:1063200084407800014d7800b0c2b300924f100055
:1063300001003a0067cd40000281e8001240780079
:106340000004e00009003200650646008e4f500050
:1063500003003a00650545008204e800aeff3700ff
:106360000fb897003eff07000500370065004500a5
:1063700000c8eb00efe897004140980001003700ab
:106380008005eb000b0078004f0778004f06be0039
:106390004f05be004f04be008f00b1000000060094
:1063a0008f04b000889fbe008a9fbe008c9fbe00f5
:1063b0008e1f7800f0b79f0081f79f005001be004c
:1063c0004000be00f0979f00819f9f00929f9f001a
:1063d000a39f9f0010c6b3000ff19700804f51009c
:1063e0001600320010c4b300804f51001300320079
:1063f000ffb19700530890000000e00003003d004b
:1064000060002000d00998000c0037000000e00078
:106410000a003a0070c6b3000ff29700804f520096
:106420000300320070c4b300804f520003003a00f2
:1064300010002000ffb29700d00a9800ffb097002c
:10644000c0fa2f000f00400096040700800178007a
:10645000e20f500015003a0030002000ffb0970016
:106460009008980010c6b3000ff19700804f5100bc
:106470000a00320064404000804f510007003200a3
:106480000040e800804f51000400320001cb2000a2
:106490000040e800804f510001003a0041cb20004d
:1064a000ffb1970063009000160037000000e00085
:1064b00018003400300020007fb29700100a9800c6
:1064c00010c6b3008ff2970080cf52000a0032004e
:1064d0006440400080cf5200070032000040e800d6
:1064e00080cf52000400320081cb20000040e80041
:1064f00080cf520001003a00c1cb20007fb197004d
:1065000062009000315878003158780011487800c6
:10651000c601370014c6b3008ff2970084cf520033
:106520000300320010c4b30080cf520013003a00c1
:106530007fb09700600190008200780000c3b30034
:1065400080587800ffb29700e102980080c7b3003e
:106550008ff2970084cf52000100320080c5b30053
:10656000804878000280e800ffb09700e0009800c3
:10657000710090000080e800f00098000300e00047
:1065800005003a00e3979f0064fb2f000f014200d3
:1065900003077800a001370005cc2000e5b79f0075
:1065a00010c6b3008ff0970080cf50000500320076
:1065b00010c4b30080cf5000a7003a0012cd2000d5
:1065c000e2b79f00ffb19700530890001e02200021
:1065d0000000e000010035000007e8000e02e800be
:1065e000d4b79f006022b8006033b8007f90970056
:1065f0008f9897001f999700af999700d90a0700c5
:10660000ffb097003102be002103be000000e00091
:1066100004003d000400be000601be0003f0a2001d
:10662000020037000400be000601be00f0979f0084
:10663000819f9f00929f9f00a39f9f006f91970053
:1066400064015100e2979f00c3fa2f008f8141003f
:106650006a8041000048eb006b824100c4b79f0094
:1066600031003700c201200003002000e5fa2f00ae
:106670000f804200370407007f9497008f9c97009b
:106680001f9d9700af9d97000800be000a01be0045
:10669000b90a07000006be005fb19700670151000c
:1066a000d2b79f004240a9000a003400de0a07006a
:1066b0000002be000203be000800be000a01be00c8
:1066c000dc0a0700f0979f00819f9f00929f9f0028
:1066d000a39f9f00cfb19700678041007100200009
:1066e000050037006f6066004c6add004466de001e
:1066f0000c067200c4eede00e00f5600e08f5e0074
:10670000050034008100e900e18f4000f5ff3a0008
:10671000010037000060eb008100e900fdff3b0055
:1067200067004000c0b79f00dfb297000500e0009f
:10673000090034006022b8006033b8007f909700f1
:106740008f9897001f999700af999700bb0a070091
:106750000000e000c3ff3c0060fb2f008f00400002
:106760004fb19700010051000000e9008e0f50006a
:1067700001003d00000778000e00e00003003d002e
:1067800073fb2f000f8141002c003700800f570052
:1067900005003d000e80400010409000f3c0b300a3
:1067a000e74f500001003c008041eb00c4fa2f008d
:1067b0000f0242000e0042006a0040008e00780086
:1067c000010037000000e9008100e9001041780075
:1067d000834f5100fbff32000107e800efcf51006b
:1067e00001003a000248e8000100e0000300350023
:1067f00075fb2f000f814200060037000e07e800ee
:106800006f90970064004000e0979f0061fb2f00ad
:106810000f8140008e0041008e0178000300370098
:106820001100fb006fb29700e44878008301e90093
:106830008100e9000300e000f9ff3d00ffb297008e
:10684000550890000000e000f3003d000e00e90054
:10685000d00a9800f00037007f9497008f9c970033
:106860001f9d9700af9d97006022b8006033b8006d
:106870000800be000a01be003a0a07000000e0005e
:1068800005003d000bf0a200f8979f00899f9f0034
:106890009a9f9f00ab9f9f006f90970072592700af
:1068a0000280b900026a2800130020007608070061
:1068b000e4005000e1979f0015003b00e3801000ca
:1068c000c0ff2f00008460000800ea00e0979f00ee
:1068d0007f9097008f9897001f999700af99970026
:1068e00089c62000070037000808a3000300320013
:1068f0003902be002903be00550a07000884d100f2
:10690000e88444000800e000f7ff3c001b0037006b
:106910000100e0001d003400c0ff2f000080600077
:10692000e0979f00000478006000b800020020009b
:1069300003ff230089c62000070037000808a300d2
:10694000030032003902be002903be00400a0700de
:106950000884d100e88444000800e000f7ff3c0010
:106960000002be000203be007f9097008f98970040
:106970001f999700af999700aa0a0700f0979f0008
:10698000819f9f00929f9f00a39f9f00ffb0970051
:106990005109900060c6b3008ff1970080cf51007d
:1069a000040032006100200060c4b30080cf5100b9
:1069b00002003a006f929700ea004200010741008e
:1069c000f30f5700010034003e01200000c3b30064
:1069d000e0779f0075fb2f008f824200b5b79f00c4
:1069e000330037000800be000a01be00e2090700bc
:1069f0000006be00680757004240a9000e003400a0
:106a0000090a07000002be000203be000800be0023
:106a10000a01be00070a07006022b80046782d0070
:106a2000771924000a0a0700f0979f00819f9f00b2
:106a3000929f9f00a39f9f003fb097006804400073
:106a4000890020000d003700a40020000500200070
:106a50000c01be00e0fd2f000f004000b80307004e
:106a60007fa897008fb097001fb19700afb1970034
:106a700004c3b300046441000006be00e00f5600ea
:106a8000e08f5e00060034008904e900e18f4400d5
:106a9000edff3a000200370000c3b3000064780045
:106aa0008904e900fcff3b0068044400b8b79f007c
:106ab0000e00e0000b0034007f9497008f9c97003d
:106ac0001f9d9700af9d97006022b8006033b8000b
:106ad0000800be000a01be00d80907000000e0005f
:106ae000c0ff3c00c5fa2f008f8242006a8042003e
:106af000bfb09700008050008001e9006f919700bf
:106b0000e70041006b81420000c3b3000100370081
:106b10000201e800924f1000fdff320074fb2f00cd
:106b20000f004200808040008280500000804100c1
:106b300002025000e1979f00ffb29700d509900034
:106b400060c6b3008ff2970080cf5200030032007e
:106b500060c4b30080cf520002003a008100e80018
:106b60000a00370050c6b3008ff0970080cf500066
:106b7000050032008000eb0050c4b3008ff2970094
:106b800080cf520001003a0011002000018741002f
:106b90008e0f520001003d00040778000e00e00057
:106ba0001d003500840f570005003d00e2407f00c6
:106bb00095c3b30040c3b30080cf500001003c0038
:106bc00005c3b3000e0041008000e9008e0178008b
:106bd000010037008100e9008301e90011427800db
:106be000854f5200fbff32000307e80090c3b3005b
:106bf00080cf520001003a008448e8000300e00022
:106c000005003d000201e9000e07e8006f909700c3
:106c10000000e800e0979f006f9297008e017800d7
:106c20008ff097007fb09700620307004f0778004e
:106c30004f06be004f05be004f04be008f04b100da
:106c4000000006002f02b000889fbe008a9fbe0091
:106c50008c9fbe008e1f780080047800600090003a
:106c60000000e00001003c00f0ff27000000e90008
:106c7000d0049800c90090000c0033000100e80027
:106c8000c0049800190090009901780012002000bb
:106c90008000eb000300010000057800b002200036
:106ca000800f550006003a000b0037000100e80095
:106cb000c00498002cfd2f000f0646001b00370073
:106cc000d0022000800f5500030032002cfd2f0061
:106cd0000f0646001600370030fd2f000f0440005d
:106ce000aad79f00590090000000e900d004980046
:106cf000c90090000a0033000100e800c0049800b9
:106d00001900900099017800120020008000eb002b
:106d10000300010000057800080678000400370031
:106d20000100e800c0049800080678000085eb0028
:106d300038d42000390090009000fb000800780053
:106d400058f4070008005000c1d3200061447800c7
:106d50008805fb0000032000800f550033003a0037
:106d6000590090000000e900d0049800c90090008c
:106d70000c0033000100e800c004980019009000e6
:106d800099017800120020008000eb000300010050
:106d90000005780080072000800f550005003a00ac
:106da000070037000100e800c00498000085eb00f0
:106db0001b00370080052000800f550018003a00a6
:106dc0000804e00002003200f04f54001d003a00b9
:106dd000590090000000e900d0049800c90090001c
:106de000090033000100e800c00498001900900079
:106df00099017800120020008000eb0003000100e0
:106e000000057800030037000100e800c004980086
:106e10000085eb000047eb000b012000110037005c
:106e20000804e000b8003200060037000047eb001d
:106e30000804e00004003a00ad0020000847780094
:106e40001c0037001ec0b300ad002000ea4f540004
:106e500018003200e88f550002003a008b067800d7
:106e6000140037006d012000120037005900900017
:106e70000000e900d0049800c90090000900330028
:106e80000100e800c0049800190090009901780002
:106e9000120020008000eb000300010000057800d4
:106ea000030037000100e800c00498000085eb00f3
:106eb0001ec0b30000032000800f5500ebff32001e
:106ec0000e04e00018003200005e78001600370063
:106ed0006f805700800f5600010031000a5e780075
:106ee000590090000000e900d0049800c90090000b
:106ef000090033000100e800c00498001900900068
:106f000099017800120020008000eb0003000100ce
:106f100000057800030037000100e800c004980075
:106f20000085eb001ec0b300e10f450007003200f2
:106f30000d0178008a007800b0d42000c4f3070067
:106f40000000e000e2ff3a006600370049009000d0
:106f50000000e900c00498000e04e00008003a00b8
:106f600020fd2f000f004000800f56005b003a000c
:106f7000e10f450059003a008a00780065003700ab
:106f8000004eeb0069489000110020000004e00072
:106f900060003a00390090009040780040c6b3008d
:106fa00080cf5000030032006540400080cf500089
:106fb0000a003a000b0178008000eb0020fd2f0052
:106fc0000f004000af0307000203be000002be0036
:106fd00010c0b300805498000d0037000b017800fa
:106fe0008000eb0020fd2f000f004000ff03070092
:106ff0000203be000002be0010c0b300805498001f
:10700000b900900000c7b300914f10002c0032006f
:10701000f9489000c0c6b30080cf50002200320073
:107020000a003c006440500080cf50002400320031
:1070300000c0e80080cf50001400320068405000cb
:1070400080cf50001e003a000a00370040c7b3004e
:1070500080cf50001a0032006640400080cf5000c0
:10706000170032006940500080cf500014003a00f1
:1070700006003700290090000080e900a004980075
:1070800010007800044878001200370029009000b2
:107090000080e900a0049800100078000498be0069
:1070a0000690be000b003700290090000080e90028
:1070b000a0049800100078000488be000500370086
:1070c000290090000080e900a004980010007800da
:1070d00004087800110020000e0037008000eb004b
:1070e0000c003700490090000000e900c00498003f
:1070f00019009000990178000001eb008a007800e7
:107100000300010094ff37001ec0b3008b00200075
:1071100052ff3700010078004f0778004f06be008d
:107120004f05be004f04be002f02b1000000060054
:1071300080017800d4c2b3000f0037000300e800dc
:10714000904f120008003a0093cf100003003e0059
:107150002340900080cf500012003600e3814100b0
:10716000630151000400370093cf10000d0032007e
:107170000201e90080017800e20f5100efff3e00bc
:107180000002eb000400370064c079000402e8004c
:10719000814f500003003200820f5200faff3a0084
:1071a0000000050010000500f0874700889fbe0022
:1071b0008a9fbe008c9fbe008e1f7800000478005e
:1071c000810678000000eb00c0b79f00f8489000ef
:1071d000c0c6b30080cf500002003a00110020006a
:1071e000c1b79f000d00e00023003d00b8009000f3
:1071f0000100e80030049800e2c5b3008041eb00d4
:1072000083f79f00904f110003003a000180e800cf
:107210003004980082f79f00b8049000d0c5b300f6
:10722000994f100002003200090078000100370079
:107230000900e800d10520001af30700d0b79f002d
:107240008000eb000000e000bd00320009065000a5
:10725000e20f5600080034000c81e9000900e80044
:10726000d1022000faf2070011c0b300c1ef9f0065
:107270000000e00002003a008041eb00c3ef9f00f5
:10728000680090000000e00004003c00f0ff2700d0
:107290000d00e00001003a001000200050049800aa
:1072a000684890000004e0000d003a0028009000bb
:1072b000cfb097000100e000050032000080e90037
:1072c0002004980010007800b0b79f000400370039
:1072d0000080e9002004980010007800f0b79f00bb
:1072e0000045eb005e0037000d00e00003003400b5
:1072f00009007800c7f207001e0037000d00e0000b
:107300001e003200cfe997000304e0000c003a00b1
:10731000380090008ff097000104e00004003a006c
:107320000c01780089007800c9f207000b003700d3
:107330000c01780089007800c5f207000d003700c5
:10734000380090008ff197000304e00006003a0037
:107350000c0178008900780075ff07000000e0004c
:1073600006003a006d0037000c01780089007800b3
:107370006fff07000000e00068003a004fb0970080
:107380000000e00009003a00684890000004e000b6
:1073900032003a00ffb0970089587800f1b79f009b
:1073a00010c0b300005498002c003700c9e79f00bc
:1073b0008905fb000b00780001003200100020005e
:1073c000000578001e0020000000e00016003a00d2
:1073d0000904e00004003a007c805700fdf3070038
:1073e0000005e800100037000e07e900fc81570097
:1073f00063407f008000fb0048019000e14f4000a7
:10740000070032000200e9004004980018009000d4
:10741000980178000001eb00030001000200370032
:107420000200e900400498008e0f5500eeff350081
:10743000684890000004e00005003a003fb0970063
:107440000b187800b0b79f0010c0b300005498002c
:10745000680090000000e900600498002ac0b300b2
:10746000580090000000e900500498004801900086
:107470000b0033000200e800400498001800900060
:1074800098017800120020008000eb00030001004a
:1074900080047800e10f400093ff3a0002003700bb
:1074a0000200e80040049800480090000000e90055
:1074b000400498000d00e00002003200e24f550049
:1074c000040032000a00fb008080eb001c00320048
:1074d00010003700684890000004e00009003a00fe
:1074e000cfb097000100e00003003200bfb1970069
:1074f0008009eb00030037008fe897007fb097000a
:10750000014878000d00e00002003d00dfb1970067
:107510003304980011002000090037004800900053
:107520000000e900400498001800900098017800dd
:107530000001eb008900780003000100ddff370047
:10754000010078004f0778004f06be004f05be00cf
:107550004f04be000f01b10000000600889fbe006e
:10756000e30440000900a100808f54004a00360067
:10757000e38f540001003e0049002000727080003b
:107580000200e00002003200820078000c003700a8
:1075900001e1200003003700908f540023003600e3
:1075a0008080e800110078000000e000faff3a0057
:1075b0000f003700908f54001c0036008080e800d8
:1075c000110078000000e000faff3a001201780094
:1075d00001e1200003003700908f540013003600b3
:1075e0008080e80011007800820f5000faff3a0016
:1075f00068708000890f5400010031000904780090
:10760000080078005b0307000000e00004003a0077
:10761000890f5400200032000804d100f5ff370024
:10762000081878008efa0700d4ff3700110178009f
:107630009201780064805100890f500003003100ee
:107640001200900080087800070037000900410010
:1076500080087800920190001300980011007800d3
:107660001288140009097800910078000100e000f8
:1076700005003200110090000000e000020032001e
:107680000180e800010037000000eb007070880006
:107690000280e800010037000000eb004f04be004c
:1076a00000000600889fbe008004780066844000c9
:1076b00000ff2700180060004401de00f07f20007a
:1076c000800f51000e003a00800ceb001804780087
:1076d0006f0064001c003a00210090000000e000f0
:1076e00019003a00110090000000e00016003a0076
:1076f000100020001100e0001400320012003700da
:107700000200e00005003c000100780020030700b3
:10771000000178000000e00008003c00f0002800b4
:107720001800600001fe2300010c700020c02f0033
:10773000800c41000080eb0004003700800ceb005f
:107740000000eb0001003700200020004f04be00c5
:1077500000000600889fbe008a1f78008c9fbe0034
:10776000000478000206be00e6044000190178001b
:107770000200d0004505de008a007800f07f20007e
:10778000800f55000c003a006f00610067003a005e
:10779000280090000000e00064003a00180090000b
:1077a0000000e00061003a00100020001800e00036
:1077b0005f0032005d0037000a00e00007003a0079
:1077c00008007800f2020700800078000000e00066
:1077d000020034000a007800550037006108b90043
:1077e0000c0140008d814800e07f2000800f510097
:1077f000e08f59000d0034001900e00004003d0046
:107800006000b8000200200003ff2f0003003700d3
:107810006000b8000200200003ff2700009cbe00ab
:107820000294be001000200041003700e00f51001c
:10783000e08f590005003400f000280019006000b6
:10784000c410dd00810c700036003700190078008c
:1078500001002800010360006f0060000040a000ec
:10786000800c780061015100e0815900c0fc2f00bc
:10787000f1ff2f00800f5100818f590006003d005d
:10788000860c78000000eb0020049800100498009b
:10789000000c780026003700020078000881e8001c
:1078a000e400440005003700120c7800110978004c
:1078b00099087800800ceb0070004000f00f400049
:1078c000f9ff34008002ea00150032008881e800e8
:1078d00070821200980078008508de00130078009e
:1078e0000400dd00008c7000640144009300780007
:1078f0008508de00120078000400dd008089700039
:10790000920078008508de00190078000400dd0090
:1079100000897000190078000500de00800c7800f6
:10792000990c73000080eb0001003700200020005c
:107930004f06be004f0578004f04be000000060051
:107940000400fa00889fbe008a9fbe008c1f78004a
:107950000006780092bf9f00a3bf9f000404be00f2
:107960000401be001fb89700afb897004604070097
:107970000005be000001be000800be0001030700b4
:107980001fb99700afb997000000510081805900de
:1079900020069800310698000a8ebe000c00780080
:1079a0004f0678004f05be004f04be000080fa006d
:1079b000000006000e00fa00889fbe008a9fbe00ed
:1079c0008c9fbe0000047800014578000206780014
:1079d00083047800840678000300e00002003c0085
:1079e000190020002ce2200060c6b300804f550033
:1079f0000e00320060c4b300804f55000b0032000f
:107a000070c6b300804f55000300320070c4b3004d
:107a1000804f55009c003a00e48f460080003500fe
:107a200058089000808f56007d003d008d05e800cd
:107a300060c6b300804f55001000320060c4b30030
:107a4000804f55000d003200081090000038a30050
:107a500004003a0058089000808f540001003d0057
:107a6000590c9800580890000b005000500c9800da
:107a700002003b000000eb00500c98000b00e000ff
:107a800027003c00180990006800900001c3b30073
:107a9000017079008201e800130c980058089000ea
:107aa0000000e00003003c00081090000038a30034
:107ab0000500320068009000e1c2b30001f07900d7
:107ac0000280e800100c9800d80890000b00ea0033
:107ad000808f500001003d008105ea000b00ea00a4
:107ae000200c980001804500500c9800890f500030
:107af00001003d0080047800390c98006800900077
:107b00009808900001004000090178008c0078007e
:107b1000c7ed070058089000090050001a00370010
:107b200098089000680090008b8f540018003d006a
:107b300001004000090178008c007800bced0700ce
:107b40001808900000814400120c9800098055002c
:107b5000200c9800580890000000e00003003c0052
:107b6000081090000038a30006003200e8009000e2
:107b7000e0c2b30080707900380890000000e8008f
:107b8000300c980058089000400c9800a600370070
:107b9000010040000b0178008c007800a4ed070084
:107ba0001808900000814500120c98008b84540046
:107bb000580890000000e00003003c00081090000e
:107bc0000038a3000500320068009000e1c2b30055
:107bd000017079000200e800100c9800580890002d
:107be000890f500001003d0080047800680090007b
:107bf00098089000010040008b00460009017800c1
:107c00008bed07001808900000804400100c9800cd
:107c10005808900009005000200c9800820037009e
:107c200070c6b300804f55000300320070c4b3002b
:107c3000804f550014003a0058089000808f54007f
:107c400004003d00081090000038a30001003a0035
:107c5000590c9800580890000000e900500c98005a
:107c600002003b000000eb00500c980070c6b3000f
:107c7000804f550002003a005ac6b3000b0037008f
:107c80005ac4b3000900370010c6b300804f550036
:107c900002003a000ac7b3000400370010c4b30062
:107ca000804f550001003a000ac5b3001809900042
:107cb000680090003c7079008201e800130c980085
:107cc0000c027800580890000000e00003003c001f
:107cd000081090000038a30017003200e800900060
:107ce000e0c2b30080f079008280e800110c9800b7
:107cf000580890000000e0000f0034008904e900fb
:107d0000890f500001003d00800478006800900059
:107d100000804000090178008400780044ed0700ed
:107d20001808900000804400100c9800580890003b
:107d300009005000200c98006800900098089000fe
:107d4000010040000086e8000a58780080007800b2
:107d50000d00e00004003500b0c2b3008048780098
:107d60008c04780004003700d0c2b300804878004b
:107d70008c0478008d06ea008005eb000a003700cd
:107d8000a20020008d00780070805700cc01070011
:107d90000fb897009fb897007a81550001f17f00d6
:107da0008b05e800800678000d00e000f4ff3c0041
:107db000e18f550009003c0050c6b300804f5500cc
:107dc0000300320050c4b300804f550003003a0056
:107dd00000c3b300005e78008c0478000b00e00064
:107de000040032000b00e900fa80570000804000d8
:107df0000600370000c3b300805c78000500370040
:107e00008b05e90002c3b300a05c41000b00e00059
:107e1000fbff3c00680090009808900001004000c3
:107e200000805400300c980008109000740060002e
:107e3000f00f50000e003a00780090009808900073
:107e400001004000a808900001004000b808900020
:107e500001004000c80890008100400078089000b0
:107e6000808f500002003d0001005000000c98007f
:107e70004f06be004f05be004f04be000080fa0052
:107e8000000006000200fa00889fbe008a9fbe0024
:107e90008c1f7800800578000105780002067800c4
:107ea0000100e00001003a006c8557000b047800e7
:107eb000010037000804e800984478000900fb003e
:107ec000d4ef07000000e000faff3a00d0c2b30090
:107ed00080cf54000500320000c0e90080cf54007c
:107ee0000200320080447800010037000804e800f6
:107ef0000c0178008a007800080078003b00070039
:107f00000203be000002be009a0f540001003a00b6
:107f10000b0d78009a8f550005003a00e00f5200d3
:107f2000e08f5a00e00f5b00e08f5b0014003a0026
:107f3000b0c2b30080cf540006003a00e00f5200f8
:107f4000e08f5a00e00f5b00e08f5b0020003d00f7
:107f50000b003700d0c2b30080cf54001c003a00a1
:107f60006000b80002002000030028000020e100ab
:107f700001a8e10002b0e10003b8e1000e00360004
:107f800020022000e07088006b40400080cf540049
:107f900004003a006000b80002002000030028003e
:107fa0000d003700f0ff2f00f1ff2f00f2ff2f0030
:107fb000f3ff2700080037006000b8006011b80028
:107fc0000402500085825800060359008783590037
:107fd0000400be000601be004f0678004f05be003b
:107fe0004f04be000080fa0000000600fc87470036
:107ff000889fbe008a9fbe008c9fbe008e1f7800a7
:108000000007780081067800820478000004780078
:10801000010037000804e800184678000c00fb0057
:108020007cef07000000e000faff3a00d0c2b30086
:10803000804f56000500320000c0e900804f560016
:108040000200320000467800010037000804e80012
:108050000900e00005003500e18f54000300320004
:1080600040022000808f5400040034000d00e00026
:10807000b00032008e0e7800ae0037000900e0003c
:108080000e003400f08f54001a003a0000c3b30011
:10809000984f100016003a009840900080c7b30037
:1080a00080cf50000300320080c5b30080cf500065
:1080b0000f003a000884e8000e003700a9002000f5
:1080c00000c3b300984f10000a003a009840900097
:1080d00080c7b30080cf5000040032008900200028
:1080e00080c5b30080cf500002003a000884e80049
:1080f000090120000805780000c3b3000100370023
:108100000a05e8009a4f1000fdff32008a0578004a
:108110006022b8006033b8002600370030c4200069
:1081200080c0500081ef9f0009027800cfa2de00de
:1081300005037800860378000fb097009fb0970082
:108140002fb19700bfb197005e020700d0b79f0024
:10815000e1b79f00f2b79f0083bf9f000fe8970031
:108160000002fb00cfa2de00050378008603780042
:108170008b05e8000fb097009fb097002fb19700d4
:10818000bfb19700c0af9f00d1af9f00e2af9f008b
:10819000f3af9f005fb09700efb097007fb19700fb
:1081a0008fb997000002420081824a0002034b000f
:1081b00083834b0084b79f0095b79f00a6b79f00ad
:1081c000b7b79f001b00fb001aef07008000780084
:1081d0000901780030c420001def070080007800fe
:1081e0000000e000cdff3a008b0f54000a003a0077
:1081f0000d00e0004f0032008e0e78006022b800c3
:108200006033b80084b79f0095b79f00a6b79f0062
:10821000b7b79f004d0037008a805500e0c12000ad
:1082200060c07c000000fb00008050002c00330088
:108230004240a90020003c008fea97000500fb00a7
:10824000cf80de0001017800820178000fb2970034
:108250009fb297002fb39700bfb397000000520062
:1082600081805a0002015b0083815b000020e100f5
:1082700001a8e10002b0e10003b8e1000e003900fe
:1082800009027800cfa2de0005037800860378009b
:10829000230307004faa9700dfaa97006fab970050
:1082a000ffab97000400e1000588e1000690e100c3
:1082b0000798e1000a00320020022000e0708800e8
:1082c000f0ff2f00f1ff2f000001be0080b79f00dc
:1082d00091b79f00a2b79f00b3b79f00110037006e
:1082e000d0c2b300804f56000e003a006000b800c4
:1082f0006011b8000fb297009fb297002fb397009c
:10830000bfb397000402500085825800060359004d
:108310008783590084b79f0095b79f00a6b79f0039
:10832000b7b79f000d00e000080032008b0e780008
:10833000060037006000b8006011b80080b79f00e9
:1083400091b79f00a2b79f00b3b79f000fb09700ef
:108350009fb097002fb19700bfb197004f077800eb
:108360004f06be004f05be004f04be00cf01b10056
:10837000000006000000e000030034005c0007007d
:10838000e10f400001003a000000eb000000060091
:1083900000017800e6014000130078000100280089
:1083a000810360006f0060008009780012003a00cd
:1083b000220090000000e0000f003a001200900040
:1083c0000000e0000c003a00160020001200e0005f
:1083d0003800320008003700e400410091097800bd
:1083e0000280e80090087800120878000009eb008d
:1083f0007003530001003700160020001300e00056
:10840000f5ff3200e40241000282e800110037006b
:1084100080004000150078004f00de008089700069
:108420009500780081804000140078004f00de0045
:10843000808a7000940078008180400012007800eb
:108440004f00de00008a7000120078000009400032
:108450000603e90013007800ef0f5000ecff360030
:108460008282e800640241000e0037009200d100d1
:10847000150078004f00dd00008970009500d100e4
:10848000140078004f00dd00808a70009400d10055
:10849000130078004f00dd00008a70009309d100be
:1084a0000603e80013007800ff0f5000efff3e00c6
:1084b000ef09600093897300060078000000060051
:1084c00002027800809fbe00110009008200d800df
:1084d000000178004f00be0002a2b9008480500065
:1084e0001100980002087800000006000000050056
:1084f000889fbe0080047800307180000000e0009a
:1085000003003a00100007000000e0000a003500f8
:10851000307180000900e00002003a000004780099
:10852000060037000004780009004000060007003c
:108530000000e00001003d000084eb00080078002e
:108540004f04be0000000600800078000000e0003c
:1085500004003a0080e220003071880001017800b8
:10856000060037000081eb0080622100808f500000
:1085700002003e00317188000001eb00020078002b
:1085800000000600020ab900001bb9000200b80092
:108590008100420081004300000006006022b80014
:1085a000060220000000d0008180d2000482d200a8
:1085b0008582d2000000a0000202520083825a008d
:1085c000030031000202420083824a000000a10041
:1085d0000603e900f3ff3a0000000600889fbe0092
:1085e0008a9fbe00010578000100e000040035000c
:1085f00008003c000000e0002000320005003700c9
:1086000060001000e080180002003b0001f02c0028
:108610001a0037000004be006011b8006b0920008a
:108620000982cf00020039000882cf000441b00067
:10863000694252000e00320008003b008281710046
:10864000610164008904d1000884d3008b05e8002f
:108650000442e800f9ff3a0005003700080444002e
:1086600089844c008b05e9000442e900fbff3a00d5
:10867000b20007000af0a70001f0a0004f05be00fd
:108680004f04be000000060003f0a200889fbe0059
:108690008a9fbe008c1f7800ce000700d5003300f3
:1086a0006450e1004f0032006420e10052003200cb
:1086b00003826c0007003b000905d0000306d000d0
:1086c000820f54000c065d000200390002003200e7
:1086d00089017800030678008582550004003d007a
:1086e0000003fd008103fd008502ea008b85420046
:1086f000840f720002003b0060001000e080180050
:108700006011b8000005eb007a28e1000a0039008a
:1087100006007800c75ddd00f707b20087807500ae
:108720002d003700828171000a0178006105600028
:108730008180d1000080d3008502e900f9ff3b0071
:10874000060440008784480002003b0060041400d7
:10875000e0841c000988a300070032008a817100b0
:1087600082817100610164008904d1000884d30012
:108770008b05e800170037000978a30013003a00c2
:108780000b00e000130034008b05e90008044400ee
:1087900089844c000a4474000978a3000d003a0053
:1087a0000b00e000070034008b05e90008044400da
:1087b00089844c0001003a000b0020000978a300d6
:1087c000f7ff32000001eb000200370082817100e8
:1087d0000a017800590007000cf0a70001f0a00082
:1087e0008d0037006420e10002003a00838f6c00a6
:1087f0008d0033000801be000200be008600370075
:10880000889fbe008a9fbe008c1f78007100070001
:108810007800330003866c006450e10024003200cd
:108820006420e100270032006150e10022003200a4
:108830006120e100210032008b854200eb07b1008e
:108840000134b800003ab8000804420089844a00a4
:10885000013ab8000030b8008880400009014a00a1
:1088600004003300000040008180480002014900fc
:108870008b05e900c909dd008301700001003200a9
:1088800013002000c814de004814dd004709de0094
:108890001200b200c808de0008847000270007003c
:1088a00001f0a1000cf0a70001f0a0005a00370071
:1088b0006120e1005c0032000801be000200be0041
:1088c000f7ff37006150e100fcff3a005600370027
:1088d0000001be00570007000470a70003f0a100cc
:1088e00003f8a30013003a006509b100100032003c
:1088f000090035006928e100020035000100280068
:108900000000050000004000818048008502e90069
:10891000fcff3a0000000600f88f42000500350019
:108920008100d1000080d3008502e800fcff3a00fe
:10893000000006008000eb00000005008100200020
:10894000618055000b003d000b00200061fe2f00f0
:108950000100e1001d0034008281710061016400aa
:108960008904d1000884d3000000e800faff3a002f
:1089700071002000610064000300700002006000cc
:108980000900320061044400e0844c000988a5001d
:10899000050032008b05e8006808e10002003a009b
:1089a0008904d1000884d300f20f20000258e100ae
:1089b00005003d00c75ddd00f907b2008980750044
:1089c00008007800000006000bf827008b007800f4
:1089d000000005000004be00160007000003be00f2
:1089e0000405be000200be0012000700844f75009f
:1089f000000006000200be006450e10005003600e1
:108a00006420e100020036000968a30001003a007a
:108a10000800be000160a0004f0678004f05be00b0
:108a20004f04be0000000600f0ff2f00f1ff2700fa
:108a3000f9ff3700c70ade00f107b200f50fb200f8
:108a400008003200e1cf4200020032000170a000b5
:108a500024000500810f70000100320004080500a9
:108a600044000500810f700002003a001400050068
:108a70008502e9000000400081c04800fcff3b0087
:108a80000170a00024000500839f68000100e00041
:108a900002003d0060001000e08018000300e000cc
:108aa00002003d0060011100e0811900bbfe0700db
:108ab0004f00e00002003b0060001000e080180062
:108ac00000000600889fbe008a9fbe008c1f7800b1
:108ad0000205be000004be000006eb00e00f5000df
:108ae000e08f5800e00f5900e08f590007003d006b
:108af0006000b8006011b800080450008984580074
:108b00000a0559008b8559001c002000e00f520017
:108b1000e08f5a00e00f5b00e08f5b0002003d0039
:108b20000f0007000c00a2000800be000a01be00f2
:108b3000960207000203be000002be000c00e00027
:108b400001003200060007000400be000601be005e
:108b50004f0678004f05be004f04be00000006001f
:108b60006000b8006011b80004025000858258000f
:108b7000060359008783590000000600889fbe0045
:108b80008a9fbe00030578000300e0000500350061
:108b90000b003c00008270000402710030003200c3
:108ba0000700370060001000e08018006001190025
:108bb000e081190002003b0001f02d002800370081
:108bc0000004be000200be006011b8006b09200066
:108bd000950220000182cf000a0039000541b10052
:108be0000082cf00070039000541b1000982cf00a3
:108bf000040039000541b1000882cf0001003900ae
:108c00000541b10005425200120032000a003b004b
:108c100082817100610164008100d1000080d30075
:108c20008984d3000884d3008b05e8000442e8005f
:108c3000f7ff3a00070037000804440089844c001d
:108c400000004800818048008b05e9000442e900eb
:108c5000f9ff3a0039ff07000af0a70001f0a00071
:108c60004f05be004f04be000000060014002000a7
:108c700068023700811f78000100e00002003d001b
:108c800060001000e08018000300e00002003d00da
:108c900060011100e0811900050007004f00e000ad
:108ca00002003b0060001000e08018000000060099
:108cb0003afe07000400be000000060081037800b1
:108cc0005cff07000001be006000b8000478a3004c
:108cd00013003a006220e10015003e000d0039004b
:108ce0008301d1000281d3008180d3008301d100b0
:108cf0000281d3008180d3008301d1000281d3009f
:108d00008180d3000538b000c42add00f300b20032
:108d10008381720007f0a70003f0a00000000600a6
:108d2000f3ff2700f2ff2f006110b900fbff3700af
:108d300003ff2700f7ff3700881f78000004780042
:108d40005001be004000be00040040008580480085
:108d50000601490087814900009cbe000294be00c4
:108d60000400e1000588e1000690e1000798e100b9
:108d700002003100680044001008e8004f04780049
:108d800000000600f4874700889fbe008a9fbe004f
:108d90008c9fbe008e1f78000205be000004be003e
:108da000d4b79f00e5b79f00f6b79f0087bf9f002d
:108db0000000eb00c0b79f00b0b79f00a0b79f00b6
:108dc00090b79f0080b79f000d042000bfb09700b0
:108dd0004fb09700000140000000e0000f003d0090
:108de0004f08de0000007100c0b79f009e00070022
:108df00001003d0012002000a100070001003d001d
:108e000012002000a6000700b1000700b60007000e
:108e10000f004000c8ff0700220037004f08de00a7
:108e200000067100ccb79f008f00070001003d00d5
:108e3000120020009200070001003d0012002000f7
:108e400097000700a20007000fb297009fb297009b
:108e50002fb39700bfb39700a9000700000052008e
:108e600081805a0002015b0083815b0080b79f0014
:108e700091b79f00a2b79f00b3b79f000007eb0018
:108e80009f0007000020e10001a8e10002b0e1001e
:108e900003b8e100010031001e0020000e00560062
:108ea000c0b79f004fb297000400e00007003500f4
:108eb00010002000010020006011b80008047000bc
:108ec000898470000a0571008b8571008d06e900a8
:108ed000beff3a000400e00003003d0082000700ee
:108ee0000f00400094ff07004fa897000000e0002b
:108ef00004003a000fb497009fb497002fb5970075
:108f0000bfb59700940007004f0778004f06be00da
:108f10004f05be004f04be004f01b1000000060027
:108f2000881f780018002000881f780095ff070030
:108f30008f87e9004f04780000000600801feb00d7
:108f400090ff07008f87e90000000600889fbe00a1
:108f50008a9fbe008c1f78006e00070007003d004e
:108f600073000700e00f5b00e08f5b0007003d002f
:108f7000320007000006eb00040037003400070051
:108f800002003d002a0007001c00200072000700bc
:108f9000e3ff07000203be000002be000c00e00079
:108fa00001003200220007000400be000601be00de
:108fb0004f0678004f05be004f04be0000000600bb
:108fc000889fbe008a9fbe008c1f7800510007005a
:108fd00005003d0056000700e00f5b00e08f5b00de
:108fe00006003d00040037001900070003003d00a3
:108ff0006000b8006011b8001000070056000700bc
:10900000ceff07000203be000002be000c00e0001d
:1090100001003200060007000400be000601be0089
:109020004f0678004f05be004f04be00000006004a
:109030006000b8006011b800000037000402500062
:1090400085825800060359008783590000000600f6
:109050000006eb00e00f5200e08f5a00e00f5b00cb
:10906000e08f5b00000006000180400090b79f0089
:109070000001eb008fb097000100e0000000060047
:109080000200700090b79f000180400080b79f00f1
:109090000001eb00ffa897000100e00000000600bf
:1090a0000200700080b79f00018040006faa970007
:1090b000cf20de0001007000f0af9f0004024200ec
:1090c000250007004f18de000002720000000600b5
:1090d000e4af9f000804440089844c000a054d0059
:1090e0008b854d00000006003fb29700cfb297007d
:1090f0005fb39700efb3970000fe2f00000006005b
:109100003fb09700cfb097005fb19700efb19700e5
:10911000000006000205be000004be00e00f500083
:10912000e08f5800e00f5900e08f59000000060062
:109130006000b8006011b80008045000898458002d
:109140000a0559008b8559001c002000e00f5200d1
:10915000e08f5a00000006000800be000a01be00b1
:10916000000006008f1fd100450107008f87e9002e
:109170000000e000000006001400fa00889fbe0016
:109180008a9fbe008c9fbe000004be000205be0088
:10919000680047000a90be000890be006101070009
:1091a0000070a7000bf0a100304320009e02900049
:1091b00080825200b0fe2f000028e10011003d0027
:1091c000b0fc2f000028e100150034001e099000bb
:1091d0008e0890007e0090000501b0000201d100d1
:1091e0008180d3000080d3008502e800fbff3a00b5
:1091f0000b00e00086013b0060001000e0801800da
:1092000083013700f0ff2f00f1ff27000b00e00083
:109210007f013b0001002800000020007c01370096
:109220006000b8007a0137004f89de0082017800c3
:109230007c01370007f0a200b1013700809feb00ee
:109240000f0107008f87e9000000e0000000060022
:109250002800fa00889fbe008a9fbe008c9fbe0037
:1092600003866b00560107000028a30064003a0043
:109270000128a30067003a000008a30062003a003a
:109280000108a30065003a001e009000be0890008f
:1092900081064000ed3fb100f4805700ee019000e0
:1092a000111ab8008e099000311bb8009e09900079
:1092b000311cb800511db800f48557004600070066
:1092c000fe0190003a0007008b85e8003e00070091
:1092d0008e09900040000700ee0190003400070066
:1092e0008b85e800380007008e09900040000700d9
:1092f0009e0990001b18b800890440000a854800a8
:10930000fe019000340007008b85e800380007005c
:10931000ee019000300007008e0990001b18b80085
:10932000890440000a8548000a98a30008003a0012
:109330000402420085824a0006034b0087834b00eb
:1093400008044c0089844c000a054d008d06e90094
:1093500084827200850273004c3add00850272003f
:109360000100320015002000443ade001400b20073
:109370004538de00cb45dd000b007000c540de0047
:10938000cb4ddd008b8070004549de00cb55dd0004
:109390000b017100c551de000d037800d5010700f7
:1093a00003f0a1000cf0a70003f0a00018013700a3
:1093b0001b18b8008502400006834800e0834b007c
:1093c00060044c00070037001b18b800060340007b
:1093d00087834800faff37001b18b8008703400056
:1093e00008844800e0844c0060054d000000060041
:1093f0001b18b8000804400089844800faff3700b1
:109400000108a300ff003a005800be005801be004a
:10941000e3ff37000008a300fa003a0009047800cf
:10942000f9ff37002800fa00889fbe008a9fbe001f
:109430008c9fbe0003866b00e10007006400e10022
:10944000440032006408e1004a0032006100e1009b
:10945000460032006108e10049003200ec06470096
:109460006000b8003d02be003d03be00f486570018
:109470006011b8003d04be003d05be007d03200024
:109480000b0037000000a0008d06e9001300320039
:109490000402420085824a0006034b0087834b008a
:1094a000000040008180480002014900838149009a
:1094b0000802520089825a000a035b008b835b001a
:1094c000f0ff3b000802420089824a000a034b0079
:1094d0008b834b008d06e900edff3a008482720019
:1094e00086827200f707b2008782720001003200a4
:1094f000150020001e0490003e0b9000060354004f
:10950000e63fb0000368a300070032000000a70098
:109510000500a0008301d1000281d3008180d30027
:109520000080d3000603e8008301d1000281d3004c
:109530008180d3000080d3000002eb000482d200bf
:109540006c01070003f0a1000cf0a70003f0a000dd
:10955000af003700640247006408e100a900320050
:109560003400be003401be00f6ff37006108e100a0
:10957000a40032006011b8006000b800f1ff3700ad
:1095800003ff270002002000fbff3700889fbe007a
:109590008a9fbe008c9fbe000404b8000506b80078
:1095a0008904460060854e000606b8000a0546009c
:1095b000e0854e000706b8008b054600040eb80093
:1095c000890446000a854e00e0854d00050eb8006e
:1095d0000a0546008b854e00060eb8008b05460036
:1095e0000416b8000a0546008b854e000516b80023
:1095f0008b054600041eb8008b0546000800be001f
:109600000a01be004f06be004f05be004f04be005b
:1096100000000600889fbe008a9fbe00841f78005d
:10962000ecfc07004f00780011003300f0ff2f0022
:10963000838f6c0006003b00040565000a00a7004c
:109640000800370009f0a6001000200008003700cd
:10965000820f5400838f5c0003003900100020004b
:1096600001003e000000200009f0a7000000ea0011
:109670004f05be004f04be000000e00000000600e1
:10968000889fbe008a9fbe008c9fbe000404be005f
:109690000605be00809fbe00829fbe0041010700fc
:1096a000040678000800be000a01be003d01070064
:1096b000840678004f03be004f02be008d4f760037
:1096c0007fb0970013003300f0ff2f008b8f6b00eb
:1096d00006003b000d0666000c00a7000a003700dc
:1096e00007f0a600100020000a003700880f520083
:1096f000898f5a008a0f5b008b8f5b000300390053
:109700001000200001003e000000200007f0a7002c
:109710000000ea004f06be004f05be004f04be0029
:1097200000000600800078005002be005003be001a
:109730004439de00f700b200f37f2000030161002e
:10974000090032000218e10016003a00850172009b
:1097500083017300838173000008200015003a0024
:109760004000200013003700850172008301730060
:109770008381730005003a0004a8be0006a8be005d
:10978000100020000b0037000201e9000402420033
:1097900085824a0006034b0087834b000748a300dd
:1097a000f9ff32000740a00004a8be0006a8be00d2
:1097b0002000200080009800920098000000060021
:1097c000680447000294be000094be00fc044700f9
:1097d0008694be008494be0009007800d1ff070083
:1097e00008007800cfff070099007800814f7000d3
:1097f0000b003b000800be00fc0007004f00b1005a
:1098000003003700f3ff2700f2ff2f006110b900bb
:109810004f06be004f05be004f04be000080fa0098
:1098200000000600889fbe00830478000300e0006b
:109830002c00350003003c0000827000040271001f
:109840002600320036432000c50020008383cf006d
:109850000a0039000541b1008283cf0007003900ba
:109860000541b1008183cf00040039000541b100fa
:109870008083cf00010039000541b10085c353004a
:109880006022b800120032000a003b00848272009d
:10989000610260008301d1000281d3008180d30086
:1098a0000080d3000603e8008743e800f7ff3a0092
:1098b0000700370000004000818048000201490095
:1098c000838149000603e9008743e900f9ff3a0074
:1098d0008800070009f0a70003f0a0004f04be00b5
:1098e0000000060060001000e08018006001190010
:1098f000e0811900d3ff3b00033e2c00f7ff370047
:109900002800fa00889fbe008a9fbe008c9fbe0080
:1099100007067800878669000c003b000304780086
:109920008704780008f0a10009f0a100840f50001e
:10993000858f5800860f5900890f5c0003003300a3
:109940000cf0a20001003a000cf0a1009cff0700ff
:109950006400e1005f003200780147006408e10024
:10996000610032006c014700748557003200be0070
:109970001201be003a04be001a05be001e0390008c
:10998000be0a90008503530006003d000004fd0060
:109990008104fd000205fd008305fd008703ea0048
:1099a000050378000df8a3000400320060041400e1
:1099b000e0841c0060051d00e0851d006022b800e9
:1099c0007d0320000d38e1008006eb000b0039001c
:1099d0004433dd00f300b200830173003900370027
:1099e000848272000d027800e10664008b85d1004c
:1099f0000a85d3008984d3000884d3008703e90053
:109a0000f7ff3b0008004000898048000a01490038
:109a10008b81490004003b0060001000e0801800ca
:109a200060011900e08119000358a3000900320009
:109a30008d82720084827200610260008301d10015
:109a40000281d3008180d3000080d3000603e800a8
:109a50001b0037000348a30017003a000600e0008f
:109a6000170034000603e9000d00a30000004800c1
:109a70008180480002014900838149000348a30016
:109a80000f003a000600e000090034000603e90078
:109a900000004000818048000201490083814900a4
:109aa00001003a000003eb000348a300f5ff320079
:109ab0006022b80002003700848272006182660072
:109ac0000c00070003f0a1000cf0a70003f0a000b9
:109ad0004fff3700640147006408e10002003a00cc
:109ae0000df8a30047ff3a003200be001201be008d
:109af00047ff3700180020005700200008045300db
:109b00000d003d000600200097fc2f000740e100fb
:109b10001e00340084827200610260008301d10063
:109b20000281d3008180d3000080d3000804e800c4
:109b3000f8ff3a004700200061046000050474004b
:109b4000040464000d00320061004000e080480021
:109b500060014900e081490003b8a5000700320018
:109b60000603e8006538e10004003a008301d100f3
:109b70000281d3008180d3000080d300f87f2000d1
:109b80000830e10003003500080378006000b800e9
:109b90006011b8004433dd00f300b20083017300ac
:109ba0000000060005ff2700058261000700320063
:109bb0000428e1000100320024000500060007002f
:109bc00001003a00440005000408050002000700f7
:109bd000f9ff3a00140005006f82610081027000f5
:109be000850271008502720000000600e4824000d8
:109bf0001078a30007003200640240001178a3002f
:109c00003400be001401be00040032000330a7007f
:109c1000000006003500be001501be000330a000a4
:049c2000000006003a
:020000040000fa
:020000040005f5
:0457f400ffff0000b3
:020000040000fa
:020000040005f5
:0457f8009d7200009e
:020000040000fa
:020000040005f5
:0457fc007f3f0000eb
:020000040000fa
:10000800fc0f0000fc0f0000fc0f0000fc0f0000bc
:10001800fc0f0000fc0f0000fc0f0000fc0f0000ac
:10002800fc0f0000fc0f0000fc0f0000fc0f00009c
:10003800fc0f0000fc0f0000fc0f0000ae7c00006d
:10004800fc0f0000fc0f0000fc0f0000b86b000064
:10005800a06b0000fc0f0000fc0f0000fc0f00006c
:10006800fc0f0000fc0f0000fc0f0000fc0f00005c
:10007800fc0f0000fc0f0000fc0f0000fc0f00004c
:10008800fc0f0000fc0f0000fc0f0000fc0f00003c
:10009800fc0f0000fc0f0000126c0000fa6b00005f
:1000a800fc0f0000fc0f0000fc0f0000fc0f00001c
:1000b800fc0f0000fc0f0000fc0f0000fc0f00000c
:1000c800fc0f0000fc0f0000fc0f0000fc0f0000fc
:1000d800fc0f0000fc0f0000fc0f0000fc0f0000ec
:1000e800fc0f0000fc0f0000fc0f0000fc0f0000dc
:1000f800fc0f0000fc0f0000fc0f0000fc0f0000cc
:10010800fc0f0000fc0f0000fc0f0000fc0f0000bb
:10011800fc0f0000fc0f0000fc0f0000fc0f0000ab
:10012800fc0f0000fc0f0000fc0f0000fc0f00009b
:10013800fc0f0000fc0f0000fc0f0000fc0f00008b
:10014800fc0f0000fc0f0000fc0f0000fc0f00007b
:10015800fc0f0000fc0f0000fc0f0000fc0f00006b
:10016800fc0f0000fc0f0000fc0f0000fc0f00005b
:10017800fc0f0000fc0f0000fc0f0000fc0f00004b
:10018800fc0f0000fc0f0000fc0f0000fc0f00003b
:10019800fc0f0000fc0f0000fc0f0000fc0f00002b
:1001a800fc0f0000fc0f0000fc0f0000fc0f00001b
:1001b800fc0f0000fc0f0000fc0f0000fc0f00000b
:1001c800fc0f0000fc0f0000fc0f0000fc0f0000fb
:1001d800fc0f0000fc0f0000fc0f0000fc0f0000eb
:1001e800fc0f0000fc0f0000fc0f0000fc0f0000db
:0801f800fc0f0000fc0f0000e9
:020000040000fa
:10020800fc0f0000fc0f0000fc0f0000fc0f0000ba
:10021800fc0f0000fc0f0000fc0f0000fc0f0000aa
:10022800fc0f0000fc0f0000fc0f0000fc0f00009a
:10023800fc0f0000fc0f0000fc0f0000ae7c00006b
:10024800fc0f0000fc0f0000fc0f0000b86b000062
:10025800a06b0000fc0f0000fc0f0000fc0f00006a
:10026800fc0f0000fc0f0000fc0f0000fc0f00005a
:10027800fc0f0000fc0f0000fc0f0000fc0f00004a
:10028800fc0f0000fc0f0000fc0f0000fc0f00003a
:10029800fc0f0000fc0f0000126c0000fa6b00005d
:1002a800fc0f0000fc0f0000fc0f0000fc0f00001a
:1002b800fc0f0000fc0f0000fc0f0000fc0f00000a
:1002c800fc0f0000fc0f0000fc0f0000fc0f0000fa
:1002d800fc0f0000fc0f0000fc0f0000fc0f0000ea
:020000040000fa
:020000040000fa
:109c24000d0a000000480000454c000050200000d0
:109c34002d20000064690000737000006c61000056
:109c4400792000007468000069730000206d000032
:109c5400656e0000750d00000a0000005449000004
:109c64004d450000202d00002064000069730000b1
:109c7400706c0000617900002063000075720000c0
:109c8400726500006e7400002064000061740000be
:109c940065200000616e000064200000746900000b
:109ca4006d6500000d0a00000052000045530000dd
:109cb40045540000202d0000207200006573000050
:109cc40065740000207400006865000020630000d3
:109cd4006f6e0000747200006f6c00006c65000011
:109ce400720d00000a0000005041000052410000c3
:109cf4004d2000002d200000736800006f770000e5
:109d04002063000075720000726500006e7400002c
:109d1400206300006f6e0000666900006720000089
:109d240070610000726100006d65000074650000e0
:109d3400727300000d0a0000005300004156000039
:109d4400452000002d2000007361000076650000ae
:109d54002063000075720000726500006e740000dc
:109d6400206300006f6e0000666900006720000039
:109d740070610000726100006d6500007465000090
:109d8400727300000d0a0000004400004546000004
:109d9400415500004c540000202d000020720000aa
:109da40065730000746f000072650000206300009a
:109db4006f6e00006669000067200000706100009b
:109dc400726100006d65000074650000727300002c
:109dd400207400006f2000006465000066610000cc
:109de400756c0000747300000d0a0000004200004e
:109df40041540000542000002d2000006d65000037
:109e04006173000075720000652000007468000032
:109e14006520000062610000747400006572000037
:109e240079200000766f00006c7400006167000008
:109e3400650d00000a0000004c4100004e43000084
:109e4400204d00004f440000452000002d2000005c
:109e540043740000726c00002d4c0000207400005c
:109e64006f200000656e000074650000722c000015
:109e740020430000747200006c2d00005820000084
:109e8400746f00002065000078690000740d000004
:109e94000a000000434100004d200000505700001c
:109ea400522000002d20000074750000726e000026
:109eb40020630000616d00006572000061200000f5
:109ec400706f000077650000722000006f6e000064
:109ed400206f0000722000006f660000660d000015
:109ee4000a0000004c4500004431000020500000ee
:109ef40057520000202d00002074000075720000ed
:109f04006e2000004c450000442000006c690000f5
:109f1400676800007420000031200000706f0000aa
:109f240077650000722000006f6e0000206f000053
:109f3400722000006f660000660d00000a00000039
:109f44004c450000443200002050000057520000ed
:109f5400202d000020740000757200006e200000a7
:109f64004c450000442000006c6900006768000054
:109f74007420000032200000706f0000776500003c
:109f8400722000006f6e0000206f0000722000003d
:109f94006f660000660d00000a00000048440000df
:109fa4004d4900002050000057520000202d0000b1
:109fb40020740000757200006e2000004844000008
:109fc4004d490000207400006f2000004e54000032
:109fd40053430000206300006f6e000076650000ac
:109fe4007274000065720000207000006f7700003a
:109ff40065720000206f00006e2000006f72000088
:10a00400206f0000666600000d0a00000053000087
:10a01400545200004f4200004520000050570000f9
:10a02400522000002d20000074750000726e0000a4
:10a0340020730000747200006f620000652000004d
:10a04400706f000077650000722000006f6e0000e2
:10a05400206f0000722000006f660000660d000093
:10a064000a000000494e0000535400002050000034
:10a0740057520000202d000020740000757200006b
:10a084006e200000696e0000737400007275000099
:10a094006d6500006e740000207000006f77000092
:10a0a40065720000206f00006e2000006f720000d7
:10a0b400206f0000666600000d0a000000490000e1
:10a0c4004e5300005432000020500000575200004c
:10a0d400202d000020740000757200006e20000026
:10a0e400696e000073740000727500006d650000f5
:10a0f4006e7400002832000029200000706f0000f8
:10a1040077650000722000006f6e0000206f000071
:10a11400722000006f660000660d00000a00000057
:10a124004745000054200000494d0000414700000d
:10a13400452000002d2000007472000069670000b3
:10a144006765000072200000636100006d65000017
:10a1540072610000206900006d6100006765000005
:10a1640020630000617000007475000072650000d7
:10a174000d0a00000047000045540000205600006e
:10a1840049440000454f0000202d000020740000c9
:10a1940072690000676700006572000020630000b8
:10a1a400616d0000657200006120000076690000a6
:10a1b400646500006f20000063610000707400009b
:10a1c40075720000650d00000a000000474500009c
:10a1d4005420000054520000494700003120000080
:10a1e4002d200000676500007420000073740000d7
:10a1f40061740000652000006f6600002074000098
:10a204007269000067670000657200002069000041
:10a214006e70000075740000203100000d0a00000b
:10a22400004700004554000020540000524900003b
:10a2340047320000202d00002067000065740000f4
:10a24400207300007461000074650000206f00003a
:10a2540066200000747200006967000067650000f2
:10a2640072200000696e0000707500007420000008
:10a27400320d00000a000000534500005420000085
:10a28400544900004d450000202d000020730000bb
:10a2940065740000206300007572000072650000a0
:10a2a4006e74000020740000696d000065200000d9
:10a2b4004d4d00002f440000442f00005959000068
:10a2c40020480000483a00004d4d00003a53000079
:10a2d4005320000044410000590d00000a00000012
:10a2e4005345000054200000434100005054000036
:10a2f40055520000452000004d4f00004445000029
:10a30400202d00002073000065740000206300000d
:10a31400617000007475000072650000206d00001b
:10a324006f640000652000005b4f0000464600009b
:10a334007c4900004d4700007c5600004944000061
:10a344005d0d00000a000000534500005420000089
:10a3540044450000504c00004f59000020440000c8
:10a36400454c000041590000202d000020730000de
:10a374006574000020640000657000006c6f0000cc
:10a38400796d0000656e00007420000064650000b3
:10a394006c61000079200000696e0000206d0000ef
:10a3a400696e000075740000657300000d0a0000fa
:10a3b40000530000455400002044000045500000b4
:10a3c4004c4f000059200000445500005241000049
:10a3d400544900004f4e0000202d0000207300005f
:10a3e4006574000020640000657000006c6f00005c
:10a3f400796d0000656e0000742000006475000033
:10a4040072610000746900006f6e00002069000032
:10a414006e2000006d6900006e7500007465000018
:10a42400730d00000a000000534500005420000092
:10a43400534100004d5000004c45000020490000ed
:10a444004e54000045520000564100004c200000cc
:10a454002d2000007365000074200000736100006b
:10a464006d7000006c650000206900006e740000cf
:10a4740065720000766100006c200000696e0000c7
:10a48400206d0000696e00007574000065730000a3
:10a494000d0a00000053000045540000205600003f
:10a4a40049440000454f000020440000555200007c
:10a4b40041540000494f00004e2000002d200000b0
:10a4c4007365000074200000766900006465000074
:10a4d4006f20000064750000726100007469000060
:10a4e4006f6e0000206900006e200000736500009c
:10a4f400636f00006e640000730d00000a0000002a
:10a504005345000054200000424100005454000010
:10a51400204c000045560000454c0000202d000052
:10a524002073000065740000206d0000696e000057
:10a53400696d0000756d0000206f000070650000fb
:10a5440072610000746900006e6700002062000000
:10a5540061740000742000006c65000076650000e2
:10a564006c2000000d0a0000005b0000444600005f
:10a574004c5400005d00000020200000202000005a
:10a5840020200000004f0000464600000049000063
:10a594004d4700000056000049440000003f000001
:10a5a4003f3f0000004300004150000054550000ac
:10a5b40052450000204d00004f440000452000009b
:10a5c4002020000020250000732000003a20000015
:10a5d400257300000d0a00000044000045500000ef
:10a5e4004c4f000059200000444500004c4100003d
:10a5f40059200000202000002025000073200000c6
:10a604003a200000256c0000752000004d49000030
:10a614004e0d00000a00000044450000504c0000ac
:10a624004f590000204400005552000041540000de
:10a63400494f00004e20000025730000203a00001e
:10a64400202500006c750000204d0000494e0000dc
:10a654000d0a000000530000414d0000504c000062
:10a6640045200000494e00005445000052560000a9
:10a67400414c000020250000732000003a20000017
:10a68400256c0000752000004d4900004e0d0000af
:10a694000a00000056490000444500004f20000015
:10a6a4004455000052410000544900004f4e000040
:10a6b4002020000025730000203a0000202500001f
:10a6c4006c75000020530000454300000d0a000093
:10a6d4000042000041540000542000004c4500009a
:10a6e400564500004c2000002020000020200000df
:10a6f40020250000732000003a200000256c000093
:10a70400752000006d5600000d0a00000042000094
:10a7140041540000544500005259000020560000e6
:10a724004f4c0000542000003a2000002575000022
:10a73400206d0000560d00000a0000004f4e00007e
:10a7440000430000414d000020500000575200001b
:10a75400204f00004e0d00000a000000434100009d
:10a764004d20000050570000522000004f460000ca
:10a77400460d00000a0000004c4500004431000072
:10a784002050000057520000204f00004e0d0000e2
:10a794000a0000004c450000443100002050000035
:10a7a40057520000204f0000464600000d0a0000ea
:10a7b400004c0000454400003220000050570000c7
:10a7c400522000004f4e00000d0a0000004c000013
:10a7d4004544000032200000505700005220000081
:10a7e4004f460000460d00000a00000048440000e7
:10a7f4004d4900002050000057520000204f000037
:10a804004e0d00000a000000484400004d490000bd
:10a814002050000057520000204f00004646000020
:10a824000d0a000000530000545200004f42000083
:10a834004520000050570000522000004f4e0000f9
:10a844000d0a000000530000545200004f42000063
:10a854004520000050570000522000004f460000e1
:10a86400460d00000a000000494e00005354000049
:10a874002050000057520000204f00004e0d0000f1
:10a884000a000000494e000053540000205000000c
:10a8940057520000204f0000464600000d0a0000f9
:10a8a400004900004e5300005432000020500000c4
:10a8b40057520000204f00004e0d00000a00000017
:10a8c400494e00005354000032200000505700004d
:10a8d400522000004f460000460d00000a00000010
:10a8e4004445000042550000472000004d4f000041
:10a8f4004445000020490000532000004f4e000052
:10a904000d0a0000004400004542000055470000c5
:10a91400204d00004f440000452000004953000032
:10a92400204f0000464600000d0a000000440000cd
:10a934004542000055470000204d00004f440000f0
:10a944004520000049530000200000004d45000050
:10a954004f5700000d0a0000005400006865000015
:10a96400726500002061000072650000202500006f
:10a974006620000073650000636f00006e640000d1
:10a9840073200000756e0000746900006c200000e4
:10a994006d690000646e000069670000687400005f
:10a9a4002e0d00000a000000256400002025000090
:10a9b400642000002564000000720000746300003d
:10a9c400446d0000795400006f4400006f7900006a
:10a9d40028250000642c000020250000642c0000c1
:10a9e4002025000064290000203d000020250000ef
:10a9f400640d00000a00000045520000523a0000b5
:10aa0400204900004d41000047450000204300005c
:10aa140041500000545500005245000020420000ff
:10aa240055530000590d00000a0000004552000073
:10aa3400523a00002056000049440000454f0000ef
:10aa440020430000415000005455000052450000ce
:10aa54002042000055530000590d00000a00000078
:10aa640054520000494700004745000052200000ae
:10aa7400313a0000200000004f4e00000d0a000093
:10aa8400004f0000464600000d0a0000005400007c
:10aa940052490000474700004552000020320000a0
:10aaa4003a20000000250000642f00002564000007
:10aab4002f25000064200000256400003a250000d2
:10aac400643a0000256400002025000064000000b2
:10aad40045520000523a0000204200004144000068
:10aae400204600004f5200004d410000540d00006c
:10aaf4000a0000005553000041470000453a000099
:10ab0400204d00004d2f0000444400002f59000048
:10ab140059200000484800003a4d00004d3a00001a
:10ab24005353000020440000415900002028000035
:10ab34000044000041590000203d00002031000085
:10ab44002d3e0000537500006e2c000020320000e2
:10ab54002d3e00004d6f00006e2c0000202e0000e2
:10ab64002e2e0000202c0000203700002d3e000077
:10ab740053610000742900000d0a00000045000024
:10ab8400525200003a2000004d4f00004e54000085
:10ab9400482000004f550000542000004f4600009c
:10aba40020520000414e00004745000020280000cc
:10abb400312000002d20000031320000290d00005a
:10abc4000a00000045520000523a000020440000f0
:10abd40041590000204f000055540000204f000050
:10abe40046200000524100004e470000452000006e
:10abf40028310000202d00002033000031290000fe
:10ac04000d0a000000450000525200003a200000e6
:10ac14005945000041520000204f000055540000e7
:10ac2400204f000046200000524100004e47000023
:10ac3400452000002028000031310000202d0000b4
:10ac440020390000392900000d0a000000450000e9
:10ac5400525200003a200000484f000055520000b4
:10ac6400532000004f550000542000004f460000c0
:10ac740020520000414e0000474500002020000003
:10ac840028310000202d000020320000342900006b
:10ac94000d0a000000450000525200003a20000056
:10aca4004d4900004e55000054450000532000005b
:10acb4004f550000542000004f4600002052000071
:10acc400414e0000474500002020000028300000cd
:10acd400202d000020350000392900000d0a000055
:10ace40000450000525200003a2000005345000085
:10acf400434f00004e440000532000004f55000015
:10ad0400542000004f46000020520000414e000035
:10ad1400474500002020000028300000202d0000be
:10ad240020350000392900000d0a0000004500000c
:10ad3400525200003a200000444100005920000013
:10ad44004f550000542000004f46000020520000e0
:10ad5400414e00004745000020200000283100003b
:10ad6400202d000020370000290d00000a000000fb
:10ad7400544900004d450000205300004554000094
:10ad8400205400004f3a00002000000061630000de
:10ad9400744300006c72000053740000756200007c
:10ada400436d00006428000025730000290d000095
:10adb4000a0000002a2a00002a200000544900004a
:10adc4004d450000204c0000415000005345000058
:10add4002053000043480000454400002054000074
:10ade400415300004b2000002a2a00002a0d0000d5
:10adf4000a000000746900006d6500004c610000e9
:10ae0400707300006553000063680000656400000f
:10ae14005374000061740000652000003d200000b0
:10ae2400005400004c5f00005343000048450000fc
:10ae3400445f00005741000049540000494e00009f
:10ae440047000000544c00005f53000043480000da
:10ae5400454400005f520000554e00004e4900007a
:10ae64004e470000005400004c5f000053430000b4
:10ae740048450000445f0000535400004f50000058
:10ae84005045000044000000554e00004b4f0000a8
:10ae9400574e0000000d00000a0000007469000015
:10aea4006d6500004c610000707300006553000084
:10aeb4006368000065640000576100006974000065
:10aec400203d0000202500006c7500002053000088
:10aed40045430000530d00000a000000746d00009b
:10aee400724700006574000053650000636f000042
:10aef4006e64000073280000292000002020000058
:10af0400203d0000202500006c7500002053000047
:10af140045430000530d00000a000000546900007e
:10af24006d65000020520000656d0000616900003d
:10af34006e6900006e6700002020000020200000e1
:10af4400203d0000202500006c7500002053000007
:10af540045430000530d00000a0000000d0a0000e4
:10af64002a2a00002a200000544900004d45000010
:10af7400204c0000415000005345000020490000cf
:10af84004d4100004745000020540000415300009b
:10af94004b2000002a2a00002a0d00000a000000ad
:10afa400746900006d6500004c610000707300005e
:10afb400654900006d61000067650000537400007e
:10afc40061740000652000003d2000000074000052
:10afd400696d0000654c000061700000736500003d
:10afe400496d00006167000065540000696d000050
:10aff40065720000203d0000202500006c750000f3
:10b00400206d0000730d00000a0000000d0a00000e
:10b014002a2a00002a200000544900004d4500005f
:10b02400204c000041500000534500002056000011
:10b0340049440000454f00002054000041530000e3
:10b044004b2000002a2a00002a0d00000a000000fc
:10b05400746900006d6500004c61000070730000ad
:10b064006556000069640000656f000053740000b9
:10b0740061740000652000003d20000000740000a1
:10b08400696d0000654c000061700000736500008c
:10b0940056690000646500006f540000696d00008b
:10b0a40065720000203d0000202500006c75000042
:10b0b400206d0000730d00000a0000000d0a00005e
:10b0c4002a2a00002a200000544900004d450000af
:10b0d400204c000041500000534500002042000075
:10b0e4005f4d00004f4e000020540000415300000b
:10b0f4004b2000002a2a00002a0d00000a0000004c
:10b10400746900006d6500004c61000070730000fc
:10b114006542000061740000744d00006f6e000011
:10b124005374000061740000652000003d2000009d
:10b13400005400004c5f0000425f00004d4f0000cf
:10b144004e5f0000494e00004954000000540000c6
:10b154004c5f0000425f00004d4f00004e5f000056
:10b164004c4f000057000000544c00005f420000a8
:10b174005f4d00004f4e00005f4e00004f52000034
:10b184004d4100004c000000544c00005f420000a0
:10b194005f4d00004f4e00005f530000544f00000d
:10b1a400505000004544000000740000696d000028
:10b1b400654c00006170000073650000426100008e
:10b1c400747400004d6f00006e540000696d00003f
:10b1d40065720000203d0000202500006c75000011
:10b1e400206d0000730d00000a0000006261000081
:10b1f4007474000065720000795600006f6c0000e2
:10b2040074730000203d000020250000752000001c
:10b214006d5600000d0a000000740000736b0000fe
:10b224005374000061720000744900006d610000f5
:10b2340067650000436100007074000075720000cf
:10b2440065280000292000005b200000005d00004c
:10b254000d0a000000740000696d0000654c0000d8
:10b264006170000073650000496d000061670000b3
:10b27400655300007461000074650000203d000007
:10b28400205400004c5f0000494d0000414700007d
:10b29400455f00005354000041520000540d00006b
:10b2a4000a00000045520000523a000020740000d9
:10b2b400696d0000654c000061700000736500005a
:10b2c400496d00006167000065530000746100006f
:10b2d40074650000203d000020000000455200007d
:10b2e400523a000020740000696d0000654c0000b3
:10b2f4006170000073650000566900006465000019
:10b304006f5300007461000074650000203d00006c
:10b3140020000000747300006b530000746100008f
:10b324007274000056690000646500006f430000f9
:10b334006170000074750000726500002829000027
:10b34400205b000020000000746900006d650000af
:10b354004c610000707300006556000069640000d1
:10b36400656f0000537400006174000065200000e4
:10b374003d200000544c00005f560000494400008a
:10b38400454f00005f530000544100005254000038
:10b394000d0a0000005400004c5f0000494d0000fd
:10b3a40041470000455f0000535400004152000033
:10b3b40054000000544c00005f4900004d4100005f
:10b3c400474500005f5000004f5700004552000001
:10b3d4005f3100005f570000414900005400000045
:10b3e400544c00005f4900004d41000047450000f7
:10b3f4005f5000004f570000455200005f320000cc
:10b404005f5700004149000054000000544c000004
:10b414005f4900004d410000474500005f500000b7
:10b42400484f0000544f00005f570000524900008d
:10b4340054450000005400004c5f0000494d0000da
:10b4440041470000455f0000504800004f54000091
:10b454004f5f0000574100004954000000540000b1
:10b464004c5f0000494d000041470000455f00006b
:10b474004c4100004e4300005f4f00004646000070
:10b48400005400004c5f0000494d0000414700009b
:10b49400455f0000504f000057450000525f000018
:10b4a400444f0000574e0000005400004c5f000061
:10b4b400494d000041470000455f0000524500002f
:10b4c4004144000059000000544c00005f49000052
:10b4d4004d410000474500005f5500004e4b000001
:10b4e4004e4f0000574e0000005400004c5f000017
:10b4f40056490000444500004f5f000053540000cb
:10b504004152000054000000544c00005f560000fb
:10b5140049440000454f00005f5000004f570000b1
:10b52400455200005f3100005f57000041490000b0
:10b5340054000000544c00005f56000049440000d1
:10b54400454f00005f5000004f5700004552000077
:10b554005f3200005f5700004149000054000000c2
:10b56400544c00005f56000049440000454f000061
:10b574005f520000454300004f52000044000000a9
:10b58400544c00005f56000049440000454f000041
:10b594005f520000454300004f520000445f00002a
:10b5a4005741000049540000005400004c5f000063
:10b5b40056490000444500004f5f0000524500001a
:10b5c400434f0000524400005f530000544f0000fa
:10b5d40050000000544c00005f5600004944000035
:10b5e400454f00005f4c0000414e0000435f0000e7
:10b5f4004f46000046000000544c00005f56000017
:10b6040049440000454f00005f5000004f570000c0
:10b61400455200005f4400004f5700004e000000f8
:10b62400544c00005f56000049440000454f0000a0
:10b634005f520000454100004459000000540000de
:10b644004c5f000056490000444500004f5f000075
:10b65400554e00004b4e00004f5700004e000000b6
:10b66400434100005054000055520000455f000063
:10b674004d4f0000444500005f4f00004646000067
:10b68400205b000020000000544c00005f490000d3
:10b694004d410000474500005f5000004f57000037
:10b6a400455200005f3100005f570000414900002f
:10b6b400540d00000a0000004154000053500000e3
:10b6c4000d000000544c00005f4900004d41000093
:10b6d400474500005f5000004f57000045520000ee
:10b6e4005f3200005f57000041490000540d000024
:10b6f4000a000000544c00005f4900004d41000066
:10b70400474500005f500000484f0000544f0000c0
:10b714005f57000052490000544500000d0a000024
:10b724000031000030320000420d000000540000df
:10b734004c5f0000494d000041470000455f000098
:10b74400504800004f5400004f5f00005741000074
:10b75400495400000d0a0000005400004c5f000032
:10b76400494d000041470000455f00004c41000086
:10b774004e4300005f4f0000464600000d0a0000e3
:10b784000031000030350000450d00000054000079
:10b794004c5f0000494d000041470000455f000038
:10b7a400504f000057450000525f0000444f000016
:10b7b400574e00000d0a0000005400004c5f0000ca
:10b7c400494d000041470000455f0000524500001c
:10b7d40041440000590d00000a000000544c0000d0
:10b7e4005f56000049440000454f00005f500000d0
:10b7f4004f570000455200005f3100005f570000c2
:10b8040041490000540d00000a000000544c00009f
:10b814005f56000049440000454f00005f5000009f
:10b824004f570000455200005f3200005f57000090
:10b8340041490000540d00000a000000544c00006f
:10b844005f56000049440000454f00005f5200006d
:10b85400454300004f520000440d00000a00000060
:10b8640031300000334100000d000000544c000052
:10b874005f56000049440000454f00005f5200003d
:10b88400454300004f520000445f00005741000050
:10b89400495400000d0a000000310000303300005c
:10b8a400330d0000005400004c5f000056490000b6
:10b8b400444500004f5f000052450000434f000024
:10b8c400524400005f530000544f0000500d00002c
:10b8d4000a000000544c00005f5600004944000078
:10b8e400454f00005f4c0000414e0000435f0000e4
:10b8f4004f460000460d00000a000000544c0000b2
:10b904005f56000049440000454f00005f500000ae
:10b914004f570000455200005f4400004f5700009d
:10b924004e0d00000a000000544c00005f56000059
:10b9340049440000454f00005f52000045410000ab
:10b94400445900000d0a00000000000047450000b3
:10b95400540000005345000054000000434c000014
:10b9640045410000527c0000434c0000520000009e
:10b97400544900004d45000000480000454c0000bb
:10b98400507c00003f000000524500005345000079
:10b9940054000000534100005645000000500000d0
:10b9a40041520000414d00000044000045460000a3
:10b9b400415500004c540000004200004154000076
:10b9c40054000000535400004154000000430000a0
:10b9d400414d00002050000057520000004c000070
:10b9e4004544000031200000505700005200000080
:10b9f4004c45000044320000205000005752000023
:10ba040000480000444d0000492000005057000049
:10ba14005200000053540000524f00004245000001
:10ba24002050000057520000004900004e5300000f
:10ba3400542000005057000052000000494e0000fe
:10ba44005354000032200000505700005200000000
:10ba5400484500004c4c00004f2000004b490000ba
:10ba640054540000590000004445000042550000b1
:10ba740047000000455200004153000045200000eb
:10ba84004d4500004d00000057520000495400008d
:10ba9400452000004d4500004d00000052450000c7
:10baa40041440000204d0000454d000000540000ba
:10bab4003100000054320000005400003300000044
:10bac4005434000000000000a8dc00000e600000f8
:10bad400acdc00001e600000b0dc00002e60000042
:10bae400badc00003e600000bfdc000058600000cb
:10baf400c6dc0000fe600000ccdc00000a6100002f
:10bb0400d1dc00003e610000d7dc0000b062000020
:10bb1400dfdc0000da620000e4dc0000f862000010
:10bb2400e9dc000004630000f1dc00002a6300008b
:10bb3400fadc00005063000003dd000076630000bf
:10bb44000cdd00009c63000017dd0000c2630000f0
:10bb540020dd0000e86300002add000070640000be
:10bb640036dd00000e6400003cdd0000806400004f
:10bb740046dd00008c64000050dd00009e6400007f
:10bb840059dd0000086500005cdd00006065000010
:10bb94005fdd0000ae65000062dd0000b8650000f6
:10bba40065dd000000000000494d0000477c0000f6
:10bbb400494d00004147000045000000564900007f
:10bbc400447c000056490000444500004f0000003a
:10bbd4005452000049470000310000005452000054
:10bbe4004947000032000000d6dd0000c2650000b5
:10bbf400e0dd0000f4650000eadd000026660000d8
:10bc0400f0dd00004e66000065dd0000000000006d
:10bc140043410000505400005552000045200000ec
:10bc24004d4f000044450000004400004550000012
:10bc34004c4f000059200000444500004c410000d6
:10bc44005900000044450000504c00004f590000ca
:10bc5400204400005552000041540000494f0000a8
:10bc64004e000000534100004d5000004c450000c0
:10bc7400204900004e540000455200005641000087
:10bc84004c00000056490000444500004f200000cd
:10bc94004455000052410000544900004f4e00003a
:10bca4000042000041540000542000004c450000b4
:10bcb400564500004c000000badc00007466000029
:10bcc4000ade0000e267000017de000016680000cc
:10bcd40024de00002e68000034de00004668000008
:10bce40044de00005e68000053de00007668000059
:10bcf40065dd0000000000005354000055420000c0
:10bd0400000000007ede00008e68000065dd00009b
:10bd140000000000303700003a320000303a0000e2
:10bd240030300000004d000061720000202000004f
:10bd3400382000003230000031320000000d0000d5
:10bd44000a7400006c430000616d0000657200001d
:10bd540061200000436f00006e740000726f0000e9
:10bd64006c6c00006572000020250000732c00003c
:10bd740020250000730d00000a000000244e00007e
:10bd8400616d0000653a0000206d000061720000e2
:10bd94005f3800005f3200003031000032200000c4
:10bda400240000004356000053200000746100008a
:10bdb4006720000022250000732200000d0a000005
:10bdc40000450000525200003a200000434f00009a
:10bdd4004e46000049470000205200004541000043
:10bde4004420000046410000494c00004544000046
:10bdf4002c20000055530000494e0000472000004d
:10be04004445000046410000554c0000540d00001c
:10be14000a00000020090000004500005252000002
:10be24002025000030340000640d00000a000000ea
:10be340052440000590d00000a0000004c4100006b
:10be44004e430000204d00004f44000045200000f8
:10be5400454e0000414200004c450000440d0000e6
:10be64000a0000004c4100004e430000204d000039
:10be74004f440000452000004449000053410000a5
:10be8400424c0000454400000d0a00000000000080
:10be9400537500006e200000004d00006f6e00001e
:10bea40020000000547500006520000000570000c9
:10beb4006564000020000000546800007520000044
:10bec4000046000072690000200000005361000079
:10bed40074200000003f00003f3f000020000000ed
:10bee4004a6100006e200000004600006562000008
:10bef400200000004d61000072200000004100009d
:10bf040070720000200000004d61000079200000e4
:10bf1400004a0000756e0000200000004a75000011
:10bf24006c20000000410000756700002000000044
:10bf34005365000070200000004f0000637400008f
:10bf4400200000004e6f0000762000000044000036
:10bf54006563000020000000256400002025000027
:10bf640030320000643a00002530000032640000e2
:10bf74003a250000303200006420000025640000ef
:10bf840000250000642f0000256400002f25000018
:10bf94006420000025300000326400003a250000cf
:10bfa40030320000643a00002530000032640000a2
:10bfb400000000004552000041530000494e0000bb
:10bfc400472000004e5600004d0000002e000000e7
:10bfd4000d0a0000455200004153000045200000b6
:10bfe400434f00004d5000004c45000054450000f4
:10bff4000d0a0000000000002009000000200000dd
:10c0040000300000313200003334000035360000c7
:08c0140037380000390000007c
:020000040000fa
:100400000000fa0020922000933c0700c0922000d8
:10041000913c0700609320008f3c070056528000fb
:100420006752800086007800c00320000009b800f1
:100430006030b9000302780000024200c0032000cf
:1004400000b8b9000002420084017800c248880068
:10045000d34888000080fa00000006000200fa007d
:10046000000f78009e007800618060000004e000ca
:10047000010032006e3c07001e0078000000d10031
:10048000610060000004e000010032000000000094
:100490001e0078004200de00610060000004e00001
:1004a00001003200d80207000080fa0000000600b8
:1004b0000400fa00889fbe00c16d2d0020002000be
:1004c000df330700c16f2d0020002000dc33070060
:1004d00010528000100798001e009000e20f50009c
:1004e0000b0032001e009000e30f50000c003200a1
:1004f0001e009000e10f5000010032000c00370098
:1005000031712d0020002000cd3307000b00370093
:1005100041722d0020002000c9330700070037007a
:1005200051732d0020002000c53307000300370061
:1005300061742d0020002000c1330700d1742d000c
:1005400020002000be330700c0488000d148800052
:10055000809fbe0000752d00801f78000094200051
:100560006a0a0700e6875700019420002000200057
:10057000b3330700e33c0700809fbe0000772d00e7
:10058000801f780000942000600a0700e68757006b
:100590000194200020002000a933070010528000a1
:1005a000e30f50000e003200c8488000d948800098
:1005b000d43c07000000540081805c00809fbe0096
:1005c00000792d00801f7800009420004f0a07005a
:1005d000e687570001942000200020009833070090
:1005e000017b2d002000200095330700217d2d0088
:1005f000200020009233070000942000160107001d
:1006000001942000200020008d330700d1742d00bc
:10061000200020008a33070020922000223c07009f
:10062000809fbe00907e2d00801f780000942000e7
:10063000360a0700e68757000194200020002000ba
:100640007f33070081802d00200020007c330700cd
:10065000a1822d00200020007933070000942000a3
:10066000550107000194200020002000743307008a
:10067000d1742d002000200071330700c0922000ab
:10068000093c0700809fbe0010842d00801f780069
:10069000009420001d0a0700e687570001942000ff
:1006a000200020006633070001862d002000200076
:1006b0006333070021882d002000200060330700ed
:1006c00040528000000f78001e007800e20f5000ba
:1006d000120032001e007800e20f500004003c00bf
:1006e0001e007800e10f50000800320017003700ac
:1006f0001e007800e30f50000c0032001e0078004e
:10070000e40f50000d00320010003700b1892d00b9
:10071000200020004a3307000f003700918a2d0087
:1007200020002000463307000b003700618b2d00ae
:10073000200020004233070007003700618c2d00a5
:10074000200020003e3307000300370061742d00b5
:10075000200020003a330700d1742d002000200033
:100760003733070060932000cf3b0700809fbe0017
:10077000708d2d00801f780000942000e309070091
:10078000e687570001942000200020002c3307004a
:100790000c000700801f7800808f2d00801f7800dc
:1007a00000942000d9090700e48757000194200035
:1007b00020002000223307004f04be000080fa0012
:1007c000000006000a00fa00881f7800b000200030
:1007d0002e3d0700000478006140b9007f1f07002c
:1007e00030079800410798000800e00007003d002e
:1007f00002002000037824003e009000ce0090000c
:10080000a21f070030079800410798003e009000a3
:10081000ce009000008fbe0092ac2c00f3d22300db
:100820001e00be00f61f0700008fbe0092ac2c0019
:10083000f3d223001e00be00941f0700008fbe00ed
:1008400002002000a34724001e00be00ec1f07008a
:10085000008fbe001e00be001d200700200798006c
:100860002e0090004f0478000080fa00000006007f
:100870000200fa00f0902d00b80307000094200059
:100880003d04070000942000b403070090922d005f
:10089000b2030700580007000000e0000a00320021
:1008a000610007000000e00007003200d0922d0038
:1008b000aa0307001000200020528800100020002a
:1008c000000f7800180037004b0007000000e00020
:1008d00008003a0040952d00a00307000094200076
:1008e0005d000700009420009c030700d0742d00d9
:1008f0009a0307004c0007000000e00008003a00df
:1009000000972d009503070000942000aa0007001f
:100910000094200091030700d0742d008f0307007e
:100920000000eb00000f78001e0078000080fa0045
:10093000000006000200fa00c0982d00870307009f
:10094000009420000c04070000942000830307009b
:1009500090922d0081030700270007000000e000af
:100960000a003200300007000000e00007003200fb
:10097000609a2d0079030700100020003052880093
:1009800010002000000f7800180037001a00070040
:100990000000e00008003a0040952d006f030700ba
:1009a000009420002c000700009420006b03070037
:1009b000d0742d00690307001b0007000000e00051
:1009c00008003a0000972d006403070000942000ff
:1009d000790007000094200060030700d0742d0008
:1009e0005e0307000000eb00000f78001e00780097
:1009f0000080fa00000006000200fa002052800089
:100a0000e80f500003003a0010002000000f7800ab
:100a1000020037000000eb00000f78001e00780095
:100a20000080fa00000006000200fa003052800048
:100a3000e90f500003003a0010002000000f78007a
:100a4000020037000000eb00000f78001e00780065
:100a50000080fa00000006000400fa00000f780091
:100a600020528000100798009e009000e48f5000f4
:100a70002c0032001e009000e40f50000a003c00e1
:100a80009e009000e28f50001a0032001e0090007d
:100a9000e20f50001d003c009e009000e18f5000ce
:100aa0000e0032003d0037001e009000e60f50009f
:100ab000280032009e009000e68f50001f00350095
:100ac0001e009000e70f5000280032009e009000aa
:100ad000e88f50002b003200300037001e007800f5
:100ae000d19c2d000e00090031587800f000b100b3
:100af0002f0037001e007800c19d2d001500090051
:100b0000315878006001b100290037001e007800dc
:100b1000219f2d0015000900315878006001b100b7
:100b2000230037001e00780081a02d00140009006a
:100b3000315878005001b1001d0037001e007800c8
:100b4000d1a12d0013000900315878004001b100f7
:100b5000170037001e00780011a32d0011000900b6
:100b6000315878002001b100110037001e007800d4
:100b700031a42d0013000900315878004001b10064
:100b80000b0037001e00780071a52d000e00090033
:100b900031587800f000b100050037001e007800e1
:100ba00061a62d0010000900315878001001b10035
:100bb0000080fa00000006000400fa00000f780030
:100bc00030528000100798009e009000e58f500082
:100bd000390032001e009000e50f500011003c006b
:100be0009e009000e28f5000210032001e00900015
:100bf000e20f500004003c009e009000e18f500086
:100c0000150032004a0037001e009000e30f50002c
:100c10001d0032009e009000e48f50002000320042
:100c2000430037001e009000e70f50002e003200f6
:100c30009e009000e78f5000250035001e009000b8
:100c4000e80f50002e0032009e009000e98f500007
:100c500031003200360037001e00780071a72d00e9
:100c60000e00090031587800f000b100350037005f
:100c70001e00780061a82d00150009003158780089
:100c80006001b1002f0037001e007800c1a92d00bf
:100c900015000900315878006001b10029003700c3
:100ca0001e00780021ab2d000f000900315878009c
:100cb0000001b100230037001e00780021ac2d0098
:100cc00014000900315878005001b1001d003700b0
:100cd0001e00780071ad2d00140009003158780015
:100ce0005001b100170037001e007800c1ae2d0082
:100cf00011000900315878002001b10011003700bf
:100d00001e007800e1af2d00130009003158780073
:100d10004001b1000b0037001e00780021b12d000a
:100d20000e00090031587800f000b10005003700ce
:100d30001e00780011b22d00100009003158780013
:100d40001001b1000080fa00000006000000fa0067
:100d5000e04880000080fa00000006000400fa006d
:100d6000000f78001e007800e0488800e04880000e
:100d7000100798001e009000e10f5000080032009c
:100d80001e009000e20f5000050032001e0090008f
:100d90000000e000020032000000eb00e0488800a4
:100da0000000eb000080fa00000006000000fa00de
:100db00050528000615280000080fa00000006005e
:100dc0000400fa00008fbe001e00be0050528800d2
:100dd000615288005252800063528000005a200005
:100de00001002000800f5100818f5900040036005f
:100df000005a2000010020005052880061528800f3
:100e00000000eb000080fa00000006000000fa007d
:100e100070528000815280000080fa0000000600bd
:100e20000400fa00008fbe001e00be007052880051
:100e3000815288007252800083528000400020005e
:100e400001002000800f5100818f590004003e00f6
:100e5000500020000100200070528800815288005c
:100e600072528000835280000052200081002000d6
:100e7000800f5100818f590004003600005220007d
:100e80008100200070528800815288000000eb0031
:100e90000080fa00000006000000fa009052800076
:100ea000a15280000080fa00000006000400fa0051
:100eb000008fbe001e00be0090528800a152880024
:100ec00090528000a1528000e00f5000e08f580047
:100ed00004003a0010002000010020009052880019
:100ee000a152880092528000a3528000005a200034
:100ef00001002000800f5100818f5900040036004e
:100f0000005a20000100200090528800a152880061
:100f10000000eb000080fa00000006000000fa006c
:100f2000b0528000c15280000080fa00000006002c
:100f30000400fa00008fbe001e00be00b052880000
:100f4000c1528800b2528000c3528000900020003d
:100f500001002000800f5100818f590004003e00e5
:100f6000a000200001002000b0528800c15288007b
:100f7000b2528000c352800000e120000100200036
:100f8000800f5100818f59000400360000e12000dd
:100f900001002000b0528800c15288000000eb0020
:100fa0000080fa00000006000000fa00f04880000f
:100fb000014980000080fa00000006000400fa00e9
:100fc000008fbe001e00be00f04888000149880066
:100fd000f2488000034980000053270001002000f0
:100fe000800f5100818f5900040036000053270004
:100ff00001002000f0488800014988000000eb0053
:101000000080fa00000006000000fa00889fbe0081
:101010006a000700e40007007f010700105280000b
:10102000e10f50000c003a00363a07000001be0004
:10103000c0488000d1488000800f5100818f590046
:101040004b0039002f3a0700c0488800d14888007b
:10105000200020001052880010528000e20f500043
:101060003f003a00273a07000004be007652800095
:101070008752800086007800c00320000009b80075
:101080006030b9000302780000024200c003200073
:1010900000b8b9000002420084017800820f5400b9
:1010a000838f5c0002003600300020001052880060
:1010b000143a07000001be00c0488000d1488000fb
:1010c000800f5100818f590029003900965280000d
:1010d000a752800086007800c0032000000ab800f4
:1010e0006030b9000501780000014100c003200014
:1010f00000b8b9000001410082027800c0488000b9
:10110000d14880000400400085804800c048880025
:10111000d1488800e0488000e10f500001003a000b
:10112000d3fd0700e0488000e20f500001003a00c4
:1011300000fe0700e04880000000e00008003a00e0
:1011400020b32d0085010700009420000a0207004b
:10115000009420008101070090922d007f0107007c
:1011600010528000e30f500001003a000000000020
:101170004f04be000080fa00000006000000fa00e4
:10118000100020002c31070010002000563107000d
:10119000d1c0b300100020007130070040062000cd
:1011a000b93907001000200023310700100020008b
:1011b0004d3107000080fa00000006000000fa0030
:1011c00020528000e80f500075003200205280004d
:1011d000e10f500009003a00ec02a8002092200024
:1011e0006f390700209220002339070020002000db
:1011f0002052880060b42d00580107002052800062
:10120000e20f500012003a00209220002639070019
:101210000001be00f070220001002000800f51008c
:10122000818f59005e003600d4ff0700e1b52d0024
:101230001000200082300700209220000e390700a5
:10124000300020002052880040b62d0043010700e6
:1012500020528000e30f50000c003a002092200042
:10126000113907000001be00f070220001002000cb
:10127000800f5100818f5900490036004000200046
:1012800020528800c0b72d00340107002052800092
:10129000e40f50000e003a00cd82a80000000000cc
:1012a000cda2a80000000000b4ff070031b92d0056
:1012b000100020006230070020922000ee38070066
:1012c000500020002052880090b92d002301070013
:1012d00020528000e50f500010003a0020922000bc
:1012e000f13807000001be0070a9230001002000b2
:1012f000800f5100818f590029003600cd82a9004e
:1013000000000000cda2a900000000006000200045
:1013100020528800f0ba2d001001070020528000f2
:10132000e60f50000a003a0094ff070031bc2d0080
:10133000100020004230070020922000ce38070025
:10134000700020002052880090bc2d00030107008f
:1013500020528000e70f500011003a002092200038
:10136000d13807000001be00f0702200010020000b
:10137000800f5100818f590009003600ec02a9004e
:101380008000200020528800209220001a39070097
:1013900020922000b8380700f0bd2d00ef000700b4
:1013a0000080fa00000006000000fa00889fbe00de
:1013b00030528000e90f500094003200305280001b
:1013c000e10f500009003a00ec02a800c092200092
:1013d000f3380700c0922000a73807002000200043
:1013e0003052880000bf2d00dc0007003052800022
:1013f000e20f500012003a00c0922000aa38070005
:101400000001be00f070220001002000800f51009a
:10141000818f59007d00360058ff0700e1b52d008f
:101420001000200006300700c0922000923807000c
:10143000300020003052880080c02d00c700070017
:1014400030528000e30f50000c003a00c0922000a0
:10145000953807000001be00f07022000100200056
:10146000800f5100818f5900680036004000200035
:101470003052880000c22d00b800070030528000b2
:10148000e40f50000e003a00cd82a80000000000da
:10149000cda2a8000000000038ff070021c32d00e6
:1014a00010002000e62f0700c092200072380700cd
:1014b000500020003052880080c32d00a700070094
:1014c00030528000e50f500020003a00c09220000a
:1014d000753807000004be00b6528000c752800075
:1014e00086007800803e20000009b8006030b90016
:1014f0000302780000024200803e200000b8b900dc
:101500000002420084017800820f5400838f5c0047
:101510003e003900cd82a90000000000cda2a90044
:101520000000000015ff0700f1c42d00100020008e
:10153000c32f0700c09220004f3807006000200032
:101540003052880050c52d008400070030528000c2
:10155000e60f50000c003a00c092200052380700fd
:101560000001be00f070220001002000800f510039
:10157000818f59002500360070002000305288000d
:10158000c0c62d007500070030528000e70f5000e4
:101590000a003a00f9fe070031bc2d0010002000bf
:1015a000a72f0700c09220003338070080002000da
:1015b0003052880000c82d006800070030528000bb
:1015c000e80f500011003a00c092200036380700a2
:1015d0000001be00f070220001002000800f5100c9
:1015e000818f590009003600ec02a900900020000c
:1015f00030528800c09220007f380700c09220003f
:101600001d38070060c92d00540007004f04be00bc
:101610000080fa00000006000400fa006000b80034
:10162000008fbe00f048800001498000e00f5000ac
:10163000e08f58004700320040528000e40f500015
:10164000440032005ffc070001002000008fbe0054
:1016500040528000e10f500012003a00f048800034
:1016600001498000be0f1000ae8f18000700310046
:101670002000200040528800609320004838070076
:1016800060932000fc370700060037003000200080
:101690004052880060932000573807006093200074
:1016a000f537070040528000e20f500016003a0064
:1016b000f048800001498000be0f1000ae8f180076
:1016c0000f00310060932000f73707000001be00d3
:1016d0000053270001002000800f5100818f590026
:1016e00009003600609320004338070030002000d6
:1016f000105288004000200040528800020037004d
:10170000300020004052880040528000e30f50001b
:1017100010003a00f048800001498000be0f100020
:10172000ae8f1800070031002000200040528800d2
:10173000609320001a38070060932000ce3707001e
:1017400004003700609320002b38070060932000ce
:10175000c93707000080fa00000006000200fa0006
:10176000000f7800d05280000000e000030032003b
:101770009e00780020002000312f07000080fa0032
:04178000000006005f
:020000040000fa
:10c01c000200fa00000f78005200200061df2d00b2
:10c02c001e0078003c0d07000080fa00000006009e
:10c03c000200fa00000f780052002000e1e52d000c
:10c04c001e007800340d07000080fa000000060086
:10c05c000200fa00000f78005200200041e82d0089
:10c06c001e0078002c0d07000080fa00000006006e
:10c07c000200fa00000f7800009820003bd6070061
:10c08c000198200020002000ea04070021e12c0088
:10c09c0020002000e70407000000eb000080fa00fd
:10c0ac00000006000200fa00000f780051e12c009d
:10c0bc0020002000df04070001e32c0020002000fa
:10c0cc00dc04070071e52c0020002000d9040700d7
:10c0dc0061e72c0020002000d6040700f1e92c00b9
:10c0ec0020002000d304070071ec2c00200020005d
:10c0fc00d004070091ef2c0020002000cd04070095
:10c10c00e1f12c0020002000ca040700c1f42c002f
:10c11c0020002000c704070041f72c00200020005d
:10c12c00c404070021fa2c0020002000c1040700e1
:10c13c0001fd2c0020002000be04070091002d0002
:10c14c0020002000bb04070041032d00200020002c
:10c15c00b804070011062d0020002000b5040700cc
:10c16c0021092d0020002000b2040700d10b2d0066
:10c17c0020002000af040700810e2d0020002000bd
:10c18c00ac04070031112d0020002000a904070089
:10c19c00e1132d0020002000a604070021172d001c
:10c1ac0020002000a3040700611a2d0020002000ad
:10c1bc00a0040700b11d2d00200020009d040700e5
:10c1cc0061212d00200020009a040700d1242d00ad
:10c1dc00200020009704070021282d0020002000bb
:10c1ec00940407000000eb000080fa000000060039
:10c1fc000200fa00000f78000000fe000000eb00c7
:10c20c000080fa00000006000200fa00000f78001f
:10c21c000000eb00004e8800c9d20700104e8800c9
:10c22c00dfd20700204e8800314e8800f4d2070080
:10c23c00404e8800514e880014d30700604e880091
:10c24c00714e880032d30700804e8800914e8800d2
:10c25c0052d30700a04e8800b14e8800009c2000ed
:10c26c004a0907000000eb000080fa0000000600fd
:10c27c000c00fa0050079800b1d207004007980054
:10c28c004e0090000000e00003003a00702b2d00df
:10c29c001007980002003700e02b2d0010079800c3
:10c2ac004e0090000000e00003003a00502c2d00de
:10c2bc00000f78000e0037004e009000e10f500088
:10c2cc0003003a00902c2d00000f78000800370076
:10c2dc004e009000e20f500003003a00d02c2d00cd
:10c2ec00000f780002003700102d2d00000f780091
:10c2fc001e007800801f78009e009000811f78003f
:10c30c00502d2d00801f780000982000fcda0700cb
:10c31c00e687570001982000200020004504070004
:10c32c009fd2070020079800310798002e0190003b
:10c33c00be019000e001200001002000800f5100a0
:10c34c00818f590003003a00702b2d0010079800c4
:10c35c0002003700e02b2d00100798002e009000f3
:10c36c00be009000809fbe009e009000811f780050
:10c37c00f02e2d00801f780000982000e0da0700d6
:10c38c00e8875700019820002000200029040700ae
:10c39c009bd2070020079800310798002e019000cf
:10c3ac00be019000c003200001002000800f51004e
:10c3bc00818f590003003a00702b2d001007980054
:10c3cc0002003700e02b2d00100798002e00900083
:10c3dc00be009000809fbe009e009000811f7800e0
:10c3ec00e0302d00801f780000982000c4da070090
:10c3fc00e887570001982000200020000d0407005a
:10c40c00a2d2070020079800310798002e01900057
:10c41c00be019000c003200001002000800f5100dd
:10c42c00818f590003003a00702b2d0010079800e3
:10c43c0002003700e02b2d00100798002e00900012
:10c44c00be009000809fbe009e009000811f78006f
:10c45c00d0322d00801f780000982000a8da070049
:10c46c00e88757000198200020002000f103070006
:10c47c00a7d2070020079800310798002e019000e2
:10c48c00be019000c003200001002000800f51006d
:10c49c00818f590003003a00702b2d001007980073
:10c4ac0002003700e02b2d00100798002e009000a2
:10c4bc00be009000809fbe009e009000811f7800ff
:10c4cc00c0342d00801f7800009820008cda070003
:10c4dc00e88757000198200020002000d5030700b2
:10c4ec00aed2070020079800310798002e0090006c
:10c4fc00be009000e00f5000e08f580003003a009f
:10c50c00702b2d001007980002003700e02b2d0037
:10c51c00100798002e009000be009000809fbe0077
:10c52c009e009000811f7800b0362d00801f78008f
:10c53c000098200072da0700e88757000198200065
:10c54c0020002000bb0307000000eb000080fa0075
:10c55c00000006000200fa00000f78000000eb005b
:10c56c00fbd10700e00120000100200011d20700e0
:10c57c00c00320000100200026d20700c0032000c9
:10c58c000100200046d20700c0032000010020005b
:10c59c0064d207006000b80085d207000000eb00f1
:10c5ac000080fa00000006000200fa00000f78007c
:10c5bc0081d00700801f780090382d00801f7800f4
:10c5cc00009820004eda0700e487570001982000fd
:10c5dc0020002000970307000000eb000080fa0009
:10c5ec00000006000200fa00000f7800adcf070033
:10c5fc000000eb000080fa00000006000200fa00c8
:10c60c00000f7800013a2d001e007800160b070071
:10c61c000000e00005003200313a2d00200020001f
:10c62c0084030700ec02a80004003700013b2d0036
:10c63c00200020007f030700ec02a9000000eb00a3
:10c64c000080fa00000006000200fa00000f7800db
:10c65c00013a2d001e007800030b07000000e000db
:10c66c0005003200e13b2d00200020007103070083
:10c67c00cd82a80004003700c13c2d002000200012
:10c68c006c030700cd82a9000000eb000080fa00cb
:10c69c00000006000200fa00000f7800013a2d009d
:10c6ac001e007800f00a07000000e00005003200d0
:10c6bc00b13d2d00200020005e030700cda2a80094
:10c6cc0004003700913e2d00200020005903070084
:10c6dc00cda2a9000000eb000080fa0000000600cb
:10c6ec000200fa00000f7800013a2d001e007800bd
:10c6fc00dd0a07000000e00005003200813f2d003c
:10c70c00200020004b030700ec22a8000400370097
:10c71c0061402d002000200046030700ec22a900f8
:10c72c000000eb000080fa00000006000200fa0096
:10c73c00000f7800013a2d001e007800ca0a07008d
:10c74c000000e0000500320051412d0020002000c7
:10c75c0038030700d5a2a8000400370051422d0071
:10c76c002000200033030700d5a2a9000000eb0035
:10c77c000080fa00000006000200fa00000f7800aa
:10c78c00013a2d001e007800b70a07000000e000f7
:10c79c000500320061432d00200020002503070016
:10c7ac00d5c2a8000400370041442d002000200011
:10c7bc0020030700d5c2a9000000eb000080fa009e
:10c7cc00000006000200fa00000f7800013a2d006c
:10c7dc001e007800a40a07000000e00005003200eb
:10c7ec0031452d002000200012030700cdc2a80007
:10c7fc000400370021462d00200020000d03070007
:10c80c00cdc2a9000000eb000080fa000000060079
:10c81c000400fa00000f7800013a2d001e00780089
:10c82c00910a07000000e000080032001000200010
:10c83c00d052880021472d0020002000fd02070067
:10c84c000000eb00100798001f003700512c2d0042
:10c85c001e007800840a07000000e0000800320087
:10c86c000000eb00d052880051482d002000200021
:10c87c00f00207000000eb001007980012003700d0
:10c88c0091492d0020002000ea020700d0528000c0
:10c89c000000e00004003200013a2d0020002000ce
:10c8ac00e402070003003700512c2d00200020006b
:10c8bc00e002070021e12c0020002000dd0207002f
:10c8cc000000eb00100798001e0090000080fa009a
:10c8dc00000006000200fa00000f7800814a2d00cb
:10c8ec0020002000d30207000000eb000080fa00bb
:10c8fc00000006000200fa00000f78008009070013
:10c90c000000eb000080fa00000006000200fa00b4
:10c91c00000f78001e007800040a070020e12c00ac
:10c92c00020a07000000eb000080fa00000006007d
:10c93c000a00fa00400798000000eb00200798005e
:10c94c006000b800008fbe002500370003012000f6
:10c95c00029820001e00be008a090700000120007a
:10c96c00010020001e0f40005e9748000000eb0005
:10c97c003007980017003700be0090000098200088
:10c98c0000804000104078000004e00005003d00ed
:10c99c0010002000200798000001200030079800ac
:10c9ac000c003700be009000009820000080400072
:10c9bc0010407800804078002000200065020700bd
:10c9cc000000e000030032003e0090000000e80090
:10c9dc00300798003e009000ef0f5000e6ff340047
:10c9ec002e0090000000e000d8ff320021e12c0066
:10c9fc00200020008f0207000000eb000080fa00ee
:10ca0c00000006001000fa00700798006a0047004a
:10ca1c0018d807006a00470080d807002007980044
:10ca2c00ae0090000000eb0080087800ae00900093
:10ca3c000000eb0090009800ae0090000000eb00ae
:10ca4c00a00098002e009000300090008000e800bc
:10ca5c002e009000310098002e00900079d807002d
:10ca6c0030079800410798005e009000ee0090009f
:10ca7c003e019000ce0190000ad90700008fbe0045
:10ca8c001e00be00809fbe00f04a2d00801f780063
:10ca9c00009820001ad90700e6875700019820005b
:10caac0020002000630207000000eb000080fa0069
:10cabc00000006000a00fa004007980066004700d4
:10cacc00801f780064004700801f78000e80e8000b
:10cadc00801f7800604d2d00801f78004e00900064
:10caec0024d90700e88757003e0090000001780029
:10cafc002e009000800078001e0090006dd407007e
:10cb0c00000f78003e009000ae0090001e019000d7
:10cb1c009e017800831f7800801f7800811f7800a9
:10cb2c00821f7800f04d2d00801f780000982000a7
:10cb3c00f3d80700ea875700019820002000200056
:10cb4c003c0207000000eb000080fa000000060029
:10cb5c000200fa00000f78000000eb000080fa00e1
:10cb6c00000006000200fa00000f78000000eb0045
:10cb7c000080fa00000006000400fa00000f7800a4
:10cb8c0038cf07000000e000030032000000eb008b
:10cb9c00100798000e00370094cf07000000e0004b
:10cbac0003003a00e14f2d00200020002102070075
:10cbbc009acf07000000e00003003a0081512d00dd
:10cbcc00200020001b0207000000eb00100798005b
:10cbdc001e0090000080fa00000006000400fa001d
:10cbec00000f780050cf07000000e0000300320077
:10cbfc000000eb00100798000e0037007bcf0700f9
:10cc0c000000e00003003a00e14f2d00200020005e
:10cc1c000802070081cf07000000e00003003a0083
:10cc2c0081512d0020002000020207000000eb00c3
:10cc3c00100798001e0090000080fa00000006000b
:10cc4c000200fa00000f780021532d002000200074
:10cc5c00f8010700dac2bf0001c8b3000140600050
:10cc6c000004e00004003200e1532d0020002000fd
:10cc7c00f00107000300370031542d002000200084
:10cc8c00ec0107000000eb000080fa000000060039
:10cc9c000200fa00000f780091542d0020002000b3
:10ccac00e4010700dac2bf000044b2000004e00057
:10ccbc0004003200e1532d0020002000dd010700ac
:10cccc000300370031542d0020002000d90107004b
:10ccdc000000eb000080fa00000006001400fa00cf
:10ccec00000f98008e80e8000000eb0080087800b0
:10ccfc008e80e8000000eb00900098008e80e80029
:10cd0c000000eb00a00098008e80e8000000eb0013
:10cd1c00b00098008e80e8000000eb00c000980086
:10cd2c008e80e8000000eb00d00098008e80e800b8
:10cd3c000000eb00e00098000e80e8006600400068
:10cd4c00801f78000e80e800801f78000e80e800bd
:10cd5c000080e800801f78000e80e800640040002e
:10cd6c00801f78000e80e8006c004000801f780067
:10cd7c000e80e80068004000801f78000e80e800fc
:10cd8c006a004000801f780050552d00801f7800ed
:10cd9c000e08900077d80700f0875700000f780036
:10cdac00600020009e0f10000c003c00a1562d00ce
:10cdbc00200020009f010700c1572d0020002000fb
:10cdcc009c010700b1592d0020002000990107009b
:10cddc000000eb00100f9800740037000e80e80084
:10cdec00500090000000e000040034000e80e800c9
:10cdfc0050009000ec0f500006003400115c2d0028
:10ce0c00200020008b0107000000eb00100f9800a1
:10ce1c00660037000e80e800400090000000e00043
:10ce2c00040034000e80e80040009000ff0f50001a
:10ce3c0006003400415e2d00200020007d0107001b
:10ce4c000000eb00100f9800580037000e80e8002f
:10ce5c0060009000ea0f5000050034000e80e800de
:10ce6c00e000900030062000808f50000600340057
:10ce7c0051602d00200020006e0107000000eb0027
:10ce8c00100f9800490037000e80e8002000900039
:10ce9c000000e000040035000e80e8002000900047
:10ceac00f70f50000600340091622d002000200086
:10cebc00600107000000eb00100f98003b003700ea
:10cecc000e80e800100090000000e0000500350026
:10cedc000e80e80090009000b0032000808f50007e
:10ceec0006003400d1642d00200020005101070001
:10cefc000000eb00100f98002c0037000e80e800ab
:10cf0c00100078000000e000050035000e80e800fd
:10cf1c0090007800b0032000808f50000600340091
:10cf2c0031672d0020002000420107000000eb00bb
:10cf3c00100f98001d0037000e80e80030009000a4
:10cf4c000000e000040034000e80e8003000900087
:10cf5c00e70f50000600340091692d0020002000de
:10cf6c00340107000000eb00100f98000f00370091
:10cf7c000e80e8000bd20700009820007bd207003f
:10cf8c00a16b2d00200020002a0107000198200031
:10cf9c00200020002701070021e12c0020002000a8
:10cfac00240107000000eb00100f98001e089000f1
:10cfbc000080fa00000006000200fa00000f780062
:10cfcc00512c2d001e007800a70807000000e0007f
:10cfdc00020032000000eb005dcf0700912c2d0009
:10cfec001e007800a00807000000e00002003200dc
:10cffc001000200056cf0700d12c2d001e00780009
:10d00c00990807000000e000020032002000200018
:10d01c004fcf07000000eb000080fa000000060074
:10d02c000600fa0020079800a20020008000eb0008
:10d03c002e009000d8d70700008fbe001e00be0047
:10d04c005ccf07000000eb000080fa000000060037
:10d05c000600fa0020079800a20020008000eb00d8
:10d06c002e009000ccd70700008fbe001e00be0023
:10d07c0068cf07000000eb000080fa0000000600fb
:10d08c000600fa0020079800a20020008000eb00a8
:10d09c002e009000c0d70700008fbe001e00be00ff
:10d0ac007fcf07000000eb000080fa0000000600b4
:10d0bc000600fa0020079800a20020008000eb0078
:10d0cc002e009000b4d70700008fbe001e00be00db
:10d0dc0094cf07000000eb000080fa00000006006f
:10d0ec000600fa0020079800a20020008000eb0048
:10d0fc002e009000a8d70700008fbe001e00be00b7
:10d10c00abcf07000000eb000080fa000000060027
:10d11c000200fa00000f78001e007800801f7800d3
:10d12c00806c2d00801f78000098200074d70700b9
:10d13c00e48757000198200020002000bd00070064
:0cd14c000000eb000080fa00000006006c
:020000040000fa
:101784000000fa001000200025390700e0082000be
:101794000e3907000000eb000c3907000000eb00d5
:1017a4001f3907000080fa00000006000400fa0058
:1017b40010079800100020001939070000082000c5
:1017c400023907001e00900010007800e5010700b0
:1017d400004f78001e80fb00fc3807001e009000bc
:1017e40010009000df010700004f78001e80fb000e
:1017f400f63807001e00900020009000d901070071
:10180400004f78001e80fb00f03807001e00900097
:1018140030009000ed3807001e009000400090005a
:10182400d0010700004f78001e80fb00e738070056
:101834001e00900050009000ca010700004f78007d
:101844001e80fb00e13807001e009000600090003d
:10185400c4010700004f78001e80fb00db3807003e
:101864000000eb00ee3807000000eb000080fa00f7
:10187400000006000400fa00100798001000200081
:10188400e73807000000eb00d038070050052000bf
:10189400ce380700004f78001e407800c4010700ce
:1018a4008080fb001e009000010878005005200095
:1018b400c6380700004f78001e407800bc010700be
:1018c4008080fb001e00900011009800500520004d
:1018d400be380700004f78001e407800b4010700ae
:1018e4008080fb001e00900021009800500520001d
:1018f400b6380700800078001e0090003100980080
:1019040050052000b1380700004f78001e407800d1
:10191400a70107008080fb001e0090004100980092
:1019240050052000a9380700004f78001e407800b9
:101934009f0107008080fb001e009000510098006a
:1019440050052000a1380700004f78001e407800a1
:10195400970107008080fb001e0090006100980042
:101964000000eb00ae3807000000eb000080fa0036
:10197400000006005600fa00702798000e00780058
:10198400bcff07003e009000002f98008e289000b6
:10199400e48f5000290032000e299000e40f51001a
:1019a4000a003c008e299000e28f5100170032009b
:1019b4000e289000e20f50001a003c008e28900080
:1019c400e18f50000b003200340037000e299000e4
:1019d400e60f5100250032008e299000e68f510059
:1019e4001c0035000e289000e70f5000250032003f
:1019f4002a0037007e209000a1f42d000400090085
:101a0400315878005000b100290037007e20900042
:101a1400f2f42d0004000900325878005000b1009f
:101a2400230037007e20900043f52d0004000900b8
:101a3400335878005000b1001d0037007e2090001c
:101a440091f52d0004000900315878005000b100d0
:101a5400170037007e209000e2f52d0004000900f5
:101a6400325878005000b100110037007e209000f9
:101a740033f62d0004000900335878005000b100fb
:101a84000b0037007e20900081f62d000400090031
:101a9400315878005000b100050037007e209000d6
:101aa400d2f62d0004000900325878005000b1002d
:101ab4005e0090006101b9000080eb008080eb00c3
:101ac4000201400083814800122f9800232f9800c0
:101ad400b0002000010020001e299000ae299000d3
:101ae400800f5100818f59003f003e001e28900056
:101af400ae289000006001000b0037000e00370094
:101b04001100370014003700170037001a0037009f
:101b14001d0037002000370023003700260037005f
:101b2400290037002c00370021f72d007e2090007b
:101b3400af0507002f00370071f72d007e209000bd
:101b4400ab0507002b003700c1f72d007e20900065
:101b5400a70507002700370011f82d007e2090000c
:101b6400a30507002300370061f82d007e209000b4
:101b74009f0507001f003700b1f82d007e2090005c
:101b84009b0507001b00370001f92d007e20900003
:101b9400970507001700370051f92d007e209000ab
:101ba4009305070013003700a1f92d007e20900053
:101bb4008f0507000f003700f1f92d007e209000fb
:101bc4008b0507000b00370041fa2d007e209000a2
:101bd400870507000700370091fa2d007e2090004a
:101be4008305070003003700d1f62d007e20900006
:101bf4007f050700ee009000007d2000008040007b
:101c04009e0078001e019000ae0190004e029000ec
:101c1400ee024700801f7800811f7800821f780041
:101c2400831f7800841f7800e0fa2d00801f78005d
:101c340005007800b4040700ec875700ee00470065
:101c44007e2090006a0507000000eb000080fa0087
:101c5400000006001000fa00700798000e007800db
:101c640004ff07001e0178009e0190002e029000e0
:101c7400ee009000007d200000804000ce00900027
:101c8400de029000821f7800831f7800841f780092
:101c9400801f7800811f7800851f780030fc2d009c
:101ca400801f78007e00900097040700ee8757009d
:101cb4000000eb000080fa00000006000e00fa00ad
:101cc4001007980021079800320798001e00900022
:101cd4000000e000030032001e009000ff0f5000df
:101ce400030036000080eb004007980063003700d3
:101cf4002e0090000000e000030032002e0090004f
:101d0400ec0f5000030036008080eb004107980080
:101d14005a003700be009000f07c2000808f5000f5
:101d240004003600be00900030832000808f5000f5
:101d3400030036000081eb00420798004f00370093
:101d44002e0090006101b8000080eb008080eb0061
:101d540002014000838148005207980063079800fd
:101d6400b0002000010020005e019000ee01900010
:101d7400800f5100818f590032003e005e009000b8
:101d8400ee009000006001000b0037000d003700ea
:101d94000f0037001100370013003700150037001b
:101da40017003700190037001b0037001d003700eb
:101db4001f003700210037000000eb00000f7800ff
:101dc40020003700f0012000000f78001d003700cc
:101dd400b0032000000f78001a003700a00520008f
:101de400000f78001700370080072000000f7800ec
:101df4001400370070092000000f7800110037002c
:101e0400500b2000000f78000e003700400d20001a
:101e1400000f78000b003700300f2000000f78000f
:101e24000800370010112000000f7800050037006b
:101e340000132000000f780002003700e014200097
:101e4400000f78009e0078001e0090000080400083
:101e5400000f78003e009000630060000000e00086
:101e640004003a002e009000e20f500001003600fa
:101e74001e0fe8009e007800410798004e00900075
:101e84000080fa00000006000c00fa001007980019
:101e940021079800320798000000eb00000f78003b
:101ea4001e0090000000e000030032001e009000bd
:101eb400ff0f5000050036000080eb008080eb002f
:101ec40040079800510798001c0037002e0090002e
:101ed4000000e000030032002e009000ec0f5000e0
:101ee400050036000081eb008081eb00420798007a
:101ef4005307980011003700be009000f07c2000ca
:101f0400808f500004003600be0090003083200013
:101f1400808f5000050036000080eb008080eb00cd
:101f24004007980051079800040037001e0078000d
:101f34006101b90042079800530798004e009000d1
:101f4400de0090000080fa00000006000600fa009f
:101f5400008fbe00220798000000eb000080fa000a
:101f6400000006000400fa00204798002e4090006c
:101f74000080fb00a2002000110009000280d800ac
:101f84004400dd00004f78002e4090000080fb00ec
:101f9400a2002000110009000280d8008000fd008a
:101fa4001e4f40001e80fb000080fa000000060067
:101fb4000400fa00204798002e4090006f4f600004
:101fc4002e4090008080fb00000f20000080600005
:101fd4004480de006a00b900804078001e4078002a
:101fe40000c04000004f78001e80fb000080fa0013
:041ff40000000600e3
:020000040000fa
:10d158000200fa000000eb00000f780027003700fb
:10d168009e0178001e0078004700dd0080007800ee
:10d17800408120000080400000017800c318dd00d5
:10d188004080200000804000020878001e007800df
:10d198004300dd008080e80040802000808040005f
:10d1a8000000eb00800878001e0078004300dd00d6
:10d1b800e400400040802000808040000000eb0038
:10d1c800800878001e0078004300dd00e60040007b
:10d1d8004080200080804000f00720008008780010
:10d1e8001e007800800040004091200080804000b0
:10d1f8000000eb00800878001e0fe80010002000f7
:10d208009e0f1000d6ff3400b000200040118800a7
:10d2180021e2a80020a2a9002062a9000040200065
:10d228001011880023c2a8008560a9008580a90084
:10d23800910a200091407800f0c8b30000c0600057
:10d2480001c6b30001407000a9e0b700a10a2000a0
:10d258009140780080cfb30000c060000014a000a7
:10d26800aae0b7009560a8009580a900b00020004a
:10d27800c011880031e2a80030a2a9003062a900dc
:10d28800004020009011880087c0a90087e0a9000d
:10d29800310b20009140780080cfb30000c06000bf
:10d2a8006040b300b3e0b700310b20009140780034
:10d2b800f0c8b30000c0600001c2b30001407000b4
:10d2c800b3e0b70097c0a80097e0a9000080fa0073
:10d2d800000006000a00fa001007980021079800cd
:10d2e8001e009000400798004e009000e10f50008b
:10d2f800090032004e009000e20f50000600320094
:10d30800ae0090000040eb00804878000000eb0081
:10d31800300798000d003700810a07001e009000b2
:10d328004300dd0080007800408020006800500045
:10d33800808040002e009000ae090700000f7800a2
:10d34800810a07001e007800300798003e00900010
:10d358000080fa00000006000c00fa001007980090
:10d36800414798001e009000400798004e0090002a
:10d37800e10f5000040032004e009000e20f500010
:10d38800080032000e00370023c2bf000080fb00f7
:10d398000000d100614060000080fb00000f7800b1
:10d3a8000900370033c2bf000080fb000000d10035
:10d3b800614060000080fb00000f78000200370029
:10d3c80010002000000f78001e00e00015003a0051
:10d3d8001e009000500798005e009000e10f50007a
:10d3e800040032005e009000e20f50000700320097
:10d3f8000c0037004e4090000080fb002011880090
:10d408001000200030079800080037004e409000b8
:10d418000080fb00a0118800100020003007980051
:10d42800020037000000eb00300798003e00900033
:10d438000080fa00000006000600fa0010079800b5
:10d44800210798000000eb00000f78000b00370060
:10d458001e007800800078002e00900000804000b8
:10d4680010407800804078001e009000baff070046
:10d478000000e000010032001e0fe8001e007800e6
:10d48800800078002e009000008040001040780056
:10d498000004e000eeff3a000000eb000080fa0014
:10d4a800000006000800fa00100798001e0090000f
:10d4b800300798003e009000e10f5000060032004f
:10d4c8003e009000e20f5000030032000000eb0025
:10d4d800200798000c003700110a07001e00900072
:10d4e8004300dd0080007800408020006800500084
:10d4f800008040006b090700000f7800120a07003f
:10d508001e007800200798002e0090000080fa0086
:10d51800000006000600fa00100798001e009000a0
:10d52800200798002e009000e10f50000400320000
:10d538002e009000e20f5000080032000e00370065
:10d5480023c2bf000080fb000000d10061406000e2
:10d558000080fb00000f78000900370033c2bf00cd
:10d568000080fb000000d100614060000080fb00eb
:10d57800000f78000200370010002000000f78002c
:10d588001e0078000080fa00000006000600fa007d
:10d59800000f78001e007800200798002e009000e9
:10d5a800e10f5000060032002e009000e20f5000fc
:10d5b800030032000000eb00100798000600370057
:10d5c8001e00e900800040004091200000804000db
:10d5d80010007800100798001e0090000080fa00e4
:10d5e800000006000400fa00000f78001e00780012
:10d5f800100798001e009000e10f50000400320050
:10d608001e009000e20f50000100320006003700b3
:10d618001e00e9008000400040912000808040000a
:10d628000000eb00800878000080fa000000060087
:10d638000800fa00100798001e00900020079800c4
:10d648002e009000e10f5000040032002e009000e0
:10d65800e20f5000010032001f003700b009070038
:10d668001e0090004300dd0080007800408020000c
:10d678006800500000804000000907001e0090006c
:10d68800300798003e009000e10f5000060032007d
:10d698003e009000e20f50000a0032000d003700f3
:10d6a80030118000000f780022c2bf006140600086
:10d6b8000004e000faff3a0006003700b0118000cd
:10d6c800000f780032c2bf00614060000004e00033
:10d6d800faff3a009c0907000080fa0000000600e3
:10d6e8000400fa00000f78001e0078001007980068
:10d6f8001e009000e10f5000040032001e00900050
:10d70800e20f500006003200090037002342a9004a
:10d71800000000002342a8000000000004003700b9
:10d728003342a900000000003342a80000000000b6
:10d738000080fa0000000600809fbe000000fa008a
:10d74800004080001140800061004000e0804800f7
:10d7580000408800114088008580a9000080fa00f8
:10d768004f00be0000400600809fbe000000fa0087
:10d7780016003700304080008000e80050408000ec
:10d788008080600040408000808f500005003a0093
:10d7980030118000a048880010002000a0488800b0
:10d7a8000a0037002140800030408000808040001f
:10d7b8003011800080487800304080008000e80008
:10d7c80050408000008060003040880022c2bf00c6
:10d7d800614060000004e000e6ff3a008560a900af
:10d7e8000080fa004f00be0000400600809fbe0087
:10d7f8000000fa00004080001140800061004000f5
:10d80800e0804800004088001140880087e0a900b7
:10d818000080fa004f00be0000400600809fbe0056
:10d828000000fa0016003700704080008000e80011
:10d83800904080008080600080408000808f500091
:10d8480005003a00b0118000b048880010002000a0
:10d85800b04888000a0037006140800070408000ae
:10d8680080804000b01180008048780070408000bf
:10d878008000e800904080000080600070408800d0
:10d8880032c2bf00614060000004e000e6ff3a00d9
:10d8980087c0a9000080fa004f00be0000400600c3
:020000040000fa
:10d8a800d80900005000000002000000000000003d
:10d8b8000000000000000000000000000000000060
:10d8c8000000000000000000000000000000000050
:10d8d8000000000000000000000000000000000040
:10d8e8000000000000000000000000000000000030
:10d8f8000000000000000000000000000000000020
:10d90800000000000000000000000000000000000f
:10d918000000000000000000280a00001a000000b3
:10d9280000000000000800001801000000000000ce
:10d93800660a0000020000000000000080090000e4
:10d948005800000000000000620a00000400000007
:10d95800000000005c0a0000060000000000000053
:10d96800180900006800000000000000420a0000da
:10d978001a00000002000000010008000009000071
:10d9880001001e00000000003c000000003c0000f8
:10d9980000003c000000000000000000f20d000044
:10d9a8000a00000000000000d40b00004a0000003c
:10d9b800020000000000210015110e000d0c0b00e4
:10d9c8000b0a0a00090909000909080008080800e3
:10d9d80008080800070707000707070007070700e8
:10d9e8000707070007303100323334003536370077
:10d9f80038396100626364006566670068696a00b7
:10da08006b6c6d006e6f70007172730074757600c8
:10da1800777879007a000000680a00006c0100003d
:10da2800020000000000a3000b4d0b004d0b4d0041
:10da38000bc60a00c60ac6000a980a00980a980087
:10da48000a980a00980a98000a980a00980a980002
:10da58000a980a00970a96000a950a00940a000094
:10da6800000000007c25610020256200202565005b
:10da780020255400202559007c256d002f256400a1
:10da88002f2579007c2548003a254d003a2553007a
:10da98007c2549003a254d003a2553002025700081
:10daa800003a4a00616e3a004a616e007561720080
:10dab800793a460065623a0046656200727561000f
:10dac80072793a004d6172003a4d610072636800e4
:10dad8003a417000723a4100707269006c3a4d0028
:10dae80061793a004d6179003a4a75006e3a4a0008
:10daf800756e65003a4a75006c3a4a00756c790093
:10db08003a417500673a41007567750073743a00c9
:10db1800536570003a536500707465006d62650066
:10db2800723a4f0063743a004f6374006f62650085
:10db3800723a4e006f763a004e6f7600656d62005d
:10db480065723a00446563003a44650063656d0098
:10db580062657200003a5300756e3a0053756e00a4
:10db6800646179003a4d6f006e3a4d006f6e640043
:10db780061793a00547565003a547500657364001c
:10db880061793a00576564003a576500646e65002c
:10db980073646100793a540068753a0054687500f6
:10dba8007273640061793a00467269003a467200fd
:10dbb80069646100793a530061743a0053617400f2
:10dbc80075726400617900003a414d003a504d0089
:10dbd80000a30b004d0b4d000b4d0b00c60ac600f1
:10dbe8000ac60a00980a98000a980a00980a980033
:10dbf8000a980a00980a98000a980a00980a970052
:10dc08000a960a00950a94000a000000840d000094
:10dc18001c00000000000000120e000004000000bc
:10dc28000200000025630a0000000000b40d000097
:10dc38001200000002000000d80d3a0045535400bd
:10dc48003a454400543a2d00303530003000000089
:10dc5800160e00000400000000000000d80d0000af
:10dc68000e000000020000003a005400494d450033
:10dc78005a4f4e00450054005a000000e20c0000c4
:10dc8800300000000200000000001f00003c0000ff
:10dc98005b00790000980000b600d50000f4000091
:10dca80012013100014f010000001f00003b00007d
:10dcb8005a00780000970000b500d40000f3000077
:10dcc80011013000014e0100a00d000014000000f9
:10dcd80000000000c60d0000120000000200000055
:10dce800010002000004000008001000000000000d
:10dcf800202b2d0023300000fc0d00000800000040
:10dd080002000000686a6c00747a4c000000000091
:10dd1800e60d00000c00000002000000686a6c00bc
:10dd2800747a4c00006343006e5b00001a0e00001a
:10dd380004000000020000000000000000000000d5
:10dd48001e0e00000200000002000000fc2100007e
:10dd5800040e00000800000000000000620d000032
:10dd68002200000002000000303132003334350058
:10dd78003637380039616200636465006600300038
:10dd880031323300343536003738390041424300e8
:10dd98004445460000000000120d00002a00000063
:10dda800020000002b3a0000256d2f0025642f008b
:10ddb8002579000025592d00256d2d0025640000ca
:10ddc8000a002500483a25004d00090000254800b2
:10ddd8003a254d003a25530000250000680c000044
:10dde80048000000020000000000000000000000e1
:10ddf800244000000000000000005900400000001e
:10de08000000000088c34000000000000084d70024
:10de18009741000080e0370079c3410043176e0046
:10de280005b5b500b8934600f5f93f00e9034f0082
:10de3800384d32001d30f900487782005a3cbf0047
:10de4800737fdd004f157500b00c00003200000034
:10de5800020000004e414e00006e61006e00490055
:10de68004e460000696e66000030310032333400df
:10de78003536370038396100626364006566000032
:10de880030313200333435003637380039414200fa
:10de980043444500460000003c0d000026000000f9
:10dea800020000000a0008000a101000106469004f
:10deb8006f75780058700000303132003334350007
:10dec8003637380039616200636465006641420094
:10ded80043444500460000000c0e00000600000008
:10dee800020000000400000000000000200e0000f6
:10def800020000000200000000000000220e0000e6
:10df08000200000002000000300000001e0c0000ab
:10df18004a000000020000000000410029211c0006
:10df28001917160015141300121211001111100000
:10df380010100f000f0f0f000e0e0e000e0e0e0029
:10df48000e0d0d000d0d0d000d3031003233340073
:10df580035363700383961006263640065666700ea
:10df680068696a006b6c6d006e6f70007172730087
:10df780074757600777879007a000000240e000026
:10df8800020000000200000000000000260e000051
:0cdf98000200000000000000000000007b
:020000040000fa
:10dfa4007400fa002c03a8002c23a8002c43a8001a
:10dfb4002c63a8002c83a8002ca3a8002cc3a800c1
:10dfc4002ce3a8002d03a8002d23a8002d43a900ad
:10dfd4002d63a9002d83a8002da3a8002dc3a8009c
:10dfe4002de3a80085050700401f20002506070033
:10dff400416a20009140780000ccb30000c060006a
:10e004001041b300a4e6b700016d200091407800f0
:10e0140000ccb30000c060003040b300d0e6b700cd
:10e02400616a20009140780000ccb30000c0600019
:10e03400b040b300a6e6b700c16c20009140780060
:10e0440000ccb30000c060005040b300cce6b70081
:10e05400f0c2a900f4c2a800e802a900ec02a900d9
:10e06400c982a900cd82a900c9a2a900cda2a90094
:10e07400e822a900ec22a900d1a2a900d5a2a900f6
:10e08400d1c2a900d5c2a900c9c2a900cdc2a900a4
:10e09400d8c2a800d8e2a800416c200091407800c2
:10e0a40000ccb30000c060007040b300c4e6b70009
:10e0b400816a20009140780000ccb30000c0600069
:10e0c4003040b300a8e6b700216c200091407800ee
:10e0d40000ccb30000c060000034a000c2e6b7006a
:10e0e400d90607001bfc07009f060700570307001b
:10e0f400a3cd0700e4004700c0e82d00801f78008e
:10e1040050e92d00801f780010ea2d00801f780050
:10e11400010078007cd30700e6875700e40047003d
:10e1240020002000c5fc0700e400470000ec2d009f
:10e13400801f780040ed2d00801f780001007800da
:10e1440071d30700e4875700e40047002000200053
:10e15400bafc0700a0a22000520107000000e00062
:10e1640006003200c001070031ee2d00200020001f
:10e17400b2fc0700a0a220004a0107006051800001
:10e18400f5ca070070518000815180000bcb070055
:10e1940090518000a151800020cb0700b051800035
:10e1a400c151800040cb0700d0518000e151800074
:10e1b4005ecb0700f0518000015280007ecb070047
:10e1c4008ec80700000037000080eb00a2c80700db
:10e1d400640047006c000700100798001e009000c0
:10e1e400e20f500003003a00310007000000eb008a
:10e1f400100798001e0090000000e00003003a00a1
:10e204003000200010079800100037006400470019
:10e21400c1f02d006d040700000f78001e00780087
:10e22400104078000004e00003003a0020002000c1
:10e2340010079800050037004200200061d62d0029
:10e244001e007800b6040700100798001e00900016
:10e25400e30f5000dcff32001e0090000000e000dd
:10e264000f0032001e009000e20f50000c0032003c
:10e27400400520000e0040009e009000811f7800a1
:10e28400f1f02d00811f78001fd30700e4875700a9
:10e29400410520008e8040002000200067fc07001c
:10e2a400a1f12d002000200064fc0700c6ff370008
:10e2b4000400fa0010002000000f78001000200075
:10e2c400dcfc070020002000dafc0700100020001e
:10e2d40004fd07002000200002fd070001f22d00cc
:10e2e4002000200055fc0700180037001000200013
:10e2f40059c807008e80e80010002000f6fb0700d4
:10e304000000e00003003200ae4090002000200036
:10e3140012fc07008e80e80020002000eefb0700be
:10e324000000e000090032002e409000f84f500039
:10e3340003003a000000eb00000f780003003700f0
:10e34400ae4090001000200004fc07001e00e00016
:10e35400e6ff3a0010002000b6fc07002000200071
:10e36400b4fc070010002000defc070020002000a1
:10e37400dcfc070041f32d00200020002ffc0700e7
:10e384000080fa00000006000a00fa003007980036
:10e39400d0c0b300404798000000eb00100798007d
:10e3a400e500470020002000cbfb07000000e00050
:10e3b4004d0032005e409000ec4f50000a003a00dd
:10e3c40041518000809d2000808040000040eb008f
:10e3d400804878000000eb004051880020002000b5
:10e3e4004007980042003700de40900020002000e3
:10e3f400dafb07005e409000ed4f500003003a0046
:10e40400a1c0b30020002000d4fb0700de40900030
:10e414004e40900080cf50001a0032005e409000c1
:10e42400e84f50000d00320041518000f0042000fc
:10e43400808f500009003c00425180005e409000f3
:10e4440080407800809d2000000041000148780051
:10e454000200e80040518800060037004051800067
:10e464000000e00003003400405180000000e90097
:10e4740040518800be0090000040eb0080487800c6
:10e484001900370010002000100798004151800047
:10e49400809d2000808040000040eb008048780090
:10e4a4000000eb00000f78000a0037001e0078001f
:10e4b400800078003e009000008140009e007800bb
:10e4c400809d2000008040001040780000497800c2
:10e4d4001e0fe800405180009e0f1000f3ff34002f
:10e4e4000000eb00405188001e0090004007980097
:10e4f4004e0090000080fa00000006000600fa00ba
:10e50400000f78001e007800100078000000e00082
:10e5140003003200e0ff2f00200798005e00370060
:10e524001e00780010009000100798001e00900054
:10e53400e10f5000090032001e009000e20f50006d
:10e54400060032001e0090000000e00003003200cc
:10e55400d0ff2f00200798004f0037001e007800de
:10e5640020019000b0019000005a2000010020001a
:10e57400800f5100818f590003003600c0ff2f0027
:10e5840020079800440037001e00780040019000e6
:10e59400d00190004000200001002000800f5100b5
:10e5a400818f5900080036001e0078004001900059
:10e5b400d00190000052200081002000800f510003
:10e5c400818f590003003600b0ff2f002007980008
:10e5d400310037001e007800f000900060009000c9
:10e5e400e00f5000e08f5800080032001e00780051
:10e5f40060019000f0019000005a2000010020000a
:10e60400800f5100818f590003003600a0ff2f00b6
:10e6140020079800200037001e00780000099000b1
:10e62400900990009000200001002000800f51000c
:10e63400818f5900080036001e0078000009900000
:10e644009009900000e1200001002000800f51009b
:10e65400818f59000300360090ff2f002007980097
:10e664000d0037001e00780020099000b0099000ca
:10e674000053270001002000800f5100818f5900b2
:10e684000300360090ff2f00200798000200370097
:10e694000000eb00200798002e0090000080fa0094
:10e6a400000006002000fa00600f98000e80e800c9
:10e6b400a1012000c70007000e80e80081012000ae
:10e6c400ab000700000f78000e80e80040089000bf
:10e6d4009e0f5000030032000080eb00700f980082
:10e6e400290037000e80e800900078006e08900042
:10e6f400010878000e80e800900090006e089000f9
:10e70400110098000e80e800b000900020009000f6
:10e714006e09900020019800310198000e80e800f5
:10e72400d0009000400090006e09900040019800d5
:10e73400510198000e80e800f00090006000900005
:10e744006e09900060019800710198000e80e80045
:10e7540090089000000890006e099000000998004d
:10e76400110998000e80e800b0089000200890007d
:10e774006e09900020099800310998006e089000f5
:10e784005eff0700700f98007e0890000080fa007a
:10e79400000006001e00fa00500f98005e0890006a
:10e7a40056ff07000000e000030032000080eb0089
:10e7b400600f9800290037005e0890001000780070
:10e7c400000f78005e089000100090001007980079
:10e7d4005e089000b0009000200090002007980090
:10e7e400310798005e089000d0009000400090002f
:10e7f40040079800510798005e089000f0009000d0
:10e804006000900060079800710798005e0890000f
:10e814009008900000089000000f9800110f9800d5
:10e824005e089000b008900020089000200f980027
:10e83400310f98000e007800810120004c00070081
:10e84400400f98000c0107000e007800a101200081
:10e85400ae0007000000eb00600f98006e08900007
:10e864000080fa00000006001a00fa000000eb0025
:10e87400000f78000000eb0010079800e001200072
:10e88400010020002007980031079800c0032000f1
:10e89400010020004007980051079800c0032000a1
:10e8a400010020006007980071079800c003200051
:10e8b40001002000000f9800110f98006000b800bc
:10e8c400200f9800310f98000e007800810120007d
:10e8d40027000700400f9800e70007000e007800ab
:10e8e400a1012000890007000000eb000080fa006d
:10e8f400000006001a00fa00a0aa2a00000f7800ff
:10e904000000eb00100798006000b8002007980092
:10e91400310798006000b80040079800510798003c
:10e924006000b80060079800710798006000b800a4
:10e93400000f9800110f98006000b800200f980095
:10e94400310f98000e0078008101200008000700b4
:10e95400400f9800c80007000e007800a1012000b5
:10e964006a0007000000eb000080fa0000000600c7
:10e974000800fa0020079800310798000000eb0017
:10e98400000f78000000eb00100798000a00370021
:10e994001e009000800078002e009000008040004f
:10e9a400104078000000fb001e0f40001e00900085
:10e9b4000000e800100798009e0090003e009000c0
:10e9c400808f5000f2ff35001e0078000080fa00ae
:10e9d400000006001400fa0070079800010f980068
:10e9e4000e0890000000e000040034008e0890003f
:10e9f40000402000808f5000030034000080eb00b2
:10ea0400100f98003e0037000e0890000000e90047
:10ea140022002000110009000200d8000000e800d4
:10ea2400200798000000eb00000f78000000eb00c6
:10ea3400100798002c0037001e00900000004000d2
:10ea4400800078000000210000804000cf80de00bc
:10ea54003007980041079800be0090004e009000d7
:10ea6400ec00070050079800610798002e489000ba
:10ea7400804078007e009000014878007e0090007d
:10ea84000000e800700798001e0fe8000e089000d0
:10ea94009e0f100003003a000000eb00100f9800d6
:10eaa400170037003e489000804078007e009000b8
:10eab400014878007e0090000000e800700798008c
:10eac4001e0fe8000e0890009e0f100003003a008d
:10ead4000000eb00100f9800090037001e009000a2
:10eae4000000e800100798009e0090002e0090009f
:10eaf400808f5000d0ff35000000eb00100f98000d
:10eb04001e0890000080fa00000006001400fa00bd
:10eb140070079800010f98000e0890000000e000b4
:10eb2400040034008e08900000402000808f5000c4
:10eb3400030034000080eb00100f98004b003700f6
:10eb44000e0890000000e9002200200011000900d6
:10eb54000200d8000000e800200798000000eb0045
:10eb6400000f78000000eb00100798003900370010
:10eb74001e0090000000400080007800000021008a
:10eb840000804000cf80de003007980041079800e5
:10eb94001e0fe8000e0890000000e8009e0f100011
:10eba40007003d007e00900010407800204f980040
:10ebb4007e0090000000e800700798000200370013
:10ebc40000c0eb00204f98001e0fe8000e089000d4
:10ebd4000000e8009e0f100007003d007e0090003a
:10ebe40010407800304f98007e0090000000e8004c
:10ebf400700798000200370000c0eb00304f980007
:10ec04000040eb00404f98000040eb00504f98004c
:10ec14005e0090006e019000be0090004e029000d5
:10ec240080017800040078004e0007003b000700d4
:10ec34000e0890009e0f1000030035000000eb004a
:10ec4400100f9800090037001e0090000000e80033
:10ec5400100798009e0090002e009000808f5000b6
:10ec6400c3ff35000000eb00100f98001e08900051
:10ec74000080fa00000006000400fa0000002100f1
:10ec840001002000008fbe009e0078001e0090004e
:10ec9400430007000080fa00000006000c00fa00a0
:10eca4000000eb00100798000000eb00000f780054
:10ecb400140037001e00780000004000010020000e
:10ecc40020079800310798003e00900090018800ca
:10ecd4002e0090001000ba00400798002e0090000b
:10ece4001080ba00500798004e009000de0090009b
:10ecf400800078001e00900001004000100798007a
:10ed04001e0fe800f0bf2a009e0f1000e9ff360036
:10ed14001e0090000080fa00000006000200fa00c5
:10ed240030002400003b88001e00780050052000bd
:10ed3400303b8800a00a2000303b880061e7a8002f
:10ed4400000000000000000061c7bf0001c8b3005c
:10ed5400014060000004e000fbff3a000080fa007c
:10ed6400000006000800fa00000f78001107980060
:10ed740022079800330798001e007800900188004d
:10ed84009e0090003e0090008008bb009e00900012
:10ed94002e0090008088bb000080fa00000006006e
:10eda4000800fa00100798002107980090018000dd
:10edb400000f78001e0090009001880020042400b9
:10edc400003b8800ae0090002e0090008008bb003d
:10edd4003e00900050052000303b8800a00a20002f
:10ede400303b880061e7a80000000000000000003c
:10edf40061c7bf0001c8b300014060000004e00027
:10ee0400fbff3a001e007800900188000080fa00a1
:10ee1400000006000800fa00200798003107980057
:10ee24002e009000900188003e0090001000ba006f
:10ee3400000f78003e0090001080ba001007980080
:10ee44001e00be000080fa00000006000000fa0068
:10ee540040002000d400070060002000d20007001a
:10ee6400100020006403070010002000570307006f
:10ee74000000eb00550307000000eb005e030700f1
:10ee8400100020005c030700300020004f0307003f
:10ee94000000eb004d0307000000eb004b030700ec
:10eea4000000eb00490307000d00370010538000f9
:10eeb4002153800061004000e08048001053880026
:10eec400215388001253800023538000f0ff2f0049
:10eed400f1002000800f5100818f590006003e0090
:10eee4000000eb003903070080007800f00f2000d9
:10eef400808f5000edff3a000000eb003e03070056
:10ef04000080fa00000006000200fa004000200021
:10ef1400a500070060002000a300070000062000f1
:10ef2400a1000700c1fd2d002000200043f90700c7
:10ef3400a7000700000f780007003700a00f20008b
:10ef440050020700a2000700000f780081fe2d0088
:10ef54002000200039f907009e00780061806000dd
:10ef64000004e000f5ff3a00a1fe2d00200020007f
:10ef740032f907006000b80010538800215388005c
:10ef84000000eb000080fa00000006000e00fa000a
:10ef9400881f7800300798004107980052079800ae
:10efa40063079800400020007f00070088000700e6
:10efb400610060000004e000fcff3a001000200043
:10efc4000d03070030002000000307000e81e80055
:10efd4003e009000ce0090008a0007000e80e800fa
:10efe400204090000080fb00f80207000e80e8003b
:10eff400104090000080fb00f40207000e80e8003f
:10f00400104078000080fb00f00207000000eb00d5
:10f01400000f7800080037001e0078008000780098
:10f024005e009000008440000000eb00e70207004f
:10f03400004c78001e0fe8006e0090009e0f100038
:10f04400f5ff35000000eb00eb0207000000eb00c9
:10f054004f0478000080fa00000006000800fa005f
:10f06400404798001253800023538000f0ff2f0084
:10f07400f1002000800f5100818f590003003600f9
:10f084000080eb0030079800270037004e409000c6
:10f094000074a100404798004d0007006100600023
:10f0a4000004e000fcff3a00600020003e0007007e
:10f0b40010002000d002070020002000c302070037
:10f0c40010538000215380000e0178004d0007008a
:10f0d4002e4090000080fb00bc0207001e40900000
:10f0e4000080fb00b90207001e4078000080fb008e
:10f0f400b60207004e4090000000fb00b302070078
:10f104000000eb00bc020700105380002153800074
:10f1140061004000e08048001053880021538800bb
:10f124000000eb00300798003e0090000080fa00d9
:10f13400000006000600fa00100798000000eb002b
:10f14400000f78000c0037001e0078008000780063
:10f154001e00900000804000104078001e0fe80060
:10f16400beff07000000e00003003d000080eb004c
:10f1740020079800090037001e00780080007800fe
:10f184001e00900000804000104078000004e00061
:10f19400edff3a000000eb00200798002e009000dd
:10f1a4000080fa00000006000200fa00000f780058
:10f1b40010002000900207001e0078008302070060
:10f1c4000000eb008c0207000080fa00000006003b
:10f1d4000200fa00100020008702070050002000ff
:10f1e4007a0207000000eb0078020700000f7800a5
:10f1f4000000eb00800207001e0078000080fa0087
:10f20400000006000800fa00100798002107980083
:10f21400320798000000eb00000f78000f00370061
:10f224001e007800800078003e009000808040003e
:10f234001e009000804878001e009000ae009000f0
:10f244004809dd004800de0000007100c808de0047
:10f2540010079800210798001e0fe80030002000d6
:10f264009e0f1000eeff34000080fa00000006003c
:10f274000800fa00881f78001007980021079800fa
:10f284000000eb00000f78001e0090001040780092
:10f294000004e00003003a000000eb00300798008f
:10f2a400460037001e007800800078002e00900091
:10f2b40000804000104078000000fb00fbcd0700f8
:10f2c400000478001e007800800078001e00900082
:10f2d40000804000104078000000fb00f3cd0700e0
:10f2e400800f5400150032002e0090000000e8004a
:10f2f400200798002e009000104078000004e000e1
:10f3040003003a000000eb00300798002b003700a0
:10f314002e00900090407800c0c7b30080cf50000a
:10f32400f1ff3a002e0090000000e800200798004a
:10f334000000eb00000f78001b0037001e0fe800f0
:10f344001e007800800078002e00900000804000ad
:10f35400104078000004e000080032001e0078002d
:10f36400800078002e0090000080400090407800db
:10f37400c0c7b30080cf50000b003a001e007800d5
:10f38400800078001e00900000804000104078004b
:10f39400520007000000e00003003a001e0078005d
:10f3a4003007980005003700700220009e0f1000ff
:10f3b400bcff34001e007800300798003e00900027
:10f3c4004f0478000080fa00000006000600fa00ee
:10f3d40010079800210798000080eb00000f7800c8
:10f3e4000e0037001e009000104178001e007800c7
:10f3f400800078002e0090000080400010407800cb
:10f40400804f510005003a001e0090000000e80003
:10f41400100798000080eb00000f78001e0fe80032
:10f424001e007800800078002e00900000804000cc
:10f43400104078000004e000eaff3a001e0090004b
:10f444000080fa00000006000400fa00000f7800b3
:10f45400e1ff2d001e007800dcff0700000f78009c
:10f464001e00780090407800d0c2b30080cf5000d6
:10f47400050032001e00780090407800b0c2b3004e
:10f4840080cf500001003a001e0fe80011002e004a
:10f494001e007800cdff0700000f780031002e0019
:10f4a4001e007800c9ff0700000f78001e007800d6
:10f4b400104078000004e000030032000000eb007c
:10f4c4001007980002003700100020001007980071
:10f4d4001e0090000080fa00000006000400fa00fc
:10f4e400004f78001e00fb0077cd07000000e0000d
:10f4f40003003a00f0c5b3009e4f100003003a0029
:10f504001000200010079800020037000000eb00f4
:10f51400100798001e0090000080fa00000006000a
:10f524000c00fa0020079800310798004207980061
:10f534000000eb00000f7800e1ff2d002e0090008a
:10f54400a2ff0700200798001e0037001e00780065
:10f554004200dd00800078003e0090000080400002
:10f56400900078002e00900041ff070010079800db
:10f574001e0090000000e000110032001e00900008
:10f58400800078002e00900000804000e1ff2d00f4
:10f594008eff0700200798001e0078004200dd005f
:10f5a400800078003e0090000080400090009000b1
:10f5b4002e00900001000100500798000c00370055
:10f5c4001e0fe8001e0078004200dd008000780075
:10f5d4003e00900000804000100078001040780049
:10f5e4000004e000d9ff3a004e0090005007980054
:10f5f4005e0090000080fa00000006000000fa009f
:10f604000000eb00800888000000eb003008880050
:10f61400f07f24006008880084e0a90094e0a8003a
:10f6240011e1a8000080fa00000006000000fa00c2
:10f63400ba0007000080fa00000006000200fa0089
:10f64400000f78001e007800100078000080fa0097
:10f65400000006000200fa00000f78001e00780087
:10f66400640007001e007800020007000080fa0012
:10f67400000006000200fa00000f78001e01780066
:10f684006000b8003001980041019800960007001e
:10f694001e01780010019800210198000080fa00f2
:10f6a400000006000600fa00200798008e000700fc
:10f6b400008fbe002e009000100078000000e000d3
:10f6c400230032002e009000a00090001000900053
:10f6d400be0f5000ae8f58000f0036002e00900071
:10f6e40030019000c00190002e009000a000900016
:10f6f400100090003e024000ae8248000400be00ac
:10f7040002004000838048002e01900030019800e0
:10f71400410198000e0037002e0090003001900047
:10f72400c00190002e009000a000900010009000f6
:10f734003e021000ae8218000400be000200400029
:10f74400838048002e019000300198004101980008
:10f754002e0090001e01be001200980023009800a5
:10f764002e00900030039000c003900086007800c3
:10f77400a0002000000ab8006030b900050178003c
:10f78400000141006a38b90000014100820278009a
:10f794000400be000080fa00000006000200fa0027
:10f7a400000f78001e007800beff07009e0078005e
:10f7b40010002000800878001e00780030039000bc
:10f7c400c003900086007800a0002000000ab80062
:10f7d4006030b90005017800000141006a38b900c1
:10f7e40000014100820278000400be000080fa009b
:10f7f400000006000200fa00000f78001e007800e6
:10f80400a8ff07009e0078000000eb008008780045
:10f814001e00780030039000c0039000860078003a
:10f82400a0002000000ab8006030b900050178008b
:10f83400000141006a38b9000001410082027800e9
:10f844000400be000080fa00000006000600fa0072
:10f8540020079800240007000001be002e0090003d
:10f8640001002000001f4100019749001e0007000d
:10f87400be0f5000ae8f5800fcff39000080fa0024
:10f88400000006000600fa00200798001600070092
:10f89400008fbe002e009000e90f500008003600d3
:10f8a4002e009000a2002000110009000280d80060
:10f8b400010020001e0f40005e974800040037003e
:10f8c40010002000010020001e0f40005e97480039
:10f8d40005000700be0f5000ae8f5800fcff390032
:10f8e4000080fa00000006000000fa000b00070088
:10f8f400f0528000015380000080fa0000000600ee
:10f904000000fa00f8ff0700420620000300200070
:10f9140021e307000080fa00000006000200fa005c
:10f92400e2528000f052800001538000000f510029
:10f934001e0078006101b800f0528000015380007d
:10f944000200400083804800f05288000153880080
:10f954000080fa0000000600801f78000000fa0012
:10f964000000eb0030088800e05280000000e8004e
:10f97400e052880084e0a9000080fa004f0078007b
:10f98400004006000600fa00004f780011079800b6
:10f994001e009000440007000000e0000300320055
:10f9a4000000eb0020079800100037001e009000b4
:10f9b400900078001e00900010009000008040002d
:10f9c4001e4878001e009000100090008000e8009f
:10f9d4001e00900030009000808060001e009000a7
:10f9e4001100980010002000200798002e009000bd
:10f9f4000080fa00000006000600fa00000f7800fc
:10fa0400110798001e0090003b0007000000e00072
:10fa1400060032009e0078000040eb008048780029
:10fa24000000eb0020079800120037001e00900031
:10fa3400900078001e00900020009000008040009c
:10fa4400904078001e007800014878001e00900065
:10fa5400200090008000e8001e009000300090001c
:10fa6400808060001e00900021009800100020009b
:10fa7400200798002e0090000080fa000000060085
:10fa84000200fa00000f78009e0078000000eb00ee
:10fa9400a00098009e0078000000eb009000980001
:10faa4000080fa00000006000400fa00000f78004d
:10fab4001e007800100090008000e8001e0078000e
:10fac40030009000808060001e00780020009000cc
:10fad400808f500003003a001000200010079800a7
:10fae400020037000000eb00100798001e00900091
:10faf4000080fa00000006000400fa00000f7800fd
:10fb04001e007800a00090001e00780010009000f5
:10fb1400808f500003003a00100020001007980066
:10fb2400020037000000eb00100798001e00900050
:10fb34000080fa00000006000200fa00000f7800be
:10fb44001e007800900090001e00780020009000b5
:10fb5400808050001e00780030009000008060001b
:10fb64000080fa00000006000000fa00ec82a80001
:10fb740000000000e882a90000000000cc42a800b8
:10fb840000000000c842a9000000000042c2a80012
:10fb94004302a9004322a90042a2a80042c2bf0016
:10fba4003040b30042e2b7002124200091407800a5
:10fbb40030ceb30000c060008041b30042e2b70021
:10fbc40041e2a8000080fa00000006000200fa00ea
:10fbd400000f78001e0078004012880040c2bf0069
:10fbe400614060000004e000fcff3200401280002d
:10fbf4000080fa00000006000200fa00000f7800fe
:10fc04001e00e00002003200ec82a900010037006f
:10fc1400ec82a800000000000080fa00000006004a
:10fc24000200fa00000f78001e00e000020032001b
:10fc3400cc42a90001003700cc42a800000000001b
:10fc44000080fa00000006000000fa002d43a9001d
:10fc54002d63a900000e2000001988000000eb00ad
:10fc64001019880020f02000201988000000eb0003
:10fc74008019880021e3a800e002a900e402a90099
:10fc84000080fa00000006000600fa00000f780069
:10fc94001e007800200798002e009000ea0f500004
:10fca400040032002e009000eb0f500004003200dc
:10fcb40006003700a0002000401988000600370025
:10fcc400b000200040198800030037000000eb005a
:10fcd40010079800100037002023a800e402a800b1
:10fce40020c3bf00624060000004e000fcff3a0053
:10fcf400e402a90000000000e402a80020c3bf0041
:10fd0400614060000004e000fcff3200e402a9004e
:10fd140000188000100798001e0090000080fa0070
:10fd2400000006000000fa00305380000000e000ec
:10fd340001003a00ff3ffc00305380000000e8005f
:10fd4400305388000080fa00000006000000fa002a
:10fd5400305380000000e9003053880030538000a5
:10fd64000000e00001003a000000fc000080fa00fe
:04fd74000000060085
:020000040000fa
:041ff8000000fe00e7
:00000001FF
